:020000040000FA
:10000000C0070000D1060000D1000000B1060000CA
:1000100000000000000000000000000000000000E0
:100020000000000000000000000000005107000078
:100030000000000000000000DB000000E500000000
:10004000EF000000F9000000030100000D010000B6
:1000500017010000210100002B0100003501000004
:100060003F01000049010000530100005D01000054
:1000700067010000710100007B01000085010000A4
:100080008F01000099010000A3010000AD010000F4
:10009000B7010000C1010000CB010000D501000044
:1000A000DF010000E9010000F3010000FD01000094
:1000B00007020000110200001B02000025020000E0
:1000C0001FB5C046C04600F0EFFA04B00FB41FBD24
:1000D00008205A49096809580847382057490968CB
:1000E000095808473C2055490968095808474020E5
:1000F0005249096809580847442050490968095875
:10010000084748204D490968095808474C204B4981
:10011000096809580847502048490968095808479C
:100120005420464909680958084758204349096836
:10013000095808475C204149096809580847602068
:100140003E4909680958084764203C49096809582C
:100150000847682039490968095808476C20374919
:100160000968095808477020344909680958084740
:100170007420324909680958084778202F490968CE
:10018000095808477C202D490968095808478020EC
:100190002A490968095808478420284909680958E4
:1001A0000847882025490968095808478C202349B1
:1001B00009680958084790202049096809580847E4
:1001C00094201E4909680958084798201B49096866
:1001D000095808479C201949096809580847A02070
:1001E0001649096809580847A4201449096809589C
:1001F0000847A8201149096809580847AC200F4949
:10020000096809580847B0200C4909680958084787
:10021000B4200A49096809580847B82007490968FD
:1002200009580847BC2005490968095808470000D3
:1002300003480449024A034B7047000000000020B5
:10024000C0070000C00700000122D84B5A6000BF61
:10025000D74A1268002AFBD0016000BFD44A126856
:10026000002AFBD00022D14B5A6000BFD04A12684E
:10027000002AFBD07047F0B505460E46174600240D
:1002800006E0A200B158A2005019FFF7DDFF641C80
:10029000BC42F6D30020F0BD0120C043C549086030
:1002A000401048607047014601229204086890425D
:1002B00001D9102070470020FCE7F0B505460C4638
:1002C0001646002706E028462168FFF7BDFF2D1DD2
:1002D000241D7F1CB742F6D3F0BD70B505460C4611
:1002E0002E460BE0304600F075F9FF2C01D80024B3
:1002F00001E0FF3C013C012080023618002CF1D1C6
:1003000070BD0146012292044868904201D909203B
:100310007047A9484069401C01D10F20F8E7002030
:10032000F6E7FEB504462068030000F037FA05043E
:100330002B4249598B00201DFFF7E3FF0546002D96
:1003400001D02846FEBDFFF7A7FF0120C00200F044
:1003500041F9042221469948FFF78DFF002801D07A
:100360000320EFE708222146944800F06DF90028A9
:1003700006D1002192480068FFF766FF00F00CF9F3
:100380000320DFE7A768E6686068019031463846D9
:10039000FFF7A3FF324638460199FFF78EFFB20000
:1003A0003846019900F050F9002800D1CAE703202F
:1003B000C8E700F0E3F9834800688349086041E03A
:1003C00060680190E668A0680090B200009901980A
:1003D00000F03AF90746002F00D1B3E70E20B1E74D
:1003E000201DFFF760FF0546002D01D02846A9E734
:1003F0006068002807D1FFF74FFF0320800200F05C
:10040000E9F800F0C9F8FFF747FF0120C00200F04B
:10041000E1F8042221466948FFF72DFF002801D0AA
:1004200003208FE708222146644800F00DF90028D8
:1004300006D1002162480068FFF706FF00F0ACF823
:1004400003207FE700BF00207CE770B505460C461F
:10045000182D04D12068FFF764FF206002E001201E
:10046000206000BF00BF70BDF0B589B05248406940
:1004700003905248806881000398081802900398FE
:10048000000B01900121090302984018401E000B47
:1004900000900124002520462946019A00F0C4F866
:1004A0000022401E91410791069001260027304608
:1004B0003946009A00F0B8F80022401E914105919B
:1004C0000490049BDB43059AD2430698184307998E
:1004D00011430791069037490698086007984860CD
:1004E00009B0F0BD70B53448446934488568466841
:1004F000AA003146204600F0A7F8002801D00020CD
:1005000070BD0120FCE72D484068002801D0012083
:1005100000E000200546FFF7E5FF002807D0FFF7C1
:10052000BBFE0320800200F055F800F035F8FFF71D
:100530009BFF002D0ED020484669204884684768FC
:1005400021463046FFF7C9FE224639463046FFF7BE
:10055000B4FE00BF00F020F810B5184844681A48EF
:100560000460204600F0DCF810BD15480068006803
:10057000401C01D100BFFEE710480068002802D0EF
:10058000042806D101E0FFF7BEFFFFF7E5FF00BF3B
:10059000FEE700BF00BFFEE7BFF34F8F0B480C49DB
:1005A000C860BFF34F8F00BFFEE7000000E50140C9
:1005B00000E40140000600400010001000080000A8
:1005C000B8070000BC070000000000200400FA0586
:1005D00000ED00E010B50146104B1A6808460223F2
:1005E0000F4C636000BF0F4B1B68002BFBD0531CEC
:1005F00004D0904202D20A4B186101E0084B986087
:1006000000BF084B1B68002BFBD00023044C636029
:1006100000BF044B1B68002BFBD010BD0010001066
:1006200000E5014000E4014010B5202A04DB01464A
:10063000203A9140002010BD914020239C1A03468F
:10064000E3401943904010BD034610B50B439B0790
:100650000FD1042A0DD308C810C9121FA342F8D025
:1006600018BA21BA884201D9012010BD0020C04328
:1006700010BD002A03D0D30703D0521C07E000208E
:1006800010BD03780C78401C491C1B1B07D1037854
:100690000C78401C491C1B1B01D1921EF1D118463D
:1006A00010BD70477047704710B500F007F810BDD7
:1006B000014B1B68DB6818470000002019481A49E5
:1006C0007047FFF7FBFFFFF7FBFC00BD20BFFDE716
:1006D0001649174C24688C420BD1164B1B68994263
:1006E0000CD1154B154A1360186810498842EDD09B
:1006F0000AE0134880F30888124B18470F4A13602A
:1007000018680A498842E1D080F308880E49884277
:1007100004DD0E48026802210A4302605B68184744
:100720000346DFE7C0070000C0070000FFFFFFFF30
:10073000000C000014100010001000000000002049
:10074000000400206B05000000200020240500406C
:100750000D48704502D1EFF3098101E0EFF3088104
:10076000886902380078182802D1C046074A104725
:10077000074A12682C3212681047000000B5054B7A
:10078000054A9B58984700BDFDFFFFFF4B04000042
:1007900000000020001000000400000030B4744687
:1007A000641E2578641CAB4204D3635D5B00E318D0
:1007B00030BC18471D46F8E7000C00000010000090
:10100000981D002089500100F93D0000EF4F0100BC
:1010100000000000000000000000000000000000D0
:10102000000000000000000000000000F950010076
:101030000000000000000000F93D0000F93D000044
:10104000655101006B510100F93D0000F93D0000C0
:10105000F93D0000F93D0000F93D0000F93D0000B8
:1010600071510100F93D0000F93D00007751010088
:10107000F93D00007D5101008351010089510100BB
:10108000F93D0000F93D0000F93D0000F93D000088
:10109000F93D0000F93D0000F93D0000F93D000078
:1010A0008F51010095510100F93D0000F93D00000C
:1010B000F93D0000F93D0000F93D0000F93D000058
:1010C00000F002F813F0C1FF0CA030C80838241853
:1010D0002D18A246671EAB4654465D46AC4201D170
:1010E00013F0B3FF7E460F3E0FCCB64601263342C7
:1010F00000D0FB1AA246AB463343184754410100C7
:1011000084410100103A02D378C878C1FAD8520756
:1011100001D330C830C101D504680C6070470000AD
:101120000023002400250026103A01D378C1FBD803
:10113000520700D330C100D50B6070471FB5C046C1
:10114000C04613F023FF04B00FB41FBD82690249EB
:1011500081610248104470476111000001000000E5
:1011600001B41EB400B510F02FFC01B401988646FE
:1011700001BC01B01EBD0000F0B4404649465246D5
:101180005B460FB402A0013001B50648004700BF1E
:1011900001BC86460FBC8046894692469B46F0BC01
:1011A00070470000C1100000401E00BF00BF00BF1C
:1011B00000BF00BF00BF00BF00BF00BF00BF00BF37
:1011C00000BFF1D17047000070B505460C461646C9
:1011D00002E00FCC0FC5103E102EFAD2082E02D31B
:1011E00003CC03C5083E042E07D301CC01C5361F2E
:1011F00003E021782970641C6D1C761EF9D270BD45
:101200008307FF22DB0E9A408907090E99400028C8
:101210000BDA0007000F0838830828489B001B18CA
:10122000D86990430843D8617047830824489B00DD
:101230001B181868904308431860704710B504469F
:1012400000210120FFF7DCFF00211820FFF7D8FF65
:1012500000210B20FFF7D4FF02211920FFF7D0FF58
:1012600002210D20FFF7CCFF02210E20FFF7C8FF5F
:1012700002210F20FFF7C4FF0221C81FFFF7C0FFA4
:1012800003211620FFF7BCFF03211520FFF7B8FF4D
:10129000204600F019F8002010BD6321018070473E
:1012A00010B500F03AF810BD0648704710B500F0D0
:1012B00035F810BD704770477047000000ED00E042
:1012C00000E400E003F900C330B50446374D95B0A3
:1012D00007202870A81CFFF7E0FF5920A880344899
:1012E00001F03AFC0546072000F0DCF929462F48BA
:1012F00000F08CFA641E072C0AD830216846017071
:10130000047101F0FAFA002802D009A800F0DDFC0F
:10131000284601F083FE15B030BD7047F8B5234E66
:101320000446B61E307801270D46002807D0204617
:1013300060380B2808D8204601F0B8FB2BE0602C61
:10134000F9D01C480860F8BD20466C38032803D843
:10135000204601F0EDFB1EE0204670381F2803D820
:10136000204600F037F816E0204690380F2803D8C2
:10137000204600F0BBF80EE02046A0380F2803D826
:10138000204600F023F906E02046B0380F2804D8A4
:10139000204600F000F9286000E02F60602CD2D1D8
:1013A00028680028CFD13770F8BD00001A0000204F
:1013B000C533000001300000704770477047704728
:1013C000704770477047704710B5012801D100F091
:1013D00042FA10BD10B57038030013F0F3FE150C7F
:1013E00012161E22252C33383D41454950555C6468
:1013F0006C747B8085004A680878114603F0C3FF4F
:1014000010BD086804F027F810BD0C790B7B8A68C2
:101410000868214604F02FF810BD086804F0A5F80C
:1014200010BD03F06DFC10BD08884A6880B21146FB
:1014300004F06AFA10BD0A790888114680B204F0F7
:10144000B6FA10BD087840B204F0C1FA10BD0888A1
:1014500080B204F0DDFA10BD086804F0ECFA10BDAB
:10146000086804F0FFFA10BD086804F028FB10BDFE
:10147000088982B209C9194604F050FB10BD05C99C
:10148000114604F0A4FB10BD08884A6880B21146DA
:1014900004F0BDFB10BD0B7908888A6880B219463C
:1014A00004F011FC10BD0B7908888A6880B21946D7
:1014B00004F0CAFC10BD08884B688A6880B21946DF
:1014C00004F008FD10BD08884A6880B2114604F097
:1014D00053FD10BD088880B204F072FD10BD08886D
:1014E00080B204F092FD10BD012010BD10B59038FF
:1014F000030013F067FE09060F161D242C363F4625
:101500004E0088888A6883B20888194680B205F040
:10151000ADF910BD08884A6880B2114605F003FA9B
:1015200010BD08884A6880B2114605F047FA10BD20
:1015300008884A6880B2114605F07DFA10BD088817
:101540004B688A6880B2194605F0AEFA10BD08896A
:1015500082B2888883B20888194680B205F0E3FA1F
:1015600010BD08894B6882B20888194680B205F020
:1015700018FB10BD08884A6880B2114605F048FB88
:1015800010BD888882B20888114680B205F0DCFB65
:1015900010BD012010BD10B5B02805D0B12808D06D
:1015A000B2280BD0012010BD088880B205F0BAFE29
:1015B00010BD088880B205F0E5FE10BD08884B68B4
:1015C0008A6880B2194605F0EEFE10BD10B5A0384D
:1015D000030013F0F7FD0B070E172028323C434D94
:1015E000545D65004B6808788A68194607F01FFA51
:1015F00010BD88888A6883B20888194680B207F0CF
:101600002BFA10BD08884C68CB688A6880B22146E6
:1016100007F032FA10BD08884B688A6880B2194614
:1016200007F04CFA10BD8888CB6884B208888A68B5
:1016300080B2214607F06CFA10BD8888CB6884B26E
:1016400008888A6880B2214607F08CFA10BD0888A5
:101650004A6880B2114607F0C0FA10BD088982B20C
:10166000888883B20888194680B207F0C0FA10BD96
:1016700008884A6880B2114607F0DDFA10BD088973
:101680004B6882B20888194680B207F05AFB10BD39
:1016900008884B688A6880B2194607F017FC10BDAD
:1016A000012010BD10B507F0FEFC0FF0A7FF00F001
:1016B00007F810F0F5F808F013FA08F09FF910BDDC
:1016C00001202B49C00308602A490020087003202C
:1016D0002949800288607047F8B5264D044628786D
:1016E000A04207D0002C05D0002803D023A14D2014
:1016F00013F077FC2878A04213D02C700325002328
:101700002349AD021C48002C27D01B4A214E4032F1
:10171000214F012C06D0022C13D018A16E2013F0FB
:1017200060FCF8BD0B6002230B604E6185601B49B5
:1017300011625762091D91621749091DD162456006
:10174000F8BD0B6003230B604E610121C90281606B
:10175000134B9362D7624160F8BD0B600B608560EC
:10176000F8BD10B505A1772013F03BFC10BD0000BB
:1017700080E100E02000002000F501407372635C0E
:1017800068616C5F63636D5F6161722E630000006E
:1017900000F500407C01002000F0004000110040F6
:1017A000488100401CB50446002069460870204668
:1017B00009F014F96946204608F0D2FF002803D149
:1017C000FBA1B62013F00DFC01A9204608F027FF6D
:1017D000002803D1F6A1BB2013F003FC6846007873
:1017E0001CBD70B5F74D002428462C76203084713E
:1017F000C47113F0F5FC284640380470203084731F
:10180000847484762C74AC7070BDEAE710B50C4615
:10181000ED4982888A8042884A80007808700846AC
:101820000A38847008F0D1FEFFF7DBFF20460AF08B
:1018300039FAE44AE032114638390846144681380C
:1018400009F03AF92146E0480BF0CEFC09F0BDF86A
:1018500013F0C6FC10BD10B50120FFF7ADFD10BDA3
:10186000F8B509F093FDD84DD64C0A3D022802D0B8
:10187000207C00287CD0207E0026102819D1A0785A
:10188000002803D0CAA1D14813F0ABFBCD48E838FB
:10189000817A89070DD50146267160398989E180F1
:1018A000C17A217281896181C089A0810120A070E3
:1018B0002676C44F203FB87C002859D1C4486946D9
:1018C000808908F04DFF002805D0694668780978BE
:1018D0004018687004E06B20B5A1000113F081FB93
:1018E000207C002838D0BA488189FF300930406D0B
:1018F0008089814204D0B548ADA1223013F071FB3C
:10190000B348808908F0D2FF002804D1AF48A8A1CD
:10191000283013F066FB09F040F800281CD0AC48D2
:101920008089FFF73FFF697840186870A548403804
:10193000416D20318A7C012A0DD1A54A3E779289DA
:10194000C287C87C20700120B876207E102801D084
:10195000282800D1267626746978002908D09C486A
:101960008289FF300930C28601870120B8746E7009
:1019700009F0DCFC002805D1207C002802D0A878E2
:1019800001F00EF9F8BDF8B50F460446FFF768FF01
:101990008C4D403D28788B4E002813D0002F10D15D
:1019A000307E002804D0FF2081A1C93013F019FB3C
:1019B0002C22A91C204613F077F90E20207000205D
:1019C00028708FE07F4D203DA87B002818D0002F85
:1019D000F7D1307E102808D0282806D0002804D05F
:1019E000FF2073A1D53013F0FCFA0120E070E87BF2
:1019F000A070287C60700F2020700020A87371E018
:101A00000121204609F002F8002807D0307C002888
:101A100052D13946204608F0F9FFF8BDA97C694843
:101A20000C38009068480A38002913D0017805293D
:101A300010D2002F56D1491C0170002666700D206F
:101A40002070012028750622A01C009913F02CF9A3
:101A5000AE7447E05C4800210A380170B078002875
:101A600015D0002F3ED1307E002804D0432050A155
:101A7000C00013F0B6FA00256570012051492070AE
:101A80000A22091DA01C13F00FF9B5702AE039468F
:101A900020460BF013FB002824D1A87C002805D099
:101AA000002F1FD148480A380178C4E7A87E0028D3
:101AB00002D0307C002801D00020F8BD002F11D1C9
:101AC000307E002803D03AA1424813F08AFA00265B
:101AD00066700A203B4920700622091FA01C13F0E3
:101AE000E3F8AE760120F8BD10B53648017E002936
:101AF00008D1007C012805D001210020FFF743FF19
:101B0000002801D0072010BD012010BD10B5012410
:101B10000AF010F90443FFF7E7FF044308F056FF0B
:101B200001462143084610BDF8B51D4614460E4631
:101B300008F095FD002807D0684608F09BFD0028B6
:101B400003D0002C07D101E00120F8BD214818A1E5
:101B5000303013F046FA08F039FDA04204D22720B5
:101B600013A1000113F03DFA009808F0A7F93146DF
:101B7000009808F0B5F9E2B22946009808F06CFB2D
:101B800008F08AFD002804D1124809A1403013F062
:101B900028FA08F01DFF0E4800244030417C00293F
:101BA00002D044740AF0B1F90948C480CCE70000BF
:101BB0007372635C6C6C5F6374726C2E73302E6333
:101BC00000000000200300202C00002093060000ED
:101BD000D80100203F02000010B50179002908D08B
:101BE00001290BD0FF20FD49043013F0FAF9002041
:101BF00010BD831D42880488022103E042880488C6
:101C0000831D01212046FFF78FFF10BDF8B51F4649
:101C100015460E46044609F0B9FB022803D0F048E9
:101C2000007C00281FD0EF488089208008F03EFE0D
:101C3000002803D1E949EC4813F0D3F9052468469C
:101C400008F03FFE00280ED0009808F081F93070AF
:101C5000022809D0012807D008F073FE641E24066C
:101C6000240EECD10020F8BD3946009808F00CFB9A
:101C70002880002804D1DC48D849123013F0B1F98B
:101C800008F05FFE002804D1D748D449193013F07A
:101C9000A8F90120F8BD38B50446831D821C6946A9
:101CA000FFF7B4FF00280DD000206071684600786F
:101CB000012808D0022806D0FF20C849253013F09B
:101CC00090F9012038BD2071FBE700215BE670B57B
:101CD000C34C0546403C2078002803D1C048007E14
:101CE000002803D0BD49C14813F07BF903CD07F0AC
:101CF0005DFA00202071012060713D21E1702070AB
:101D000070BD70B5B64C0546403C2078002803D124
:101D1000B348007E002804D0B448B0490D3813F011
:101D200060F9287808F083FF28780BF0A8FB0020E2
:101D30002071012060713921E170207070BD70B593
:101D4000A74D0446403D2878002803D1A448007ED2
:101D5000002804D0A548A149253813F042F9A14E26
:101D60002188B089884203D109F010FB022807D0EE
:101D700002202871012068713821E970287070BD37
:101D80007F2070769748E17820304174A178017403
:101D90000020EEE710B5924C403C207800280BD193
:101DA0008F48007E002807D109F0F0FA032803D0FD
:101DB00009F0F0FA032804D18B488849653013F004
:101DC00010F9874900202031C8712071012060710D
:101DD0003A21E170207010BD70B5814C0646403C40
:101DE000207800280BD17E48007E002807D109F01A
:101DF000CDFA032803D009F0CDFA032804D16520D9
:101E00007649C00013F0EDF8754D2035E8790828C3
:101E10000CD2E8791022000100196830314600F038
:101E20002DFEE879401CE871002000E007202071B9
:101E3000012060713B21E170207070BDF8B5684DE4
:101E40000446403D2878002803D16548007E0028DC
:101E500004D0664861495F3813F0C3F8614F2188A8
:101E6000B889884203D109F091FA022801D00220F2
:101E700022E03E8C64887200788CF98B521C94426C
:101E800017D35B4A51439200504312F087FF401E24
:101E9000FF2180B2F531884200D90846844200D241
:101EA0002046711C401C12F079FF761C7043401EC6
:101EB00086B2FE85EE8000202871012068713C21E9
:101EC000E9702870F8BDF8B5454C0546403C2078CF
:101ED000002803D14248007E002804D043483F49EF
:101EE0008B3813F07EF8A878002801D0012804D19F
:101EF000A888FF21F531884204D93C483749853804
:101F000013F06FF8374E2988B089884203D109F061
:101F10003DFA022807D0022020710120607136218D
:101F2000E1702070F8BD2F48002720308772A98803
:101F3000B18501213176A978012900D00021817273
:101F400028484030407C002801D009F0DEFF27718E
:101F5000E3E770B5224C0546403C2078002807D1C5
:101F60001F48007E002803D109F010FA002804D091
:101F7000AD201A49C00013F034F8287809F0DDFECE
:101F800000202071012060713021E170207070BD4F
:101F900070B5134C0546403C2078002803D110480A
:101FA000007E002804D011480C490C3013F019F8B9
:101FB000287800280BD0012809D0022807D068789B
:101FC000402804D309480549133013F00AF828467D
:101FD00009F0D3F900280DD000200CE0B01B000060
:101FE00020030020D8010020AD0200001A060000E6
:101FF000C40900000C202071012060713421E170BF
:10200000207070BD70B5FF4C05462078002808D1BF
:1020100020464030007E002803D109F0B7F900289F
:1020200003D0F949F94812F0DCFF2978002914D0CF
:102030000A2912D0142910D01E290ED028290CD01C
:1020400032290AD04B2908D0642906D0FF2904D0B0
:10205000EE48ED490E3012F0C4FF284609F0ECFEC0
:1020600000202071012060713321E170207070BD6B
:1020700070B5E44C06462078251D002804D1204682
:102080004030007E002804D0E048DF49203812F0BC
:10209000A8FF3146002008F09FFD2870002804D1D9
:1020A00006223146DA4812F0FFFD0120607132212C
:1020B000E170207070BD70B5D24C054620780028C4
:1020C00004D120464030007E002804D0CF48CE49BD
:1020D000383812F086FF00216956042914D00029EF
:1020E00012D0081D10D0001D0ED0001D0CD0001DF8
:1020F0000AD0001D08D00A3006D0283104D0C348C9
:10210000C149363812F06DFFC248297801700120AC
:1021100060713121E170207070BD10B5B94C20782C
:10212000002804D120464030007E002804D0DF2063
:10213000B549C00012F055FF08F048FAE08008F0F9
:102140000DFB207200202071012060710521E170DB
:10215000207010BDF8B5AB4C07462034A07B254657
:102160002035002805D1287E002802D1A878002833
:1021700004D0A648A449623812F033FF09F006F9EA
:102180001026022822D1A4483988808988421DD18E
:102190009C49483908460A7F6038807A002A03D073
:1021A00080070CD40C200CE0800708D406200877A8
:1021B00099484030407C002801D009F0A6FE2E76D8
:1021C0000020E07326740120A073F8BD0220F8E718
:1021D00010B58C4C2078002804D120464030007E79
:1021E000002804D089488849743812F0FAFE00208B
:1021F00020710E20A0700F20E070FF20A071002041
:10220000C04320818248C01D0178A1728188A181CC
:102210004088E08101206071207010BD10B5794CBC
:102220002078002804D120464030007E002804D0C9
:10223000DF207549800012F0D4FE0821A01D0FF0A8
:1022400079FA00202071012060712B21E17020704B
:1022500010BD70B56B4D04462878002804D128467F
:102260004030007E002804D019206749800112F018
:10227000B8FE694810222146303800F0FFFB66485E
:102280001022A118203800F0F9FB634830380FF015
:1022900058FB6149102210392C46A81D00F0EEFBB6
:1022A000002020710E20A0702A20E07001206071B3
:1022B000207070BDF8B5534C05462034A07B2646EF
:1022C0002036002802D1307E002803D04E495348E2
:1022D00012F087FEA978052912D0132910D01429ED
:1022E0000ED015290CD01A290AD0292908D03D2949
:1022F00006D03B2904D049484349083012F071FE0A
:1023000028884749884204D944483F49113012F08F
:1023100068FE09F03BF80C212827022809D13E4825
:102320002A888089904215D136484838027E002A92
:1023300001D0E17310E0A97841760121017637766A
:102340000020E07334484030407C002804D009F07D
:10235000DCFD01E00220E07327740120A073F8BDCA
:10236000F8B5284F064638783D1D002804D1384678
:102370004030007E002804D028482349163812F047
:1023800030FE3146012008F027FC01242870002887
:1023900007D11C48062260303146054612F084FC05
:1023A000AC717C711720F8703C70F8BDF0B5194F16
:1023B00085B0403F3D7A064612480078002804D197
:1023C0003846A038007E002803D00F49154812F087
:1023D00008FE3078002806D0012804D035200A49AC
:1023E000000112F0FEFD082D4CD20A482038019061
:1023F000C469307800283FD0012817D00948024925
:102400000F3011E0E0020020B01B00007505000055
:102410002500002000040020D801002063040000F3
:10242000FF0E00004F03000012F0DBFD29460831CB
:102430000120884004430120A84020430090B17946
:102440007279080210436900FE4C0919FF3101310D
:102450008881B01C12F089FC717800020843A90041
:102460000919C031C862387A401C38720199009845
:10247000C8610020207108E0294608310120884009
:102480008443D8E7EF48072101710121ED480B2271
:102490004171C270017005B0F0BD10B5E94C2078F3
:1024A000002804D120464030007E002803D0E649B1
:1024B000E64812F096FD12F093FE002020710120F4
:1024C00060710A21E170207010BD10B509F0CDFBDC
:1024D000002804D0DD48DC49583812F082FD08F0AD
:1024E00073FA08F056F80AF070FE002804D0D748B6
:1024F000D5494A3812F075FD08F0B5FA002804D025
:10250000D248D149463812F06CFD12F069FED0482D
:1025100000240470FFF765F9CA4801210471417174
:102520000222C270017010BD70B5C64D04462878F5
:10253000002804D128464030007E002804D03D20E9
:10254000C149000112F04DFD20781F2801D8601C00
:1025500004D1BE48BC49903012F043FD00202871E0
:102560002078611C08F052FB012068712021E9707D
:10257000287070BDF8B5B34C064620782546403526
:10258000002802D1287E002804D0B048AE499D30F2
:1025900012F027FD3078012806D0002804D0AB487F
:1025A000A9499E3012F01DFD012060710C202071A0
:1025B00030780027A74E012808D008F0E7FE03284E
:1025C00069D008F0E7FE032873D078E008F0DEFE5B
:1025D000002803D108F0DEFE002804D008F0D6FE63
:1025E00002283DD06BE008F07DFA002867D0287CF7
:1025F000002864D1974802210C300FF024F80028FD
:1026000006D00F21B089090212F0C8FBB18100E0A9
:10261000B781012203218F4807F05EFE8D4808F044
:1026200003FCB08907F0D4FF002804D1874886490D
:10263000B93012F0D6FCB089002108F0CDF900289D
:1026400004D082488049BD3012F0CBFC297F688BD2
:1026500009F077FB002831D07C487B49C13017E076
:1026600008F098FE00282AD1287F002827D00128CA
:1026700025D0042823D008F035FA00281FD0297F60
:10268000688B09F05EFB002818D070486E49D53081
:1026900012F0A7FC12E0002009F086FA00280ED103
:1026A0002771287C00280AD1B089FFF77BF806E063
:1026B000FFE7002009F078FA002800D127711B20DD
:1026C000E07001202070F8BD70B55E4D044628789A
:1026D000002804D128464030007E002804D05B4802
:1026E0005949813012F07DFC20781F2801D8601CE8
:1026F00004D156485449823012F073FC00202871EE
:102700002078611C08F096FA012068711A21E9709E
:10271000287070BDF8B54B4D044628780C272E461E
:10272000403600280AD1307E002807D108F02EFE5E
:10273000032803D008F02EFE032804D1712042495B
:10274000C00012F04EFC6079002801D0012829D188
:10275000A079002801D0012824D1A07B002805D031
:10276000012803D0022801D003281BD1607B400739
:1027700018D0628801208003824202D821888142D9
:1027800001D920790CE02079002804D0022805D056
:10279000032803D004E0202A12D20CE0A0290FD293
:1027A00001280DD02079042805D12088202802D3C3
:1027B0006188884204D9254823495D3012F011FC14
:1027C00020887083207930776079002802D0012832
:1027D00003D00CE0204A002105E01A4A60329079CB
:1027E000002804D00121204608F080F90746012086
:1027F0002F7168711821E9702870F8BD70B5114CFF
:1028000005462078002804D120464030007E00286C
:1028100003D00D49114812F0E4FB08F0B7FD0C217C
:1028200002280ED10B482A8883899A4228D1024671
:10283000C032137F002B04D1807E0E2812D00F28C7
:1028400010D00DE0E0020020B01B000041030000AA
:1028500000040020D801002025000020D60400003C
:10286000217103E005201077002020710E20A07058
:102870002E20E0702888E08001206071207070BDFB
:102880000220F2E770B5844C05462078002804D178
:1028900020464030007E002803D08049804812F056
:1028A000A0FB08F073FD0C2102280ED17D482A8878
:1028B00083899A421FD10646C036327F002A04D14E
:1028C000807E0E2803D00F2801D0217109E07248C4
:1028D0001022A91C1E3812F0E7F9042030770020DE
:1028E00020710E20A0702D20E0702888E08001204B
:1028F0006071207070BD0220F2E710B501780B0006
:1029000012F060FC3E8B8B388B8B588B8B8B8B3B08
:102910003E8B8B8B51548B8B8B8B8B8B42288B2CD0
:10292000308B8B8B8B348B8B8B8B8B8B8B468B4A2F
:102930004E8B20248B6B5B5F63678B6F8B7E827B00
:102940007773868B001DFFF79DFF64E0001DFFF786
:1029500055FF60E0001DFFF7DDFE5CE0001DFFF7A6
:10296000B3FE58E0001DFFF705FE54E0001DFFF721
:10297000DBFD50E0FFF7A9FD4DE0FFF78EFD4AE0DB
:10298000001DFFF713FD46E0001DFFF7E9FC42E0E4
:10299000001DFFF78FFC3EE0001DFFF75AFC3AE0F8
:1029A000FFF73CFC37E0FFF713FC34E0001DFFF7B6
:1029B000D1FB30E0FFF7B1FB2DE0001DFFF77BFB03
:1029C00029E0001DFFF754FB25E0001DFFF71AFB6F
:1029D00021E0001DFFF7DCFA1DE0001DFFF7B9FA4A
:1029E00019E0001DFFF76FFA15E0001DFFF726FA4A
:1029F00011E0001DFFF7F0F90DE0FFF7CBF90AE059
:102A0000001DFFF79CF906E0001DFFF77AF902E0D0
:102A1000001DFFF75CF9012010BD002010BD10B5AE
:102A20001E49214812F0DDFA10BD70B51A4A012482
:102A300011461C4D4031030012F0C4FB05191C1C4B
:102A400004191C0001220021164807F045FC124819
:102A50000021483801774177C03809F0EEF90028A5
:102A600004D011480D49D33012F0BBFA70BD0C747C
:102A7000556570BDEB200949C000F5E730B5134638
:102A800006E0CC18203CE47FD51A44555B1EDBB22F
:102A9000002BF6D130BD0000E0020020B01B00008A
:102AA000AA040000D80100205206000010B56038CA
:102AB000030012F087FB0A060A0F13181F262A319B
:102AC000363B086800F073FD10BD05C9114600F0E3
:102AD0008DFD10BD086800F027FE10BD05C9114628
:102AE00000F02BFE10BD4B6808788A68194600F08C
:102AF00036FE10BD4B688A680868194600F04AFE29
:102B000010BD086800F05FFE10BD08884A6880B2FA
:102B1000114600F07BFE10BD05C9114600F0A6FE6F
:102B200010BD05C9114600F0BDFE10BD012010BD4D
:102B30000120704701203F49400608603E49086077
:102B40003E490A68FF231B029A4383121A430A6014
:102B5000384980390860704710B50246042038496A
:102B600004E0C3005B181B79002B0AD00346401E0B
:102B7000C0B2002BF5D133A1432012F032FAFF206E
:102B800010BDC300CA50002259184A718A7101222F
:102B90000A7110BD2A4A0021C000801801717047D7
:102BA00010B50446042803D326A1522012F019FAC6
:102BB0002348E1000C182079012803D021A15320DB
:102BC00012F00FFA6079A179401CC0B2814200D0A6
:102BD00060710120174940068031086010BD70B552
:102BE000164800680004800F022803D015A1692050
:102BF00012F0F7F9124E194C03252078C1008819FC
:102C00000279012A07D1427983799A4203D0427925
:102C10008271705880472078401CC0B22070042810
:102C200001D30020207028466D1EEDB20028E4D1AB
:102C300070BD000080E100E080E200E018E400E008
:102C40002C1200207372635C736F635F7369676E2D
:102C5000616C6C696E672E63000000003C00002010
:102C600010B5EFF31080C407E40F72B6D648417870
:102C7000491C41704078012801D10FF04BF9002C1C
:102C800000D162B610BD70B5CF4CE07800280AD1F3
:102C90000125E570FFF7E4FF0FF044F9002804D0A8
:102CA00000200FF017F9002070BDC848657145601D
:102CB000F9E770B5EFF31080C507ED0F72B6C24C9F
:102CC0006078002803D1C2A18F2012F08AF96078C1
:102CD000401E60706078002801D10FF01FF9002DB0
:102CE00000D162B670BD10B5B748C178002904D0D4
:102CF00000214171C170FFF7DCFF002010BD10B54D
:102D000004460FF00FF9B049C978084000D00120FF
:102D10002060002010BDF8B50246AB4C0026A6711D
:102D20000820042101251027130012F04BFA0D088A
:102D30000A0C0E101214161E2621232528002571B8
:102D400022E0022001E021711EE020711CE02771C9
:102D50001AE02020F9E7012616E0FFF781FF0FF0C7
:102D6000E1F80028FBD002260EE02171A5710BE0EE
:102D70002771FBE7202000E040202071F6E7FF20CC
:102D800093A17E3012F02DF90FF0D8F8002809D069
:102D90000FF0DAF8B04205D130460FF0D8F800282D
:102DA000FAD024E001208007C5608D4A00215160DF
:102DB0008C4A9661854B02225A6085608A48036975
:102DC0000569DB43DB06DB175B1C10273D43056110
:102DD000834D00E020BF6F68002FFBD0002B03D194
:102DE000076910239F430761784882606960A07972
:102DF00000280CD00FF096F805460EF0F3FF7B4A42
:102E0000002D02D0A260E06001E0E260A060002E30
:102E100001D100F0B1F8F8BD10B504460FF088F804
:102E2000002805D068490120C8704A78521C4A70B1
:102E30002046FFF770FF10BDF8B5694FB868002550
:102E4000012802D1BD600FF045F87868012800D153
:102E50007D60386801265C4C012814D13D606079A2
:102E6000002803D000200FF035F865712078002885
:102E700009D00FF057F8002805D05948C0388663AC
:102E800000060661A670386901282CD13D6100F06A
:102E900068F8012080074661A079002815D00FF05E
:102EA00041F800900EF09EFF0099002901D0E168E2
:102EB00000E0A168411A022901DA8A1C13DC00999A
:102EC000002901D0E06000E0A060FFF7C9FE0FF02C
:102ED00029F8002806D04248C038866300060661FB
:102EE000A67000E02670F868012819D100F039F8C2
:102EF00000F037F800F035F8A078002804D1FF2062
:102F000033A1053012F06DF8FD60A5702570FFF754
:102F1000D0FE0EF0DEFA002802D03148C038C66379
:102F2000F8BD10B5284CE078002801D10EF0F6FF6E
:102F300001208107886100F014F8A07800280BD0E8
:102F4000274CE068002803D10FF001F80028F8D1E1
:102F50000020E06000F005F800201C49C0438860B4
:102F600010BD08B55020694608806A461088411E89
:102F700011800028F9D108BDF8B5144819278760D9
:102F8000174900200860C8600EF0CCFFBD0701247F
:102F90000D4E002805D01248C03884632C61B470EF
:102FA00000E03470FFF75CFE084847600D49307957
:102FB0008863FFF7D6FFAC61FFF7D3FF0849002015
:102FC00008616C61F8BD0000400000200003004073
:102FD0007372635C736F635F636C6F636B2E63000C
:102FE000000100400005004000ED00E0FFFFFF7F12
:102FF00010B504460BF08FF820460CF0A4F810BD75
:1030000010FFFFFFDBE5B151006001006300FFFF2F
:1030100003B40148019001BD09000020FE49487039
:10302000704710B5030012F0CDF8080E050E080821
:103030000B0B0E1104F09BF810BDFFF7D9FF10BD6C
:103040000DF0E8FF10BD01F0A7FE10BDFF20F3A1B9
:10305000AF3011F0C6FF10BD7FB5F4490546486892
:103060008968082301910090F14A1946F1480EF051
:103070008BFD0024F0480EF0A5FD641CE4B2082C82
:10308000F8D3EB490320803140020CF031F90028DD
:1030900003D0E2A1D42011F0A4FF1E220221E748B0
:1030A0000AF0E9FCE5481E22032110300BF05DFA1E
:1030B000E2480722342174300AF036FCDF484C2104
:1030C000283011F050FEDD496A46743108464C380C
:1030D0000164FF317B31416401211172039002F0E0
:1030E000DAF802A80CF052FC002803D0CBA1E820AB
:1030F00011F077FFCF4802222421A8380AF014FCEF
:10310000CC4802222C215C380AF00EFCCC490B2062
:103110000EF082F8002803D0C0A1F52011F061FF65
:1031200004F00EF803F012FA04F06EFE6B46002273
:103130000821C4A001F09EFF002803D0B7A1FC2005
:1031400011F04FFF284605F079F9002803D0B3A10C
:10315000FE2011F046FF8521C900BD4811F003FE95
:10316000BB49B24A0020135C0C18401CC0B2E3708B
:103170000428F8D3A849002048608870C8707FBD33
:1031800070B5B44E0546706A94B00C46401C04D12C
:10319000B06AC0430004000C0BD0306AC007C00FF7
:1031A0002870706A11F0F2FDB06A2071000A607137
:1031B00014E02B206946087009A968460AF0FAFB5A
:1031C000002804D0FF2095A1233011F00AFF012030
:1031D000287006220AA9204611F066FD28780028EA
:1031E00003D06079C0210843607114B070BDF0B5A0
:1031F000984C0646206895B00D463746401C083767
:10320000002808D16068401C05D1A068401C02D18C
:10321000E068401C11D02068314611F0B7FD6068AD
:10322000311D11F0B3FDA068394611F0AFFDE06823
:1032300031460C3111F0AAFD25E02B2069460870BB
:1032400009A968460AF0B6FB002804D0FF2073A144
:103250004C3011F0C6FE08220AA9304611F024FDB8
:103260002B206946087009A968460AF0A3FB0028CC
:1032700004D0FF2069A1533011F0B3FE08220AA93F
:10328000384611F011FD20692E46401C08360028F2
:1032900008D16069401C05D1A069401C02D1E069D9
:1032A000401C12D02069294611F070FD6069291D6B
:1032B00011F06CFDA069314611F068FDE069294606
:1032C0000C3111F063FD15B0F0BD2B24684604707D
:1032D00009A90AF06FFB002804D0FF204FA171302C
:1032E00011F07FFE082209AF0AA9284611F0DCFC84
:1032F0006846047009A90AF05DFB002804D0FF208D
:1033000046A1783011F06DFE0822391D304611F0CB
:10331000CBFCD8E710B5002108460EF00BFD0021CC
:1033200001200EF007FD002102200EF003FD002118
:1033300003200EF0FFFC002104200EF0FBFC002116
:1033400005200EF0F7FC10BD10B5414CA0780B28FD
:1033500004D3FF2031A1C83011F043FE2078602152
:10336000484300190830002101704178E722C9085C
:10337000C900C91C11404170274A0121917010BD3C
:1033800070B5254CA07800280ED031480025017872
:10339000491CC9B201700B2900D105708178491C04
:1033A00081700EF092FDA57070BD70B51A4C054687
:1033B0006068002804D0FF2018A1F13011F011FE40
:1033C000656070BD70B5144E214DFFF7BDFF71688B
:1033D0000446002907D06022FDF7F6FEFFF7D0FF74
:1033E00000207060F1E72879002876D011485C3819
:1033F0000AF0AAFA6060002803D108A1164811F06B
:10340000F0FD60680AF0FEFA002833D0204600F094
:1034100070FF6078010721E0340000207372635C64
:10342000686F73745F636F72652E6300F051010003
:10343000040400200C12002023300000840A002025
:10344000B41000206E524635313832320000000090
:103450008C0C0020800000100E02000007D5C00870
:10346000C000401C60702879401E287126E0F74893
:10347000616829E0F54861680AF06FFA6879002808
:103480002BD0F2484C380AF05FFA6060002803D174
:10349000EF49F04811F0A5FD60680AF0B7FA00287E
:1034A00016D0204603F0A2FE6078010709D5C008B7
:1034B000C000801C60706879401E6871FFF760FF73
:1034C00083E7E24861684C380AF047FA7DE704E098
:1034D000DE4861684C380AF040FA70BDF7B5054621
:1034E0000078002700090C463E46062804D0D9483B
:1034F000D749223011F075FD287A00280ED0012816
:1035000014D09D20D249800011F06BFD0298002C50
:10351000068001D0278066800020FEBD0227092694
:10352000002C0ED0A889A080A87B08E003271426D1
:10353000002C06D02869E060A88A2082287B2072AF
:10354000E4E702980680E7E770B50E4600211C46C6
:1035500019801546030011F035FE0723050B1711DE
:10356000231D230022462946304603F00BFE70BD82
:1035700022462946304601F080F970BD2246294690
:10358000304604F03CFB70BD22462946304603F02D
:1035900011F870BD224629463046FFF79FFF70BDE7
:1035A000AC48AB49693011F01CFD032070BD10B56B
:1035B000A94C2178002901D0082010BDFFF74CFD4F
:1035C00001202070002010BD0146A04810B54C38E5
:1035D0000AF0C3F9A1494879401CC0B248710128DA
:1035E00003D19D484078FFF7DBFA10BDF8B50546DA
:1035F0009B480F46814208D3002D01D0854204D359
:10360000E81C80088000A84201D01020F8BD934833
:103610008178002911D03988009141786022514386
:103620000C18083420783B460007000F0022214682
:10363000FFF78AFF060004D015E00020388005203F
:10364000F8BD002D13D039880098814201D90C268D
:103650000DE020783B460007000F2A462146FFF781
:1036600073FF060005D00C2E01D0002038803046B4
:10367000F8BD7A4D6878401CC0B268700B2801D143
:1036800000206870A878401EA87061784807400F35
:10369000022810D00128EAD16C4861680AF05DF96F
:1036A0002879401CC0B228710128E0D16A484078CE
:1036B000FFF776FADBE7C806D9D46068FFF784FF26
:1036C000D5E770B50446674816460D46814204D1D9
:1036D00063205F49C00011F084FC012E05D06520F5
:1036E0005B49C00011F07DFC70BD5B480121C170D9
:1036F0006620207000202072A581A17370BD70B576
:1037000016460D46040001D1FFF71EFE662101702A
:103710000121017229680161A98881820673002C48
:1037200001D1FFF72DFE70BD4D49884201D2102016
:10373000704707210170002070474B4A10B5904236
:1037400008D30124A404464AA04201D3904201D3E5
:10375000914201D2102010BD0DF097FD10BD424BDB
:1037600010B5994208D30124A4043D4BA14201D3D2
:10377000994201D39A4201D2102010BD022803D0F1
:10378000102801D0092010BD0DF0A5FD0028FAD0A9
:10379000052010BD344B10B598420CD30124A4046D
:1037A0002F4BA04201D3984205D3994203D3002A5C
:1037B00003D09A4201D2102010BD0DF0B2FD0028B6
:1037C000FAD0072010BD10B50446254894B08442B5
:1037D00002D2102014B010BD01F0C9FD002801D0A4
:1037E0001120F7E70F2008A9087369460BA80AF013
:1037F000E1F80028EED16846007A207068464089DA
:10380000608068468089A0800020E3E710B5124CF4
:103810000846E17800290ED000280AD0104A9042CC
:1038200002D30368934201D2102010BD8288002A7F
:1038300003D0012903D0082010BD092010BD04F0D9
:1038400047FB0028FAD10021E17010BDB011002023
:103850001C34000031020000340000208C0C0020D9
:1038600000200020FFFF000000600100334A10B577
:10387000914206D301229204914204D3304A9142EC
:1038800001D21020E1E7421E1E2A02D800F019F8EA
:10389000DBE70246203A1F2A02D801F08BFCD4E76E
:1038A0000720D2E7264A10B5914201D21020CCE77A
:1038B0000246203A1F2A02D801F0D2FCC5E70720B1
:1038C000C3E710B51D4A94B0914206D30122920479
:1038D000914204D31A4A914201D210207AE700247F
:1038E000012803D0022817D0072073E70878C00703
:1038F000C00F03D001206946087101E068460471D9
:1039000039206946087009A968460AF053F800286A
:1039100012D00C498C200DE003C9029101903D208A
:103920006946087009A968460AF044F8002803D0DF
:1039300004499C2011F055FB20464BE70060010034
:10394000002000201C3400008107C90E002808DA7E
:103950000007000F083880082C4A80008018C069D2
:1039600004E080082A4A800080180068C8400006E9
:10397000800F704710B50D20FFF7E6FFC4B204209A
:10398000C043FFF7E1FFC0B2844203D021A11A2057
:1039900011F027FB10BD0121234A48031060234B7F
:1039A00000221A60224A5160224A1060224A1160A5
:1039B0001D4980390860704701211B4A4803106087
:1039C0001D4A5160194A002111601A490860704768
:1039D00010B516490868012804D00EA1562011F030
:1039E00000FB10BD154880680022C0B20A600DF0CF
:1039F000C7FE10BD10B50D4801680029FCD0FFF7C7
:103A0000E7FF01200B494003086010BD00ED00E016
:103A100000E400E07372635C736F635F68616C5F06
:103A2000726E672E6300000080E100E000D100406C
:103A300000D3004080E200E000D0004000D500400C
:103A400030B40121BC48C9020160CD1005604A03B1
:103A50000260BA4803681B021B0A03600468002363
:103A6000240A24020460B6480468240A240204607C
:103A7000B448012444608460B34C23606360A36055
:103A8000B24B19601D601A60B14B19601A600121B8
:103A9000016030BC704710B40121A748CC0204601B
:103AA0000A0202600B060360A64841608160A649D5
:103AB0000020086048608860A448046002600360D9
:103AC00010BC70470121A148C9020160C910016002
:103AD0007047002805D0012805D0022805D19D484F
:103AE00070479D4870479D48704710B59CA18B203A
:103AF00011F077FA002010BD70B500219F4CA04D49
:103B0000A04A914B002808D001281DD0022822D0BD
:103B100093A1B32011F065FA70BD01200004A060EC
:103B2000A86011601960984B42109A60974A9060A3
:103B3000814A0012106096480160874801609548EC
:103B400001609548017070BD01204004A060A8602C
:103B50005160596070BD01208004A060A860916030
:103B6000996070BDF8B59446844A854D00240127BC
:103B7000754E002808D0012836D0022844D078A1FC
:103B8000E82011F02EFAF8BD891E0902090A012069
:103B900000049060346068607A4A1160012B21D083
:103BA00000217D4A7D4B517061463D31DC63DF630E
:103BB0007B4B5C6002249C6004241C61744B196084
:103BC00074490F60614B89151960704B58606048EB
:103BD000016075487349C16086606B496003486045
:103BE0001770F8BD0121DCE701205C4E40046F4FE7
:103BF000012B04D13460506068603960F8BD90607A
:103C0000346068603960F8BD0120524E8004684F0E
:103C1000012BF4D1EEE767484068704770B54A4D14
:103C200028680026554C012806D1A068C00303D59A
:103C300001200004A0602E606868012809D1A068F6
:103C4000800306D501204004A0606E6001200FF0C3
:103C500058F9A868012809D1A068400306D50120B9
:103C60008004A060AE6002200FF04BF970BD10B56B
:103C700049490878002818D00120434AC0039060C1
:103C8000424A400090602C4A00121060404A0020D6
:103C90001060314A10603F4A106008704A78002A6C
:103CA00002D048700FF02DF910BD0320FAE7012073
:103CB0004149000608607047012024490006086059
:103CC000704701203C4940050860704701201F49AA
:103CD00040050860704731490020C86388151B49BA
:103CE00008607047410A354AC005C00D5043801C2A
:103CF0005143400A0818704710B4314C430B6343DA
:103D00001B0C5C020C602D4C6343C31A2D485C02F3
:103D100058432A4B400D4343E31A0124DB03240498
:103D20001B191B1613700A681018086010BC704726
:103D300010B50FF0BEF910BD80E100E008E400E02E
:103D400018E400E000B0004040B1004080E200E034
:103D500000E100E048B100404081004044B1004033
:103D60007372635C72656D5F68616C5F6576656ECA
:103D7000745F74696D65722E6300000000B30040CB
:103D800040B3004040B5004000F5014000830040D2
:103D9000408500400082004050000020C08F00405D
:103DA000008500400080004080F5014044B500409F
:103DB00048B5004000B5004000E200E0093D0000C9
:103DC000378600006F0C010010B50FF05EF910BDD2
:103DD00000200449C863012001218140024A11608A
:103DE00000BF7047C01F004080E200E00E4A12682A
:103DF0000C498A420AD118470B4A1268094B9A4269
:103E000004D101B50DF0D7FD03BC8E460749096802
:103E10000958084706480749054A064B70470000FD
:103E200000000000BEBAFECA1C01002004000020F1
:103E3000981D0020981D002010B5F84C94B0216802
:103E4000087A002835D017206A46107006220931FA
:103E500001A810F029FF09A9684609F0ABFD112857
:103E600025D02168C0318979062920D007291ED0A4
:103E700008291CD004291AD0092918D00A2916D0DB
:103E80000B2914D0052912D0002803D0E4A1F42076
:103E900011F0A7F82168B820405806221C300931DB
:103EA00010F002FF2068017A8030806BC17614B078
:103EB00010BD3220C8E770B5D84D0446296803000C
:103EC000C03111F07FF90C077C0B1A212E3B4851B1
:103ED0005C677080FF20D2A10A306EE088790128EB
:103EE0006DD009286BD0052869D00A2867D00B2827
:103EF00065D0FF20CAA10F305FE0887901285ED02D
:103F0000FF20C7A1163058E08879062857D0072827
:103F100055D0082853D0052851D0FF20C0A1193012
:103F20004BE0887909284AD00A2848D00B2846D087
:103F3000042844D0FF20BAA11F303EE0887903282E
:103F40003DD007283BD0082839D0092837D0FF209A
:103F5000B3A1253031E08879062830D00A282ED048
:103F6000FF20AFA12B3028E08879062827D007282A
:103F700025D00B2823D0FF20A9A12F301DE0887960
:103F800006281CD00A281AD00B2818D0FF20A4A17C
:103F9000343012E08879092811D00A280FD0FF2088
:103FA0009FA1393009E08879092808D00A2806D06D
:103FB000082804D0FF209AA13D3011F012F828689B
:103FC000C030847170BDFF2095A14230F5E7934960
:103FD000C9220968525CD206920F05D1A0318A8BA2
:103FE000824201D1887F70470020704770B5044637
:103FF000112020700021894D61702968C031897AB3
:10400000002908D003290ED0042910D0FF2084A154
:104010006B3010F0E6FF20780009012802D92868EB
:10402000807D607070BD0007000F203002E0000747
:10403000000F30302070EEE730B503887C497D4CAE
:104040008B4202D09A1FA2421ED242888A4202D0DC
:10405000951FA54218D2934216D883887D24E40088
:10406000A34211D8C088884205D0724D04460A3C4C
:104070002D1FAC4208D2884208D08A4206D05B1C71
:104080005A43C000824201DD072030BD002030BD10
:10409000FFB50022099B002802D0994205DC5CE0B4
:1040A000002902D1002004B0F0BD0920FBE7845CA8
:1040B000002C12D085186F780D2F4CD010DC3B00EF
:1040C00011F080F80A421B2A2A303032323A3A4242
:1040D000835C002B3FD1521CD2B28A42F8DBE1E76D
:1040E000122F31D004DC0E2F35D00F2F2CD132E01F
:1040F000142F11D0152F27D116E0022CD5D1AB7873
:10410000039C072B237001D25B0701D40A20CAE766
:10411000029B01241B7814E0E343DB0708E0012C39
:1041200008D011E00620BEE70F2523072D075B19F5
:10413000002BF4D03046B6E7029B1B789C070AD4CC
:1041400002242343029C2370835C521C9A18D2B22F
:104150008A4204DDA9E70B20A5E7192676028A42E8
:10416000A5DB9FE705E00278401C002A01D0002073
:1041700070470A46491E89B2002AF4D101207047CF
:1041800070B5264D00212868C943A03081830024E2
:104190008477214606200DF0CDFD002105200DF08D
:1041A000C9FD002102200DF0C5FD0120FFF783FEAF
:1041B0002868C030C471047201F063FF70BD30B56F
:1041C000164C95B02268C0329279042A0CD0052A88
:1041D0000AD028236A4613709080132906D03B2901
:1041E00004D0072015B030BD0820FBE791711046C0
:1041F00009A909F0DFFB05000BD12068C0308179E7
:10420000062908D0082906D0072904D00520FFF781
:1042100052FE2846E6E70420F9E70000540000209B
:104220007372635C6761705F636F72652E63000019
:10423000FFFF00007B0C000030B587B0040003D006
:10424000002107200DF076FDF74D012128686A4610
:1042500001720421117003210C300DF06BFA2968F2
:104260004022887B8006800E1043887368460BF0DE
:10427000AEFB00280DD12968098A00290AD0002C3C
:1042800008D08B000122002107200DF0AEFC07288A
:1042900002D0032007B030BD0020FBE770B5002539
:1042A0000646002803D0002107200DF043FDDE4C18
:1042B000012120680172062109300DF03BFA2068C7
:1042C000817B8906890E8173FFF7B6FD2068008A1D
:1042D00000280AD0002E08D08300012200210720E8
:1042E0000DF083FC072802D00325284670BD002569
:1042F000FBE7F0B59BB0040003D1CC49CC4810F0EB
:1043000070FE72202070616800260A780825521F0E
:104310000127C548130010F055FF0F097CDFFD7C15
:104320007EFCFBBB7C7C7C7CFAF97C00BE48006890
:10433000C0308079032804D0BD48BC49093010F052
:1043400050FE002108460DF0F5FC002107200DF07D
:10435000F1FC6078B44A284360701068102501466B
:10436000C0314B7A2B434B7263689D783C2D4DD006
:1043700002469D88A032977763688030DB890B8086
:1043800063681B8A4B8063685B8A8B809583616856
:10439000826BC97911756168806B0831153006220E
:1043A00010F082FC0620FFF786FD9F48FB23006883
:1043B0000146C0318E72027E1A400276B82212582F
:1043C000937A9B089B0093724682487A4006400E7F
:1043D0004872284602F0C0FE002804D09448934951
:1043E000243010F0FEFD284602F0D0F8002804D05A
:1043F0008F488E49273010F0F4FD284603F016FD53
:10440000002806D08A48894929303EE10120FFF77B
:1044100052FD1BB0F0BD074600688E88C030807921
:10442000062812D0072810D008280ED004280CD057
:1044300009280AD00A2808D00B2806D0052804D05D
:104440007B487A49353010F0CCFD607828436070A5
:104450003868C030417A294341728079092811D0E7
:104460000A280FD00B280DD005280BD0FFF788FEA7
:10447000304602F07AFE304602F08EF8304603F005
:104480000BFDC6E7FFF77CFE0220FFF714FDEFE708
:104490000068C0308079062812D0072810D008287C
:1044A0000ED004280CD009280AD00A2808D00B28DE
:1044B00006D0052804D05E485C49593010F091FDC3
:1044C0006068807902F004FF0028A2D06178294357
:1044D00061706168C8809CE707460068C0308079D9
:1044E000062812D0072810D008280ED004280CD097
:1044F00009280AD00A2808D00B2806D0052804D09D
:104500004B484A496C3010F06CFD04E037E1A1E102
:1045100090E090E015E06078284360706068C188A2
:104520003868C030018061680989418061684989C3
:104530008180002102200DF0FDFB3868C030C6717B
:1045400067E706460068C0308079062819D007283A
:1045500017D0082815D0042893D0092811D00A288C
:104560000FD00B280DD005288BD031482F49833030
:1045700010F037FD3068C03080790428ABD00528B2
:10458000A9D03068807C40063AD5606802210C30A2
:10459000FFF7E8FD002833D060680821001DFFF711
:1045A000E1FD00282CD03168B8204058807A80077F
:1045B00008D1CA20405C002808D1488AC20505D528
:1045C000C00703D1488A4022904348824A8A80200B
:1045D00082434A822D2268460270BC20425A6846B5
:1045E000828010229731801D10F05EFB09A9684679
:1045F00009F0E0F90028A3D03D200C49000144E077
:1046000062683068AC2192890A5261680822091DEB
:10461000AE3010F049FB10A805743068AE3015902C
:1046200014A80BF0D4F9F4E6540000202042000056
:10463000260300008F7106460068C0308179062984
:1046400019D0072917D0082915D00429EBD009293A
:1046500011D00A290FD00B290DD00529E3D0FD2058
:10466000FA49800010F0BDFC3068C0308079042821
:10467000D9D00528D7D060688179002902D0807808
:10468000002805D02320F149400110F0AAFCC0E623
:104690006078B8212843607030680958897A8907A2
:1046A000890F012951D1817C09064ED4017E490729
:1046B00001D5042100E00321C03081722B2069461E
:1046C000087009A9684609F075F9002803D0DF4988
:1046D000DF4810F086FC68463168008D88820E2223
:1046E00010A80274DB48B822159052580832426173
:1046F0000A4660324260927902700A4614320261C0
:10470000521D82601032C260133A82619632C261D9
:10471000921C0262473A4262103282621032C262D6
:10472000473AC263521E0264921F50314264816450
:1047300014A80CF033FB022815D0002813D0C4486D
:10474000C249293010F04DFC0DE0817C4906017E04
:10475000490701D5042100E00321C0308172002106
:1047600006200DF0E7FA3068418A0A0602D440229A
:104770009143418289B280229143418249E6B64801
:104780000068C0308079032804D0B148AF49573061
:1047900010F027FC002108460DF0CCFA002107207C
:1047A0000DF0C8FA6078AC4A284360701068102594
:1047B0000146C0314B7A2B434B7263689D783C2D88
:1047C00000D123E602469D88A03297776368803047
:1047D000DB890B8063681B8A4B8063685B8A8B80F4
:1047E00095836168826BC97911756168806B083146
:1047F0001530062210F058FA0620FFF75CFB9648A9
:10480000FB2301680A46C0329672087E184008767B
:104810004E82507A4006400E5072284602F09CFCB0
:10482000002804D08A488949723010F0DAFB284603
:1048300001F0ACFE002804D085488449753010F0A2
:10484000D0FB284603F0F2FA002897D080487F4931
:1048500077301AE7607828436070DAE500290BD0DA
:1048600088807D480068C0300288CA8002880A813A
:1048700042884A81808888817047F7B5064600786B
:104880000C460027010982B03D46012974D07248C8
:1048900000680090C03002296FD0072904D00A298F
:1048A0006CD06A496D480DE271680A78521F130096
:1048B00010F088FC0F09A451A4A42F585847A4A4B1
:1048C000A4A4656FA4008A783C2A1BD01027162563
:1048D000002C7DD08888A0807068A21DC0892082AD
:1048E0007068C089E0817068008A60827068408A60
:1048F000A082716808460831C07901F0B1FB002040
:10490000607375E019270725002CE2D00021A17102
:1049100071E011270725002CDBD089880091A18048
:104920007168F7228979A171417A1140417200982A
:1049300002F01CFC009801F033FE009803F0BAFA74
:10494000D2E101270925002CC3D08888A080706897
:1049500080792072C8E1888812270E252146FFF74A
:104960007DFFC1E118270825002CB2D08888A080DF
:10497000A01DFFF73BFBB7E144E0A6E15CE01A278E
:104980000725002CA5D04888A08070680079A07108
:10499000AAE18A783C2AB5D010271625002C98D099
:1049A0008888A0807068C08920827068C089E08192
:1049B0007068008A60827068408AA0827168607B3B
:1049C000497D40084000C907C90F0843607300E0F3
:1049D00093E17168C007497DC00F49084900084349
:1049E00060737168A21D08460831C07901F038FB78
:1049F00019480068C030417AEF2273E1A7201349BB
:104A0000C0005FE1307A012803D014480F49C8384C
:104A100058E112270E2570892146FFF71FFF002C51
:104A200092D070784007400F032889D10A48006867
:104A3000C030417AFB2255E107490968A031002CBA
:104A400001D08A8BA280327A921E09E020420000B7
:104A500015040000AC1200205400002017060000CE
:104A6000130010F0AFFB073D4853FDEB6F05FD0051
:104A700013270C25002C85D0009900224A82F1686A
:104A800089788907890F0129217A26D049084900A8
:104A90002172FD231940F3689B785B07DB0F5B00F5
:104AA00019432172E323E2801940F3681B785B0706
:104AB000DB0E19432172DF231940F3685B78DB07B3
:104AC0009B0E194321726272F1680122C978A172AA
:104AD000017A1143F7221140ADE001231943D7E7D2
:104AE00015270C25002C9BD0F06806220068A11D1C
:104AF0000EF07CFFF8E016270725002C90D0317BC4
:104B0000A171017A08221BE00172EDE01427122541
:104B1000002C85D00098A21D8030806B0146153195
:104B2000007D01F09DFAB089E081207C01210843DD
:104B3000F92108402074FD480068C030017A022243
:104B40001143E1E717273825002C94D03221A01D0E
:104B500010F007F90020A071207A03210843207289
:104B6000FB210840F14909680A7E5207D20F9200E2
:104B700010432072B8204058807A800757D0A07A1E
:104B80008A7C4008D2074000D20F1043FD2210401B
:104B9000A0728B7CFB229B07DB0F10409B0018430D
:104BA000A0728B7CF7269B07DB0F3040DB0018439D
:104BB000EF231840A072E07A10408A7CD206D20F10
:104BC00092001043E0728A7C3040D206D20FD200AD
:104BD0001043E072888AA0812046102267310E308F
:104BE00010F062F8D149A07F0968C0078A7DC00F24
:104BF00052001043A0770A7E400852074000D20FAF
:104C00001043A077084640304DC820344DC4303C96
:104C10003F20405C22463032393101F021FAC3484E
:104C200000688030806B817A890889008172BF4872
:104C30000068C030017AFB22114065E7327B022A0E
:104C400018D017273825002C11D0017AFB231940E2
:104C50000172012A17D0032A22D0042A23D000E0AF
:104C60002DE0052A1FD0B249B24810F0BAF901F080
:104C700008FA39E019270725002CF8D0898BA18084
:104C80000121A17103E00121A1710021E171417AAB
:104C9000CA094906D201890E49000A434272E6E771
:104CA0000220A07106E0707B0007000F8030A07129
:104CB000052A02D00020E071D9E70120FBE79D48DA
:104CC0009B490C3010F08DF90EE0317A00290BD1A0
:104CD00019270725002C10D0491EA1800021A171A1
:104CE000417AFD22114041720498002C058001D0C8
:104CF00027806580002005B0F0BD04980580F9E7A5
:104D000010B58A4C94B02068C0308079022809D050
:104D1000032807D0052805D0092803D00A2801D088
:104D20000B2837D11B2108A80173002101746946A3
:104D30000BA808F03FFE002804D1684640781B28E5
:104D400002D0032014B010BD002108460CF0F2FF81
:104D5000002107200CF0EEFF68468078002819D16A
:104D60002068C0308079801E030010F02BFA0A06FC
:104D70000613081313130D0F1113012000E0042074
:104D8000FFF799F80020DDE70620F9E70720F7E7AD
:104D90000820F5E70820D5E770B50025634C00280A
:104DA00007D0022817D0072828D0624860497930F8
:104DB00046E0FFF7A5FF00280CD1FEF7C5FA222137
:104DC00001700572FEF7DCFA2068C030417A0222D9
:104DD0001143417270BDFEF7B7FA12210170012133
:104DE00001722168BC22525A4281C031CD71FEF756
:104DF000C7FA2068C030417A0422E9E72168C6205A
:104E0000405C022809D0032807D0092805D00A28C9
:104E100003D00B2801D00528DCD1887B810901292A
:104E200011D0800904D043484149703010F0D9F8BE
:104E30000020FFF733FA0028CCD03E483C497430BC
:104E400010F0CFF870BD0020FFF7F6F9F3E770B56A
:104E50000D46040004D137483549813010F0C1F8BF
:104E60002078012805D0334831499F3010F0B9F837
:104E700070BDA18830482D4E814209D1E28882421E
:104E800006D130681321A030808BFFF798F970BDF0
:104E9000814202D1E08800280AD012202870687868
:104EA00008210843687007CC083507C5002106E0D3
:104EB00000227823114602200CF097FE0221306870
:104EC000C030C17170BD00B5184A87B01268C032D9
:104ED000527AD20907D106236A46137001901172E3
:104EE00068460AF074FD07B000BD00B587B0072022
:104EF0006946087068460AF06AFDF4E70B480068E6
:104F0000C030807A704738B5084C05460278206872
:104F100013000146C03110F055F909A9061111A37B
:104F2000204E738BA900FEF787FF38BD5400002088
:104F300020420000F2050000FFFF000088790628EB
:104F400005D0092803D0FE49FE4810F04AF8206831
:104F50000422017E1143017682E0A9880029E4D071
:104F6000A030808BF8498842DFD0A868002804D19F
:104F7000F448F349103010F034F82068C030407A1B
:104F8000C00904D0EF48EE49113010F02AF8A868A3
:104F900006220A38A86000902068AB88A030808B79
:104FA000042102F00DF80028BFD0DB20E449C00046
:104FB00010F017F8B9E788790528B6D928790128BB
:104FC00002D0022808D103E0487A802210434872B8
:104FD000487A012210434872284601F05CF82068A4
:104FE000C03080790628A0D9082801D8062004E01E
:104FF00009289AD90B2898D80920FEF75CFF94E776
:10500000887906280AD0042808D0092806D005285F
:1050100004D0CC48CA493D300FF0E3FF0ECDCB4859
:105020000361C2608160A2210170FEF7BEF97CE7D6
:105030008879062818D0072816D009280DD00A2804
:105040000BD0C048BE4950300FF0CBFF2068C030B5
:105050008079062808D0072806D00B20FEF72BFF02
:10506000284601F018F860E70820F7E7B548B4498A
:1050700064309DE7FFB593B0012468460321847036
:10508000C9021D4601800AF07AF900226946012012
:1050900003F085F906460AF076F9002E5CD16846E1
:1050A000152184704902018000271C2101A808975E
:1050B0000FF059FE01200146103108A801700020B0
:1050C000014608A841708178F9200140891C2143DC
:1050D00008A881706846017902263143017114994C
:1050E0008185C7851F21018608A80A9013980D9015
:1050F000684609900AF043F90EAA09A901A802F02E
:105100001CFF07460AF03FF9002F02D0384617B0BF
:10511000F0BD8F4F68463968008F488068468470BC
:105120008C49018008A88078F9210840801C41083A
:10513000490008A8817068468685068615A80D90E6
:105140000AF01DF90EAA09A901A802F0F6FE06460A
:105150000AF019F9002E01D03046D8E768463968C0
:10516000008F88807B4968468470C91C018029882B
:1051700010A8018069884180A9888180E988C18060
:10518000082168468185018610A80D900AF0F7F87D
:105190000EAA09A901A802F0D0FE04460AF0F3F80D
:1051A000002C01D02046B2E768463968008FC880DD
:1051B0000020ACE7F0B5684E95B00C46B14235D34F
:1051C0000127BF04654DBC4201D3AC422ED3202839
:1051D00004D0212824D0222837D13DE03C21684644
:1051E0000170218881806188C18009A908F0E2FBF3
:1051F000002806D108A98979002904D002290DD0F8
:10520000032015B0F0BD6168B142FAD3B94201D3B1
:10521000A942F6D36A46128D0A80F2E75048F0E7B9
:1052200008684B4C002812D0A84201D21020E8E7B1
:1052300006210EF0C5FB411C07D02168A822505062
:105240000120A03188750020DBE70720D9E720681E
:105250000021A0308175F6E7084600F028FFD0E76E
:105260003D4A10B5914206D301229204914204D3E3
:105270003A4A914201D2102010BD202805D02128A1
:1052800003D0222803D0072010BD062010BD0846F9
:1052900000F042FF10BD70B504462C48CC21AC3064
:1052A0000FF061FD29482A4EAC3000213060C9431F
:1052B000A0308183002585770120FEF7FCFD306852
:1052C000C7210D54E121C57389000182B6210D5417
:1052D000014609310830FDF753FF316808460A7A64
:1052E00060308271062209310FF0DEFC3168084619
:1052F00029311930FDF77BFF002C37D03068803022
:105300008463FEF799FD1E20E081607A8F210840BA
:105310003030607230680146143121619831616229
:10532000933921601031616025721339A162091F20
:10533000E1628531E163303921631031616311E04D
:1053400020420000C2060000FFFF00004C120020B7
:1053500054000020012A000000600100002000200D
:105360000230000010310930A163A06470BDF7481D
:105370000068C0308079042803D0052801D00020BF
:1053800070470120704770B50646F1480C468142CF
:1053900006D301208004844204D3EE48844201D223
:1053A000102070BDFFF7E3FF002801D0112070BD71
:1053B000E948E64D002E02D0012E46D12FE022789A
:1053C000002A0AD00121012A09D0022A14D0032A76
:1053D000EDD1A2799209EAD112E0002103E0A2798D
:1053E0009209032AE3D12868062201726030817194
:1053F000611C0FF059FC05E0A2799209012AD6D16F
:1054000028680172002107200CF094FC286806220D
:10541000611C09300FF048FCFEF70EFD11E0217809
:10542000002912D0012910D0022910D00329BED1A1
:105430000120FEF733FF002803D0C849C8480FF009
:10544000D0FD2868C673002070BD072070BD012004
:10545000FEF7F2FEEFE7BF4910B5884201D21020F7
:1054600010BDBA49024609680B7A0931184600F0A6
:10547000F7FD002010BDFFB599B005460020694634
:105480000871087208A90874144608750122B04909
:105490009204B0481E46002D05D08D420BD3954294
:1054A00001D3854207D3002C08D08C4203D3944209
:1054B00004D3844202D210201DB0F0BD2846204300
:1054C00018D01F270CAB01AA009728461A99FEF79F
:1054D000DFFD0028F0D10DAB02AA3146204600972F
:1054E000FEF7D6FD0028E7D16846007AC10703D051
:1054F0000A20E1E70720DFE7800705D56846007945
:10550000800701D50B20D7E7FFF731FF002801D036
:105510001120D1E703AF002D0FD01A206946087380
:105520001A9808742946781D1A9A0FF0BDFB0EA927
:1055300003A808F03FFA0028BED1002C0ED020218D
:1055400068460173067432462146781D0FF0ACFBA5
:105550000EA903A808F02EFA0028ADD17B4908A8AF
:105560000968007C08700020A6E7F0B5044678487A
:10557000002695B0844276D301208004844202D371
:1055800074488442F7D32378012B09D170496068AD
:105590008842F0D39904884202D36E498842EAD304
:1055A0006A490A681546C035A879022814D003282C
:1055B00012D0052810D009280ED00A280CD00B28AC
:1055C0000AD0012803D0002B06D0012B04D0687A22
:1055D000C506AD0F06D101E0082012E6850701D40B
:1055E000400701D511200CE6208A5E4F0546203D7C
:1055F000BD4207D3012B6ED10028FCD1658A002D56
:10560000F9D111E0022B01D0032B01D1A02862D3E4
:10561000012B01D1002807D01578ED0704D0658A49
:10562000002D58D0B42D56D8002B06D0012B08D011
:10563000022B04D0032BDED118E0002519E002254F
:1056400017E0002802D1608A00280DD00425606888
:10565000007800280DD001280AD0022808D003289D
:1056600006D03D48CDE563E00125F0E7032500E0E5
:105670000126D07B01281CD1108A002819D0907BEC
:105680008109012911D0800904D035483349EC3013
:105690000FF0A7FC0120FEF701FE00280BD03048D8
:1056A0002E49F0300FF09DFC05E00120FEF7C4FD0F
:1056B000F3E7FEF7C1FB207A002806D0012806D0C8
:1056C000022806D0032806D106E0002705E00127BE
:1056D00003E0022701E087E00327002D01D0022D1F
:1056E00048D1002F46D0E06800287DD001790029FC
:1056F00020D0082978D8027B082A75D800290AD03A
:10570000134B0168994213D301239B04994202D39E
:10571000104B99420CD3002A10D080680C49884263
:1057200006D301218904884208D30A49884205D258
:10573000102066E5027B002A6AD0DCE70348006897
:105740000078800710D00448401E5AE5540000201D
:105750000060010000200020023200002042000012
:1057600086080000E13F0000022D03D1022F4FD038
:10577000032F4DD0182168460170218A8180218A2B
:10578000C1800572FE480068007A002801D0012817
:105790007ED1694648726846867221780B300129AD
:1057A00023D006210FF0DDFA072168464174877483
:1057B00009A908F0FFF80028BBD10A206946087043
:1057C00009A9684608F0F6F80028B2D13A206946DF
:1057D000087009A9684608F0EDF80028A9D1002D45
:1057E00009D0022D07D04CE012E061680622491C66
:1057F0000FF05AFAD8E7002F43D00026374623E0AF
:105800000168B00009580978002903D0012904D0A3
:105810000720F6E469460F7102E001216A46117122
:10582000E16806220968095801A8491C01300FF0F7
:105830003BFA0B206946087009A9684608F0BAF8D7
:105840000028E6D1761CF6B2E0680179B142D7D8DB
:1058500000266F4611E08068B10041581022381DC3
:105860000FF022FA3B206946087009A9684608F043
:10587000A1F80028CDD1761CF6B2E068017BB142D8
:10588000E9D81B20694608700120087109A900E0C9
:1058900036E0684608F08EF80028BAD108A84079AA
:1058A0001B282DD12B000FF08DFC050404060604E7
:1058B0001E00032015E0B2480068C0308079030064
:1058C0000FF080FC091E061E1E0A1E080C0E1E008C
:1058D000022006E0092004E0052002E00A2000E0A2
:1058E0000B20FEF7E8FA012D0CD0608A002809D0C1
:1058F00000228300114610460CF077F9002801D0F1
:1059000003207EE400207CE470B586B00C000646DF
:1059100009D09C48844248D301208004844202D3A9
:105920009948844241D3964D2868C030C1790229F4
:1059300002D0407A400702D5112006B070BD002C7D
:1059400004D02046FEF778FB0028F6D13046FEF75B
:105950003EFB012803D0022823D08C48EDE721002C
:105960001BD1082069468882286801ABC08805AA37
:10597000002103F0F7F80028DFD16846808A082864
:1059800001D00320D9E7684681888181C188C1811F
:10599000018901824189418203A9304601F068FCF6
:1059A000CBE7002C01D00620C7E71020C5E770B573
:1059B0000C460546FEF70BFB012803D0022801D058
:1059C000724870BD21462846FEF7F9FB70BD00B550
:1059D0000146143095B0192801D2880707D008462F
:1059E0001E3004D00A3002D0072015B000BDFFF7EA
:1059F000BEFC002801D01120F7E761483122006881
:105A0000417068460270017109A907F0D3FFECE705
:105A100001B582B0022069460880594802AB00688F
:105A20006A468088002102F00DFF69460988022934
:105A300000D003200EBD38B502216A4611805249BC
:105A4000884201D2102038BD4D49034609688C8830
:105A50000021204603F086F8694609880229F2D021
:105A6000032038BD3EB504460820694608804548F5
:105A7000844206D301208004844204D342488442F5
:105A800001D210203EBD2046FEF7D6FA0028F9D1FB
:105A90002088694688806088C880A0880881E0885E
:105AA0004881374801AB00686A46C088002102F08F
:105AB000C9FE694609880829E4D003203EBD1FB508
:105AC00004460820694688812E48844206D3012076
:105AD0008004844205D32C48844202D2102004B0B2
:105AE00010BD27480B46006803AAC088002103F0B8
:105AF00039F80028F3D169468989082901D00320A3
:105B0000EDE76946098821806946498861806946D0
:105B10008988A1806946C988E180E0E7FEB50E4624
:105B20001849174605468E4206D3012292041648AC
:105B3000964203D3864201D21020FEBD1F2F01D909
:105B40000C20FEBD0E4C8D4232D3954201D38542CE
:105B50002ED3206801A9408802F026FE0028F0D14B
:105B6000287869464871206801A9408802F0FFFD45
:105B70000028E6D16946009008780221084307E032
:105B800054000020006001000020002002300000CE
:105B9000694608704979090703D008210843694616
:105BA000087020686946408802F08BFD0028C8D143
:105BB00069460F8120683346408802AA002102F01E
:105BC00041FE69460989B942BBD00320FEBD38B504
:105BD0000C46F749002801D0884201D38C4201D2FB
:105BE000102038BD21886A461180002801D0002984
:105BF0000BD0F049034609684D880021284602F081
:105C0000B1FF69460988218038BD0C2038BD30B508
:105C10000C46E94987B08C4206D3012189048C42A5
:105C200005D3E3498C4202D2102007B030BDE14DCC
:105C30002968C0310A7A520708D48A79521F1300A2
:105C40000FF0C0FA05040604040604000820ECE77F
:105C5000497AC90901D00D20E7E7FEF7B8F9012814
:105C600003D002282DD0D548DFE720881E2801D296
:105C70000720DAE72868C030807906281FD00A207C
:105C8000FEF719F905216846017000798108A078AE
:105C90008900C007C00F014368460171FB20014025
:105CA000A0788007C00F80000143684601712188F9
:105CB000C18009F08CFE0028B7D00320B5E707208B
:105CC000DEE70620B1E7F0B587B014460D46FEF7D3
:105CD0007EF9012804D0022802D0B84807B0F0BDF0
:105CE000B44B18680146C0310A7AD20707D08A79C6
:105CF000062A04D9092A02D0002D02D050E008203B
:105D0000ECE7AD4A944206D301229204944204D3B4
:105D1000A74A944201D21020E0E7A278D206520F9F
:105D2000042A0CD8E378072B09D3102B07D8227943
:105D30009A4204D3102A02D822881E2A01D00720B2
:105D4000CCE702468032966BF727F372966B237985
:105D50003373966B737A3B40A778BF06FF0FFF0043
:105D60003B437372966B2388F381966BA778B37A63
:105D7000FF079B089B00FF0F3B43B372FB273B4091
:105D8000A778966BBF07FF0FBF003B43B372926BC0
:105D9000A478537AE406DB08DB00640F23435372D4
:105DA0000B226B461A70852D22D008DC002D17D0EF
:105DB000812D17D0822D17D0832D08D116E0862D86
:105DC00018D0882D18D0892D18D08A2D18D00B22E4
:105DD0001A71B622125C774C002A13D0A83012E058
:105DE0000022F5E70122F3E70222F1E70322EFE7C1
:105DF0000522EDE70622EBE70822E9E70922E7E7BB
:105E00000A22E5E7002002908879072806D00828B2
:105E100004D00A2804D00B2802D004E0062000E0B9
:105E20000920FEF748F8684609F0D1FD002801D0A6
:105E3000032053E720680422C030017A4908490052
:105E400011430172002049E770B55A4E0D46316882
:105E500086B0C031097A1446090701D408206CE5E0
:105E6000FEF7B5F8012803D0022801D0534864E5B5
:105E7000002D10D05048844206D301208004844273
:105E800004D34B48844201D2102056E5012D0BD09B
:105E9000022D02D106E0002C01D007204DE50020A4
:105EA000029005E0022000E001206946087102949A
:105EB000032069460870684609F089FD002801D072
:105EC00003203AE53068F722C030017A11400172B0
:105ED000002032E570B594B014460E46FEF777F810
:105EE000012804D0022802D0344814B070BD314DCE
:105EF0002868C030007A800701D40820F5E7002C1C
:105F000001D00720F1E7FFF732FA002801D0112075
:105F1000EBE7002E1DD02D21684601702C68BC20B7
:105F2000015B684681801022B11C801D0EF0BCFE12
:105F3000207EFB210840B17CC907490F0843207629
:105F4000B07CFF214008A075608A823108436082DE
:105F500007E02E21684601702868A030818B6846D2
:105F6000818009A9684607F025FD2968FD23C03115
:105F70000A7A1A400A72B8E710B50C46FEF727F8FD
:105F8000012803D0022801D00C4810BD0A488442E1
:105F900006D301208004844204D30548844201D200
:105FA000102010BD2046FEF721F8002010BD000093
:105FB000002000205400002000600100023000009A
:105FC00010B594B00446FEF702F8012804D0022868
:105FD00002D0644814B0E9E763480068C0308179B2
:105FE000042910D005290ED03820694608708C800D
:105FF00001208871C87109A9684607F0DBFC0028F8
:10600000E8D00B20E6E70020E4E710B594B00446A2
:10601000FDF7DDFF012803D0022801D05148D9E760
:1060200051480068C030817904290DD005290BD072
:106030003820694608708C8000208871C87109A9D1
:10604000684607F0B7FCC5E70020C3E7464800688C
:10605000C0308079062801D30120704700207047A6
:1060600008B51346002806D040A000680090487983
:106070006A468009105C18700622581C0EF014FE47
:1060800008BD00B587B0012069460870684609F070
:106090009EFC07B000BD10B50446FDF755F9A221DE
:1060A00001700ECC08300EC0FDF76AF97EE770B5BE
:1060B0002D4C054601682068002911D02C4A9142D8
:1060C00006D301229204914204D32A4A914201D27A
:1060D000102070BD102277300EF0E6FD20680121FF
:1060E0008030806B01722068A9880182C17B012900
:1060F0000CD1807B800901280AD00120FEF7CEF860
:10610000002803D01C491D480EF06BFF002070BD15
:106110000120FEF791F8F3E770B505460068124CD0
:1061200000281AD01349884201D2102070BD20687F
:10613000B8210958097A012909D001467731293057
:106140000AF07BFF206801218030806B017221689A
:106150001022286877310EF0A7FD2068008AA880F9
:10616000002070BD02300000540000200302FF0137
:106170000060010000200020204200000303000016
:10618000FFB581B001980E46C078174610360E371D
:10619000022809D0032840D005287DD0F2A1F74875
:1061A0000EF01FFF05B0F0BDCC890A2060430E3011
:1061B000188031230A98002A0380F3D048680088A9
:1061C00090800020D0801081097B9481891FCDB2FE
:1061D0001AE030887168388048780A7800021043E5
:1061E000F880C8788A78000210433881BA1C091DEB
:1061F00028460BF070F8002D01D0002802D00020B6
:106200003871788008360A372046641EA4B2002808
:10621000DFD101990020C870C4E7CC890A2060430F
:106220000E30188032230A98002A0380BAD04868BA
:10623000002500889080D5801581087B401FC0B262
:106240000090948142E0716832880878FA803A7947
:10625000C30752085200DB0F1A43FD231A4083077D
:10626000DB0F5B001A43FB231A404307DB0F9B0045
:106270001A43F7231A400307DB0FDB001A43EF230F
:106280001A40C306DB0F1B011A43DF231A408306A3
:10629000DB0F5B011A4300E020E0BF231A404306F6
:1062A000DB0F9B011A433A71C00978718A784B78E9
:1062B0001002184338813A46C91C00980BF00BF8BD
:1062C000002801D0BD703D8008360A372046641E84
:1062D000A4B20028B7D10198C57063E7087BCC89C8
:1062E000801E85B228460830604310301880342361
:1062F0000A98002A03808FD048681746008890804B
:106300000020D080108194811037E000D581C01921
:106310000CE030883880009878602A4671680098D0
:106320000EF0C2FC0098083608374019009020464D
:10633000641EA4B20028ECD16BE7FFB50546C07817
:1063400081B00C460A9E03000EF03CFF0BA307171A
:1063500033414F6D8F9D9D9DA300207B17460828DC
:1063600006D0032804D085487FA154300EF039FEB2
:1063700004990E20088030200CE0207B174604286A
:1063800004D07E4878A171300EF02BFE04990E20C7
:10639000088031203080002F44D060680088B880A9
:1063A000607AFF300130F880E08938810020B881C0
:1063B00037E0207B1746042804D070486AA18D304E
:1063C0000EF00FFE04990E2008803220E2E7207BB9
:1063D0001746022804D0694863A1A9300EF001FED7
:1063E00004990E2008803320D4E7207B1746042828
:1063F00004D062485CA1C4300EF0F3FD0498102173
:10640000018034203080002F0CD060680088B88074
:10641000607AFF300130F880E08938810020B8814F
:10642000F881E870BEE6207B1746052806D00628CE
:1064300004D052484CA1E1300EF0D3FD0498122153
:10644000018035203080002FECD060680088B88053
:10645000607AFF300130F880E0893881E089B881C6
:1064600000203882A988F981DBE7207B17460728BE
:1064700004D042483CA1F8300EF0B3FD04990E2040
:106480000880362086E700962846049B00F02DFD04
:1064900088E635A13A480EF0A4FD83E670B50546BE
:1064A00000780C46082603000EF08CFE124C3434A3
:1064B000241C380A0A0A0A0A0A0A0A0A0A0A0A4CA0
:1064C0006878002804D02E4827A12C300EF089FDD2
:1064D000002C03D11F2024A1400108E06078304344
:1064E000607020E0002CF9D17D201FA1C0000EF0CB
:1064F00078FDF3E7002904D03F201BA100010EF036
:1065000070FDFCF721FF0446407830436070FCF7D3
:1065100037FF08E01A4814A1473002E0184812A1DA
:106520004C300EF05EFD002C0AD06078000707D5D5
:10653000932020702046582229460830FAF744FE5E
:10654000002070BD0E4808A15030EAE710B50020C9
:106550000C4C0D490346C2008C525218401C0006D8
:10656000D370000EF7D010BD7372635C67617474F2
:10657000635F636F72652E63000000005A020000C3
:10658000B3030000FFFF000058000020FE49088010
:106590000120887000207047FB49002088707047F8
:1065A00010B50021F848C94301800021C17007F0EF
:1065B0003BFAD8E7F7B584B005460027684607815F
:1065C000878068680C46008800F0ECFB0646287A55
:1065D000032805D0002E03D1EC49ED480EF001FD53
:1065E000297A2046C91E123000900B000EF0EAFDF9
:1065F0000FF2F1F03D09AA465C6D34B3CDF38B8BFD
:10660000F000F078012803D0E049AD200EF0E9FC5D
:10661000A8896946C0000E30888030200881002C8F
:1066200022D068680188A180E7802781A989A1819B
:1066300000200DE0C100B27909190A74B288CA813C
:1066400082005219D3894B82128A401C8A8280B2FE
:10665000A1898142EED8D7E002A8009001AB224682
:106660002946304600F0CCFBF1E002A8009001ABD7
:1066700022462946304600F005FCE8E0F07806287E
:106680001AD0FF20C149223014E068680188A18037
:10669000E7802781A989A181B188E181E9892182E7
:1066A000EA89296900982BE0F078062804D0FF20B9
:1066B000B6493C300EF095FCE88969461230888076
:1066C00035200881002CE0D1C1E0F078072804D003
:1066D000FF20AE4956300EF084FCA88969460E3082
:1066E000888036200881002CBED068680188A1808F
:1066F000E7802781A989A1812046AA890E302969CE
:106700000EF0D2FA80E0E8896946123080B2382271
:1067100088800A81002C79D068680188A180E78090
:106720002781A989A181287A102809D00221A17383
:10673000E9892182EA89296900980EF0B5FA86E094
:106740000121F4E702A8009001AB22462946304619
:10675000FFF716FD7BE0F078082803D08B498D48C1
:106760000EF03FFC14206946888037200881002CF9
:106770006DD068680188A180E7802781A989A181FF
:10678000678227820120A0733EE0F078092804D0B8
:1067900080487E4918300EF024FC288A694614305F
:1067A000888037200881002C51D068680188A1803A
:1067B000E78004212781A173A989A181E989218228
:1067C000298A618220462A8A1430696998E702E0A2
:1067D00038E01CE024E0F0780A2804D06D486B49CA
:1067E00033300EF0FEFB1420694688803720088184
:1067F000002C2CD068680188A180E78027810521C2
:10680000A173A78127826782F77020E017E002A8B2
:10681000009001AB224629463046FFF78EFD16E078
:106820000D206946392288800A81002C07D001207A
:10683000E08055480188A1802781277307E00699E9
:10684000088010E08F205149C0000EF0CAFB684656
:10685000069980880880002C05D068460089208031
:10686000684680886080002007B0F0BDF7B594B01E
:1068700015460F46149800F0A0FA04000AD0032031
:1068800000F088FB022802D2E078002804D0112012
:1068900017B0F0BD4048FBE7172069460126088382
:1068A000002D0FD00321684601711021018210A82C
:1068B0000246059004A928460AF033FD00280DD0B1
:1068C0000720E5E708216846017100210781C943D7
:1068D000418105218673C90281810CE0A878A071ED
:1068E0002888A080684605218673C902818100211D
:1068F0000781C943418109AA023206A901A807F00C
:10690000CCF8002802D000F06BFAC1E707A800908D
:106910006846038B04220321149800F051FB0028E1
:10692000B6D1E670B4E770B592B00D0006460ED051
:1069300000F043FA04000CD0032000F02BFB0228E7
:1069400002D2E078002806D0112012B070BD1020CD
:10695000FBE71148F9E7172168468180042101729D
:10696000298881816988C181012181740B49018253
:106970000AAA023201A902A807F08FF800280FD056
:1069800000F02EFAE1E700005800002068650000E2
:106990003C040000630200000230000002280000F6
:1069A00008A800906846838804220321304600F03E
:1069B00007FB0028C9D10221E170C6E770B592B08B
:1069C0000D0006460DD000F0F8F904000BD00320AE
:1069D00000F0E0FA022802D2E078002805D0112069
:1069E000B3E71020B1E7FA48AFE717216846818086
:1069F00004210172298881816988C1810121817402
:106A0000F44901820AAA023201A902A807F045F856
:106A1000002802D000F0E4F997E708A80090684643
:106A2000838804220321304600F0CAFA00288CD162
:106A30000321E17089E770B592B00D0006460DD0D4
:106A400000F0BBF904000BD0032000F0A3FA0228E9
:106A500002D2E078002805D0112076E7102074E7F4
:106A6000DB4872E7022168460172298881816988C2
:106A7000C181172181800AAA023201A902A807F068
:106A80000CF8002802D000F0ABF95EE708A80090EF
:106A90006846838804220321304600F091FA0028DA
:106AA000DBD10421E17050E7F0B591B015000E463E
:106AB00007460ED000F081F904000CD0032000F04E
:106AC00069FA022802D2E078002806D0112011B01D
:106AD000F0BD1020FBE7BE48F9E71721684681802A
:106AE00004210172298881816988C181B17881740A
:106AF000318801820AAA023201A902A806F0CDFF5C
:106B0000002802D000F06CF9E1E708A80090684680
:106B1000838804220321384600F052FA0028D6D197
:106B20000521E170D3E7F7B592B015460E461298ED
:106B300000F043F904000AD0032000F02BFA0228E9
:106B400002D2E078002804D0112015B0F0BDA04892
:106B5000FBE70627002D12D0684607728681C581A3
:106B6000A5801720694688800AAA023201A902A8D6
:106B700006F093FF002807D000F032F9E5E7052181
:106B8000684601728681EBE708A800906846838812
:106B900004220321129800F013FA0028D5D1E770DF
:106BA000D3E7F7B592B016460D000ED0129800F05C
:106BB00004F904000BD0032000F0ECF9022802D203
:106BC000E078002805D01120BFE71020BDE78048FD
:106BD000BBE70727684607728681172104958180E5
:106BE0000AAA023201A902A806F057FF002802D023
:106BF00000F0F6F8A9E708A8009068468388042208
:106C00000321129800F0DCF900289ED1E7709CE780
:106C1000F3B5172091B00C46002915D021780B0050
:106C20000EF0D0FA062B05051A041C2B1520C01EE9
:106C3000E28880B2002A02D0A368002B04D08242EE
:106C400004D90C2013B0F0BD1020FBE7042905D0B7
:106C5000A088002811D101E00620F3E7119800F088
:106C6000ACF805000BD02078092701281AD002289B
:106C700007D0042824D0052835D00720E2E754485F
:106C8000E0E76846077161880181E1884181A06879
:106C900008260390304600F07DF9072829D34C4898
:106CA000801CCFE70C216846017161880181E18871
:106CB0004181A06803900EE0E878002811D118E027
:106CC0000D216846017161880181A1884181E188B7
:106CD0008181A06804900326304600F05BF9022809
:106CE000EAD31120AEE70E2168460171217B0172C3
:106CF000F1E717216846018309AA023206A901A813
:106D000006F0CBFE002802D000F06AF89AE707A848
:106D100000906846038B04223146119800F050F928
:106D200000288FD12178012907D002298AD004298F
:106D300005D0052905D0032084E7082102E0EF7083
:106D400080E70A21E9707DE730B591B00C46054631
:106D500000F033F8002808D0032000F01BF90228C7
:106D600005D31B48801C11B030BD1948FBE70F212B
:106D70006846017104811721018309AA023206A91C
:106D800001A806F08AFE002802D000F029F8EAE700
:106D900007A800906846038B04220321284600F0D0
:106DA0000FF9E0E70C49884205D00C490988814277
:106DB00001D10A4870470020704710B5FFF7F2FF75
:106DC000002802D08178C90700D1002010BD000042
:106DD0000230000003280000FFFF000058000020E0
:106DE000002806D0012805D0052805D0062805D0A2
:106DF0000320704711207047082070475C48704797
:106E0000FFB583B003980C9EC0781D4614460F460C
:106E1000012803D05749D2200EF0E3F8F889C000CA
:106E20000E30288030203080387B001FC0B20190A7
:106E3000002C26D078680088A0800020E080208187
:106E4000F889A081002616E0F0000519C01900900D
:106E50002A4641690E3201980AF03DFA002802D014
:106E600000202874E8810098761C008A68820098C7
:106E7000B6B2408AA882A089B042E5D80399002022
:106E8000C870F1E4F8B50646C0781F4614460D46B2
:106E9000042804D0FF20374903300EF0A2F8A88957
:106EA000062148430E30388033210698002C01809B
:106EB0001AD068680088A0800020E0802081A9891D
:106EC000A18103460CE01946062251434A190919CB
:106ED000D789CF81977C8F74128A5B1C0A829BB200
:106EE000A1899942EFD8F070F8BD70B514460546F7
:106EF000142204981A8037220280002C18D0486887
:106F000000260088A080487AFF300130E080C889E0
:106F10002081C889A0816682E878082809D00928DC
:106F200011D00A2819D0134913480EF05AF8EE7000
:106F300070BD087B0C2804D00F480E490C380EF0A9
:106F400050F8012012E0087B0D2804D00A480949B6
:106F500008380EF046F8042008E0087B0E2804D01C
:106F600005480449001F0EF03CF80520A073DEE739
:106F70000330000068650000820300000146002025
:106F8000F74A02E0401C082803D24300D35A8B4240
:106F9000F8D1704730B50446F14A0020163A11790D
:106FA00053790AE05518AD79A54201D1401CC0B211
:106FB000491CC9B2102900D100218B42F2D130BD49
:106FC000FFB5E74881B0163841790A9C491CCDB21B
:106FD0001E46102D00D10025E14816380079A84240
:106FE00002D1042005B0F0BD0820FFF7D3FF07460B
:106FF000072804D9FF20DBA1A1300DF0F2FF029891
:10700000082801D1072F17D001982080301D6080FB
:10701000002060712071E68003982081204606F0F0
:10702000EDFC00280AD0CE48029916384379821D1B
:10703000995445710020D5E7CF48D3E7FF20C9A177
:10704000B3300DF0CEFF0320CCE7F0B58DB0044691
:1070500000256846057116468C460620FFF79AFF04
:1070600000281CD121780127C807002801D0132946
:1070700017D9684687766178C17602218183C583F6
:1070800004A8009070680C23008805220621FFF7F1
:1070900097FF002803D0B3A184200DF0A2FF0DB00C
:1070A000F0BDAF4816380278002AF8D042786378ED
:1070B0009A42F4D1012918D0132919D16146062921
:1070C00016D10570002101200AF034FE68460771D0
:1070D000706801886846C1800021C94301816079D8
:1070E00022790102114368461AE06146062908D058
:1070F000684600790028D2D0314601A8FDF7A7FEE6
:10710000CDE70570002101200AF014FE68460771E2
:107110006079227901021143684601810021C94347
:107120004181E9E78E4810B50021163801704A1EEA
:10713000428041700171417101200AF0FBFD10BDD8
:1071400010B5FFF7EFFF0020854902464300401CC1
:10715000CA520828FAD310BD10B50446FFF7E2FF63
:107160007F4816384480002010BDDBE770470EB51D
:1071700001216846017081498180C1800021FDF7AD
:1071800066FE0EBDF7B505460078002700090C46DF
:107190003E46012804D0FF2072A164300DF021FF8B
:1071A000287A02280CD0FF206EA17A300DF019FF4A
:1071B0000298002C068001D0278066800020FEBD4A
:1071C000EA89702710460A3086B2002C0BD0686816
:1071D0000088A080A8892081E28020460A302969A1
:1071E0000DF062FDE4E702980680E7E7F8B5436832
:1071F0000246D9799C79090221435C7A1E7A2502DC
:107200005C88981D3543241FA1421DD11B79022B98
:107210001AD1042D19D0052D26D0062D19D0402DB8
:1072200012D3061D0F4614462846FFF7A7FE08286E
:107230000AD01120207002202072A581E7812661EA
:107240006078082108436070F8BD001D00F0D9F88F
:10725000F8BD041D0D46FEF7F9FE0028F8D02946BA
:107260002046FDF730FEF8BD001DFFF7EEFEF8BD2D
:1072700010B53B4C8AB0163C2278012A26D0122346
:107280006A46937363789B1CD373082313820B881D
:1072900053824B8893828B88D382C988118301A93A
:1072A00000910C2305220721FFF78AFE00280BD14D
:1072B0000022F023114601200AF097FC01202070E3
:1072C0006078801C607000200AB010BD1120FBE7C0
:1072D000F8B5234C0027163C0646A51D1BE0607937
:1072E0002179884204D187201EA180000DF079FE0B
:1072F0002079405D042804D0082804D17F1CFFB207
:1073000001E0FDF7F2FD2079401CC0B22071102889
:1073100001D1002020713046761EF6B20028DED161
:107320003846F8BD10B50446402801D2072010BDEC
:10733000FFF724FE082802D03120000210BD0021F2
:10734000074802E0491C082903D24A00825A002A51
:10735000F8D1082914D049004452002010BD000083
:10736000DA1300207372635C6C326361705F636F69
:1073700072652E630000000004300000FFFF000073
:107380000420EBE700B5402801D2072000BDFFF73D
:10739000F5FD082805D000213B4A4000115208465F
:1073A00000BD052000BDF0B58BB016460C000746A9
:1073B00007D0002E05D06188402904D207200BB0E9
:1073C000F0BD1020FBE72088002801D0172801D944
:1073D0000C20F4E70846FFF7D1FD08280FD02588D8
:1073E00003A82A46314602300DF05EFC01A8009049
:1073F00062882B4608213846FFF7E2FDDFE70520CB
:10740000DDE7F0B50E46074601468BB01446012570
:10741000304606F0BFFC08281CD1002069460885CC
:107420000120FFF7B7FD002802D117206946088523
:1074300003AB02330AAA39463046009407F0BDF880
:10744000002809D0022818D0032803D00F49FC20B7
:107450000DF0C7FD2846B2E76846038D002BF9D032
:1074600001A800906068042200880121FFF7A8FDB0
:107470000028EFD00549E720EAE7607800251021D1
:1074800008436070E6E70000DA1300206473000030
:10749000002803D08178012939D101E010207047FC
:1074A0000188FA4A881A914233D01BDCF84A881ABC
:1074B00091422ED00BDC00292BD00320C002081AE9
:1074C00027D0012825D001210903401A07E001280F
:1074D0001FD002281DD0FF281BD0FF3801380028FC
:1074E00015D116E0FF220132811A904211D008DC3A
:1074F00001280ED002280CD0FE280AD0FF2806D181
:1075000007E0012905D0022903D0032901D000207A
:1075100070470F20704700B50A2821D008DC03000F
:107520000DF050FE0A1C2024241A24282224261A96
:10753000102819D008DC0B2816D00C2814D00D28E0
:107540001AD00F2808D111E011280FD0822807D0B7
:1075500084280DD085280DD0032000BD002000BD5B
:10756000052000BDCB4800BD072000BD0F2000BD99
:10757000042000BD062000BD0C2000BD70B5002910
:107580000BD0CB1FFA3B81241E46CDB2112B1BD250
:10759000012805D0022806D009E0002010701DE067
:1075A000FF20043001E0FF200330814218D0330077
:1075B0000DF008FE111613131613161613161616D1
:1075C00013131313161316000846FF3881381F28AB
:1075D00003D9FF39FE39022902D81570002070BD89
:1075E0001470072070BD00B503000DF0EBFD06041C
:1075F00006040C080A0C002000BD112000BD072065
:1076000000BD082000BD032000BD00780207120F56
:1076100004D0012A05D0022A0AD10EE0000907D1C0
:1076200008E00009012805D0022803D0032801D072
:107630000720704708700020704706207047002818
:1076400007D0012807D0022807D0032807D0072039
:107650007047002004E0112002E0212000E03120EA
:1076600008700020704738B50C4605004FD06946B9
:10767000FFF7CBFF002822D120880321890288430D
:10768000694609788907090D084320806946681C06
:10769000FFF7BBFF002812D121880320000381439C
:1076A000684600788007800C01432180A878400755
:1076B000820F2020012A03D0022A03D0072038BDE0
:1076C000814300E00143218088B20105890F08D081
:1076D000012189038843A9780907C90F8903084351
:1076E000208080B28104890F0AD0A9784004C9069D
:1076F000C90F400CC903084320808004800F02D1C9
:107700002088400403D520884021084320800020A1
:1077100038BD70B504460020088015466068FFF744
:10772000A2FF002815D12189A089814210D8616863
:10773000594E8978C90707D0711E884208D831464A
:107740000DF02CFB298009E0FF21FF31884201D98F
:107750000C2070BDFF30FF300330288060688078D7
:10776000C007A08903D031460DF018FB03E0FF30BD
:10777000FF30033081B22980206881784748017347
:1077800020684649008820394885002070BD10B522
:10779000137804785B08E4075B00E40F234313705D
:1077A000FD2423400478A407E40F640023431370EE
:1077B000FB24234004786407E40FA40023431370E0
:1077C000F724234004782407E40FE40023431370D4
:1077D000EF2423400478E406E40F240123431370CC
:1077E000DF2423400478A406E40F640123431370CC
:1077F0000078BF244006C00F23408001034313706C
:10780000002906D00878C10701D1800701D50120E1
:1078100000E00020C0015906490E0843107010BD59
:1078200030B50A8803239B0204889A4323059D0FE1
:1078300002D1A3049C0F01D09B0F00E001239B0207
:107840001A4303230A801B039A4303889804840F76
:1078500002D11805830F01D0800F00E00120000342
:1078600002430A8030BDF3B591B00D0018D01198D5
:10787000002818D0122128460DF073FA01A9012022
:1078800007F097FE00242646374677E002290000DD
:107890000128000003300000010200000C14002049
:1078A000102013B0F0BD0720FBE76846007C0128DC
:1078B0000BD16846C1890520C002081A0AD00128E8
:1078C0000AD002280CD003280CD0042C0ED0052C92
:1078D0000FD10DE0012400E002246846868908E00B
:1078E000032406E068460424878902E0052400E0BA
:1078F000062468468189119881423FD12C74002E5C
:107900003AD00BA800900CAB10220021304607F0B3
:10791000E2FE002820D16846808D2A46C0B20CA91C
:1079200009F0D9FC002817D1AE81002F24D00BA874
:10793000009006AB13220021384607F0CCFE002849
:107940000AD16846808D06A9C01E0331C0B22A1D27
:1079500009F0C1FC002801D00320A2E76846817E1F
:10796000427E08021043E881062C05D16846007C5F
:10797000A8726846C0892881002092E701A807F014
:1079800020FE002891D0FFF7C6FD8AE7002804D02A
:10799000012903D0022904D003207047F949C98D79
:1079A00002E0F8494031C988814201D10020704786
:1079B0000720704730B5F34C0025608B91B0C00BA9
:1079C0002ED1216900292BD0207B800728D40122C9
:1079D00068460271027200224272228B8281A28A60
:1079E000828204911721018309AA0023023206A989
:1079F00001A807F095F9002803D0FFF7F4FD11B0B6
:107A000030BD207B02210843207307A800906946FF
:107A10000B8B208804220121FFF7D2FA05460BE0E8
:107A2000FBF792FC842101700921017218341ECCED
:107A30000C301EC0FBF7A4FC2846E0E710B5D14C83
:107A4000034621690020002909D021460122103176
:107A50001846FBF754FE00202061A0820120217B04
:107A6000F9221140217310BD70B50C4605461C214A
:107A700020460DF076F900202080002D08D0012D41
:107A800004D0C1A1C5480DF0ACFA70BD062000E0DD
:107A90000520A07070BD10B507F06AFB10BDFEB5E3
:107AA0000546007800260C46374603000DF08AFB99
:107AB0000C91070C1D962F462F46486C89916868DB
:107AC0000A38FBF781FD89E0002904D0B348AEA154
:107AD0001B300DF086FAFBF737FC0446407808218E
:107AE00008436070FBF74CFC78E0002C04D1BB200D
:107AF000A5A180000DF075FA284601F0A2FA002831
:107B00006CD06078082108436070022666E0E8883F
:107B1000694608800190002C04D1A0489AA12F301A
:107B20000DF05FFA287807281CD10198C00B19D0F6
:107B3000944800218171A988818012E003264DE0DC
:107B4000002C04D1C52090A180000DF04AFA8D4888
:107B5000017B89070BD50069002802D0E888C00B9B
:107B60003CD00226607808210843607036E0291D69
:107B70008EC918308EC0283801880226012220467E
:107B8000FBF79FFD0127EDE7002C04D183487EA180
:107B900064300DF026FA7B480821007B4007C00FB7
:107BA0004600607808436070002E17D128790128BC
:107BB00002D16879002811D02046FFF73FFF074621
:107BC0000CE0002CCED10D206FA180010DF009FA40
:107BD000C8E772486CA17A300DF003FA002C0CD083
:107BE0006078000709D5002F07D184202070204637
:107BF000582229460830F9F7E7FA3046FEBDF7B5B6
:107C0000027A88B00C46054620460C300490069255
:107C100016300027921E02903E460A315948130042
:107C20000DF0D0FA0ADF06E62AE62AE66A98C6E6EA
:107C30004288002A02D052270726DDE051271E265F
:107C4000002C7DD06A684F481288A2800122A27160
:107C50008079C0004019C089FFF705FE002877D160
:107C600048488179C9004919C98921818079C000B2
:107C70004019408AA083BFE0688A009006980728D0
:107C800017D1E889C00B14D000985127223086B252
:107C9000002C55D0A8890499FFF7E5FD002857D19D
:107CA00068680088A0800220A071A8892081012036
:107CB00041E000985027203086B2002C40D0A8899F
:107CC000FFF7D1FD002843D168680088A080A8890B
:107CD000E080287A07280AD002202072288AA08310
:107CE0000098E083204669692030009A01E0012075
:107CF000F3E70CF0D9FF7FE0698A00910169002960
:107D000002D0E989C90B22D00099512722318EB2C5
:107D100000218171A9898180002C5FD00088A0801A
:107D2000A8890499FFF79FFD002811D10220A071B6
:107D3000A88920810420A072288AE083009801E0AD
:107D40004CE005E020846969009A0298D1E703209D
:107D50000BB0F0BD007B400702D55127222601E081
:107D600050272026002C39D06868502F0088A0802A
:107D700016D00220A0712146287B0831FFF774FE3F
:107D80003AE00000EC1300207372635C6761747466
:107D9000735F636F72652E6300000000CB0200000A
:107DA000287BA11DFFF760FE0020FFF747FE23E0C0
:107DB000A9890089884207D154270626002C0DD0B6
:107DC00068680088A08017E053270826002C05D09B
:107DD00068680088A080A889E0800DE00A98068085
:107DE00010E055270726002CF8D00020A07103E0F2
:107DF000FD49FE480DF0F5F80A98002C068001D0E8
:107E0000278066800020A3E7F9480021017220380E
:107E100001814181418081718180027BF923520877
:107E200052001A40027301618182704770B5F04CB4
:107E300086B0203C208000206080A071A080694630
:107E4000012007F0B6FB102608E0019908880246D9
:107E50001207D20FB043120110430880684607F0A2
:107E6000B0FB0500F1D02069002804D0DF48DE49CE
:107E700033300DF0B6F8207B800704D5DB48DA49B3
:107E800034300DF0AEF8822D04D02846FFF743FBC6
:107E900006B070BD0020FBE7D54810B52038017B47
:107EA000012211430173002141808171818006F01C
:107EB00033FB10BD10B5CE4C0020C043203C2080C9
:107EC0000020FFF7BBFD207B40084000207310BD61
:107ED00070B5C74D0446203D287B800704D5C348B4
:107EE000C1494B300DF07DF8287BC00706D12888AA
:107EF000C049884202D02869002801D0082070BDFE
:107F0000002C08D0A088162801D2092070BD206856
:107F10002861A088A882FFF74DFD70BD10B50C4602
:107F200007F01BFB002804D0C520AF49C0000DF0AE
:107F300058F82046FFF7EFFA10BDF0B5AC4D0446F7
:107F4000203591B00020089068820E462882E88192
:107F50002946E880403908866946088308850886EE
:107F600088838882A2480E90007A1746012808D09C
:107F7000022806D0032804D0042802D0082011B01B
:107F8000F0BD9D498C425FD301208004844202D31E
:107F90009A4A944258D398498E4255D3012080047E
:107FA000864202D3954886424ED36068002814D09A
:107FB0009149884248D301218904884202D38F49DC
:107FC000884241D360892189884203D80122520224
:107FD000914201D90C20D2E7089010AA0CA9304692
:107FE000FFF797FB0028CAD106A92069FFF73BFBE2
:107FF0000028C4D1206900280CD0607880070028B0
:108000006846008B03DA8004800F6ED002E08004A3
:10801000800F6AD16846008B810617D58004800FD7
:10802000606805D0002811D0744988420CD301E063
:1080300000280BD07049884206D301218904884268
:1080400004D36E49884201D2102098E705A96069DF
:10805000FFF709FB002892D16069002808D0684624
:10806000808A0105890F01293FD18004800F3CD00F
:1080700007A9A069FFF7F7FA002880D16846808A2F
:10808000800632D46846808B81062ED4A1690029EF
:1080900006D00105890F012927D18004800F24D043
:1080A000E068002804D0007800281ED01C281CD2CC
:1080B0004F4A611C123220460992FFF768FB0321E8
:1080C00000208902884301218902411868460D91E8
:1080D0000185012181744A490182454A0FA915325F
:1080E000306809F01EF9002801D0072047E708A8EA
:1080F000007F3F49C01CC2B26A7100201031FF32BC
:1081000000900190FF3203460291039003320AA9C6
:1081100004A807F0BDF9002827D135482038008E83
:108120000B90334833893830326901461239029155
:1081300000930192039010A90A8873890CA93068F2
:1081400007F0A6F901007DD12948E9881130817036
:10815000090AC1700026009631386A79008E3146CE
:10816000099B07F014F9002802D0FFF7D4F906E7BD
:108170000E98807CC00928D068460D9901850121A0
:108180008174292109020182AE81287B617840082F
:10819000C9074000C90F08432873FD2108406178D2
:1081A00002228907C90F490008432873104800922A
:1081B0002A30811C0191029000230396114A0AA9DA
:1081C00004A807F065F901003CD1606800283BD0A5
:1081D000206900281ED106A90CA8FFF721FB6078B2
:1081E000800717D469460FE0887D00002204000054
:1081F0000C140020FFFF00000060010000200020A0
:108200000328000003020000088B032109038843B0
:1082100069460883012069468874FD4808822089E0
:10822000FC490CF0BBFD6268089BFB48019200937F
:1082300002900A460396002306A904A807F028F92D
:10824000010000E07EE07DD12078C10601D48006E7
:108250002ED568460684606900280DD105A90CA8B2
:10826000FFF7DEFA6846808A0321890288430121EC
:1082700089024118684681826946888A48210843F4
:108280006946888201208874E14808AA401C088257
:10829000E1490192891C0220DE4A029100900023EC
:1082A0000396921C05A904A807F0F2F8010063D117
:1082B0002078C0072ED068460684A06900280DD11A
:1082C00007A90CA8FFF7ACFA6846818B032080024F
:1082D0008143012080020918684681836846818BAA
:1082E000402001436846818301218174C84908AA5E
:1082F000891C0182C8480192001D0221C54A0091D3
:10830000029000230396921C07A904A807F0C0F866
:10831000010031D1E068002832D068460D9901850E
:1083200001218174BA49C91C0182E16808A80A7850
:10833000027049784170E068418868464184E0688D
:10834000017900E018E008A80171E0680722C188FF
:1083500008A84171090A8171AF4808A9801D0092DF
:1083600001910290412200230396D2000AA904A899
:1083700007F08EF8010003D00B98FFF7CFFDFEE564
:1083800003210E98002F017207D0E8883880E88911
:108390007880288AB880688AF8800020EFE5F0B5F8
:1083A00001248BB016460F46012802D002281BD1AB
:1083B00004E0684605218474C90202E068469749D2
:1083C00084740182002F11D0032100208902884388
:1083D0000121890241186846018506AA05A9384687
:1083E00008F09FFF002803D00720B1E41020AFE47D
:1083F000894DB8782E3D287338882F46203F7885E0
:108400006A46127D0020294606AB00920E31019388
:10841000FF32029103900346FF3203320AA904A8F7
:1084200007F036F8002802D0FFF775F890E4002E28
:1084300001D0F88D30802C72002089E470B592B0A4
:108440000446012508A8857075496846018406F030
:1084500096FF002208A90120FFF7A1FF064606F0BB
:1084600092FF30003AD120780024C00700283FD086
:108470001C2168460CF077FC6846017820200143F7
:108480006846017008A885706649684601841194A1
:108490000794817FF9200140891C6846817700207C
:1084A000014668460177002001466846417704216D
:1084B0008185C485018607A80A9011A80D9008A897
:1084C000099006F05CFF0EAA09A96846FFF735FD82
:1084D000054606F058FF002D02D0284612B070BDA8
:1084E0004D486946098F4E3801816946898F41811F
:1084F00049482E3804720020F0E7F7B5464E9CB08C
:1085000000212E3E0091317A012904D0022902D0A7
:1085100008201FB0F0BD40494E39CA8D824201D0BB
:108520000620F6E71D98824201D10720F1E73B487B
:10853000012110AA9176401C1083002003239B0286
:1085400002469A438B02D31810AA93846A469184F8
:108550003549D18410AA9077908317AA0A926A4667
:1085600091850C9009A807F04BF800242546274672
:1085700004A909A807F047F8002810D082287BD169
:10858000002C7CD0002D7AD010A8048145810024D5
:10859000047518A8807812AD012872D07AE0684678
:1085A000807D002F1FD0012862D16846818A1B4838
:1085B000401C814219D114A800906846408A0EAB35
:1085C0001022002107F087F8002877D110A8008A30
:1085D000042801D006285BD16846018F1D9881428E
:1085E00046D10F2095E7012842D16846808A0521AF
:1085F000C902884202D0491C884239D106484E3807
:10860000C18D6846408A814210D101270FE00000E9
:1086100001290000010200003A1400200128000096
:1086200001180000052A0000FFFF00000027002CB1
:1086300001D0002D0DD01D99884219D114A90091A7
:1086400004460EAB1022002107F045F8002835D172
:1086500001E0009D0CE010A8008A022801D010283B
:1086600016D1C0B218AA0EA908F035FE00280FD105
:108670006846408A00907BE720E000E001E00520AA
:1086800047E72A1D15A918A808F04BFE002801D0BD
:1086900003203EE710A8007D0023001DC2B210A8F1
:1086A00002751E98029019A901950394009216A8CC
:1086B00006F0EEFE002801D102213172FEF72BFFF9
:1086C00027E73EB50B46401E84B201AA002118469A
:1086D000FFF75DF806F053FE02A8009001AB0122FF
:1086E0000021204606F053FE044606F04CFE684684
:1086F0000089012803D0FE49FE480CF072FC204698
:10870000FEF709FF3EBDF0B5FB4E0446307A89B056
:108710000F46032804D0042802D0082009B0F0BD79
:1087200004AA06A92046FEF7F4FF0500F6D1F24898
:108730002389383022690146103902910093019251
:10874000039069460A8A638906A9206806F0A0FE9C
:10875000002802D0FEF7DFFEE0E7002F03D0E64856
:10876000203000893880042030722846D6E738B59A
:108770000C00054608D00022694607F006F80028DC
:1087800004D0FEF7C8FE38BD102038BD694620462B
:10879000FEF769FF0028F8D1A0786946C207D20F1A
:1087A000284607F00DF8ECE73EB50C0008D002AA09
:1087B000694606F0EAFF002804D0FEF7ACFE3EBD95
:1087C00010203EBD032120460CF0CBFA68460088FD
:1087D00001A90005800FFEF732FF00280BD1684683
:1087E000007920706846008801A98004800FFEF798
:1087F00026FF002801D003203EBD68460079607046
:10880000A278EF20024068460088C10B09010A43A4
:10881000F7210A404104C90FC9000A43A270F92197
:108820000A40800601D5012000E002204000694690
:108830000243097A50084000C907C90F0843A070D5
:1088400000203EBDFEB51D4614460E46074606F006
:1088500096FD01A8009022882B463146384606F046
:1088600096FD054668468088208006F08CFD2846E7
:10887000FEF751FEFEBDF0B50C46002199B007464B
:10888000684681850D46002C11D0E068002806D08E
:10889000A06800280BD002886B469A850180A078DA
:1088A000012806D0022804D0072019B0F0BD1020FE
:1088B000FBE72088002807D0401E80B201A906F0FF
:1088C00078FE002842D136E08C48EEE769468A8976
:1088D00021888A420BD26846007C002501282CD1D1
:1088E0006846C0898649884227D1012525E08A4209
:1088F00003D1002D2FD06D1C01E0022D02D0032DDD
:108900001BD31FE06946097C012916D169467C4BBF
:10891000CA895B1ED11A9A421DD005DC7948101A0B
:1089200019D0012809D116E0012914D0FF390139E5
:1089300003D1032506E00D26B60201A806F041FE8C
:108940000028C3D0822804D0002806D0FEF7E3FD1B
:10895000ABE7022DFAD13046A7E7E068002813D034
:1089600006F00DFD0BA800906A46A1882088928D24
:10897000E36806F00CFD054606F005FD002D19D153
:108980006846A168808D088002980078C00601D5ED
:108990005D488AE706F0F3FC0EA8009068468089DF
:1089A0000CAB0222002106F096FE054606F0EBFC19
:1089B000002D01D02846C9E76846008F022801D063
:1089C000032072E7A078012808A8007C03D0800764
:1089D0000ED4082069E7C007FBD00820FEF7DAFABA
:1089E000072802D34548401C5FE70825022001E024
:1089F000022503206946087621886846818317216D
:108A0000818611AA002302320DA906A806F088F972
:108A1000002802D0FEF7E7FD47E70FA80090684660
:108A2000838E042229463846FEF7CAFA3DE770B520
:108A3000064615460C460846FEF72AFD00280AD1D0
:108A400006F09DFC2A4621463046FFF7A8FC044666
:108A500006F099FC204670BD70B514460D460646DA
:108A600006F08DFC224629463046FFF746FD0446B7
:108A700006F089FC204670BD70B51E4614460D00F8
:108A80001AD0002C18D06168002915D00121FEF7FA
:108A90007DFF00280FD12068FEF7FAFC00280AD1DC
:108AA00006F06DFC324621462846FFF746FA04469A
:108AB00006F069FC204670BD102070BD70B51546EB
:108AC0000C0023D00221FEF761FF00280ED12068A0
:108AD000FEF7DEFC002809D106F051FC29462046AD
:108AE000FFF711FE044606F04EFC204670BD000064
:108AF000887D00003E0600000C14002003300000BA
:108B00000328000000280000013400001020EDE7D9
:108B1000FEB50746FF481C4615460E46824218D34E
:108B2000002C01D0844214D3384600F047FA0028C4
:108B30000AD1002C0FD101AA6946384606F025FE5D
:108B4000002802D0FEF7E7FCFEBD684600888006DC
:108B500001D41020FEBD23462A4631463846FFF791
:108B600071FEFEBDFFB585B01E4614000F4609D04C
:108B700003AA02A9059806F008FE002804D0FEF713
:108B8000CAFCCBE51020C9E568460089C00601D5BE
:108B9000E148C3E506F0F3FB01A800900023DF4A9B
:108BA0003946059806F097FD054606F0ECFB002DCA
:108BB00011D1002E0CD006F0E2FB0020009022889C
:108BC00033463946059806F086FD054606F0DBFB80
:108BD0006846808820802846D1E7002906D0D04BFF
:108BE0000A885B899A4201D8CE48704743E610B59F
:108BF00086B004236C46A382C94B1C89002C07D085
:108C00005B898B4201D2914204D9C64806B010BD9F
:108C10000620FBE76B4619825A82002100910191E0
:108C20001C800221997005A9029104A9039169464B
:108C3000FFF721FEEAE7F0B591B00D4681206946C5
:108C4000087105F09BFC0646002D08D02878B44C2E
:108C5000012806D0022828D0072011B0F0BD10202E
:108C6000FBE7A98801AAFEF789FC0028F5D1B00727
:108C700034D568460079002820D1A879C0071DD0D6
:108C800006F07DFB002000906A892989A088EB68A6
:108C900006F07DFB6946087106F075FB69460879A8
:108CA00000280BD0FEF737FCD7E7A98801AAFEF70A
:108CB00065FC0028D1D1342006420FD0012168463E
:108CC0000172017301794173F00609D5A1886846E4
:108CD0000182A18A01832069059004E00820BCE795
:108CE000A08869460882FAF72FFB054617206946D7
:108CF00088830AAA2B46023207A902A806F010F8B8
:108D000007466878000701D5FAF73AFB002F03D031
:108D10003846FEF768FCA0E7F00603D5207B062165
:108D200008432073B00602D50020FEF787FE08A88E
:108D3000009069468B8B208804220121FEF740F9C0
:108D40008BE7F0B5002695B014460D4600290FD0EC
:108D5000022C4FD3A71EBAB270480AF057FE291949
:108D60001039CA7B8B7B11021943884242D1BCB2B5
:108D700001A9012006F01DFC7AE0029F3888010756
:108D800076D5002D41D0A9190691CA788B78361D69
:108D90001102B6B219438919A1422BD869468A89B2
:108DA00006994B7809781B020B439A4222D1C006E0
:108DB00023D506F0E4FA07A800900698AB19C1780D
:108DC00080780A020699024348780978000208432D
:108DD000002106F0DCFA009006F0D5FA0098002891
:108DE0003ED10698C178827808026946898B104383
:108DF000884202D00B2015B0F0BD0698C178827869
:108E000008021043801986B22EE0C0062CD500203F
:108E100007AA01461154401C80B21028FAD306F06C
:108E2000AEFA06A8009068460023808910221946F1
:108E300006F051FC0090002803D006F0A4FA009838
:108E40000EE00BA86946009088890A8B07AB0021C9
:108E500006F09DFA009006F096FA0098002803D0DC
:108E6000FEF759FBC7E703E03888102188433880B4
:108E700001A806F0A6FB002800D17EE7284D6988EE
:108E8000002921D001226846027602770024447727
:108E90000184172181850EAA234602320BA906A858
:108EA00005F03EFF002802D0FEF79DFBA3E70CA8CB
:108EB000009069468B8D288804220121FEF780F8F6
:108EC000002898D16C8096E7002094E7F0B5002444
:108ED00087B015460E46002A04D002A9012006F0EC
:108EE00068FB4CE0102007B0F0BD03980078000745
:108EF00045D506F044FA01A8009068460023008A90
:108F0000064A194606F0E7FB074606F03CFA002F32
:108F10002ED109E00020002001340000FFFF0000F6
:108F2000EC13002003300000002E23D06846808818
:108F3000298820183719001D814230D36946098AD3
:108F40003970090A797069468988B970090AF97017
:108F500006F015FA01A869460090088A8A883B1D28
:108F6000002106F0B8FB074606F00DFA002F01D0ED
:108F70000320B8E7684680882018001D84B202A844
:108F800006F01FFB0028B0D0822802D0FEF7C3FAFB
:108F9000A9E7002E0ED02988A01C814201D20C2006
:108FA000A1E72246314639480AF030FD31190870F0
:108FB000000A4870A41C2C80002094E700B585B0FE
:108FC0006946FEF750FC00280AD16846007C030081
:108FD0000CF0F8F808052F2F2F2F08080531032073
:108FE00005B000BD68468078012807D16846008832
:108FF0000321C902401A1CD001281AD06846807982
:10900000012806D16846808815214902401A0528A2
:109010000FD96846807A012811D168460189292034
:109020000002081A05D0022803D0032801D0042822
:1090300005D10F20D4E7164916480BF0D2FF0020C7
:10904000CEE738B5144A0021518003791AE0CC00EC
:109050002418A46800946C462488250707D5E506E3
:1090600005D5D90008182038C08B508006E064046C
:1090700006D59171C9000818C0889080012038BDBC
:10908000491CC9B28B42E2D8002038BDFFFF000066
:10909000887D000033020000EC1300200120F84915
:1090A00040068862704770B5F54D0024AC702846C4
:1090B0006C7020304473C4762C622C756C6309F09C
:1090C00016FFEC602C61686228463C300AF0B6FD61
:1090D000002804D0FF20EBA140300BF082FFED48C8
:1090E000C46301204006A86270BD70B50125EA493D
:1090F00002260E60E749CD63E849C96AE04B0907DB
:1091000017D4E64ADC68E6494032002C04D01B69DB
:10911000002B01D04C6202E0D36A4B62136B8B626E
:10912000536BCB62936B0B63D26B0123DB071A4348
:109130004A63D349DB4C896A00282BD001282DD003
:10914000FF20D0A16F300BF04CFFD748A063FF2069
:10915000043060632563D549032008602061D1494C
:10916000962040314860D348D1494163CF49FC390A
:109170000163CF49091FC163CC49F03981630320E2
:10918000CC49000340394860CB4910204860CB48A7
:10919000066070BDCA486061CA4804E0C948E03052
:1091A0006061C848801F0143A161CEE7B44A1161E4
:1091B000D0607047B249012008707047B049002064
:1091C0000870704770477047B649403100280868FA
:1091D00002D00122104301E04008400008607047BF
:1091E00070B50C46A64D01460622E81C0BF05CFD4E
:1091F0006C7270BDA2482030407B7047A04A9170CD
:109200005070704770B50D460446082904D9FF20F8
:109210009CA1D2300BF0E5FE0022AB4809E09100A2
:10922000635809180B6053001B191B8C0B62521CEE
:10923000D2B2AA42F3D3206BA3494031086070BD7B
:109240000B23DB4310B5C21A964998421FD008DCA5
:109250001C3222D00A2A20D0142A1CD0182A08D165
:1092600017E0083011D004280DD0082809D00C28A8
:1092700005D0FF2083A1FE300BF0B3FE10BD04200B
:109280000CE000200AE0FC2008E0F82006E0F420D2
:1092900004E0F02002E0EC2000E0D820C86010BD1F
:1092A00077482030007E704710B57E4CC1786162EF
:1092B0000BF05BFD0002E06110BD252808D02628D8
:1092C00008D0272808D041000A2807D8091D06E041
:1092D000022105E01A2103E0502101E0891DC9B2F5
:1092E000704A91606F494031486170476449086233
:1092F000704770B5624C207500F028FB207DC007D8
:1093000040D06A4D2868800703D45EA16F480BF0F7
:1093100068FE207D01061DD5800707D56B4859A141
:10932000801C0BF05EFE207D000613D52078614E78
:10933000012816D0002804D0A52052A180000BF0EF
:1093400050FE63487061606A3061FF205949013006
:1093500040394860207D800714D52868C00708D1AF
:1093600002E05B48001FEDE7584846A11A300BF0B9
:1093700038FE207D4007286801D5042100E008213F
:109380000843286070BD70B500213D4C0125617710
:10939000002807D0012818D002281AD04B4839A13C
:1093A00045380BE000F0D2FA49482178001F012926
:1093B00007D0002907D08B2032A180000BF011FECE
:1093C00070BD056070BD456070BD8120FFF791FFE5
:1093D00070BD00F0BBFA206A002804D18D2029A1BD
:1093E00080000BF0FEFD216A606B40183949C860AF
:1093F000304839494030016035490C31416008142A
:109400002C49403948601E482030C57670BDF8B5FB
:109410000C2069460870284C6068C006C50F1026ED
:10942000A6602B480021FC300161294B01221B1F43
:109430001A610BE000BF00BF00BF00BF00BF00BF4C
:1094400000BF00BF6B461A78521E1A706A46127827
:10945000002A02D00269002AECD001616846007837
:10946000002804D1194807A131380BF0BAFD002DAE
:1094700000D06660F8BD0249002088627047000095
:10948000481400207372635C68616C5F7263732EB2
:1094900063000000C01F004080E100E08000001079
:1094A00000170040001500405B060000001200405D
:1094B0004480004040F501400013004080E200E09D
:1094C0000601020025000300001600408302000090
:1094D00004100040408500404C81004010B50BF066
:1094E00044FC0002FE49000AC86310BDFD49022089
:1094F0000860C3E7FB4902200860FB490860BDE73C
:10950000F849022080390860B8E7F8490870B5E7E3
:1095100010B5F7480AF09AFB002803D0F549F64841
:109520000BF05FFD10BD10B5F1480AF0A7FB10BDB0
:10953000EB494860A2E7EE4910B53C39EF4B0022F9
:1095400088615A60496B0818ED49486000F005FAD7
:1095500010BDE74810B5C6213C388161E74A0021BB
:109560005160406BE649C630486000F0F6F910BD26
:109570000120E44940028860DD4900203C398861CF
:10958000DF4948607AE7DA4900203C39486375E7EB
:10959000D748DB493C38406BFE3088606EE7D849DD
:1095A000002088606AE7D848016810229143016072
:1095B000D6490120886161E7D5490020C861D248B9
:1095C000016810221143016058E700B5FFF7EBFF77
:1095D000C74900203C39087700BD00B5FFF7ECFF14
:1095E000C34901203C39087700BDC949CA69012A2D
:1095F00001D0002042E7BA4A403292685206520E29
:10960000524202700020C861012037E7F8B5C04C13
:109610002069012806D00021B5483C38007801288F
:1096200002D004E04021F7E7E268012A04D00022DA
:109630000A43012802D004E02022F9E761680129E9
:1096400005D000211143B34A002802D007E01021C1
:10965000F8E71368012B02D1E368012B04D0002343
:109660000B43002802D007E00823F9E7116800291E
:1096700002D1E168012905D000221A439F4D00283C
:1096800002D004E00422F8E76968012904D000212F
:109690001143002802D009E00221F9E7606801289F
:1096A00004D16868012801D0012600E000269A480C
:1096B0000E4301680906090E02D06169012900D034
:1096C00000218B4F1C3F397600680006000E02D047
:1096D000A069012800D00020787689488068002899
:1096E00003D000F03FFA012800D00020B876002116
:1096F000E160216161606161A16169603046F8BD2E
:109700007B493C394877B9E6F8B5794E01271C3ECC
:10971000F07E0025002826D07B4C20680090256034
:10972000FFF775FE009820607948C56005614560C7
:10973000456185617349001488603446203C217876
:10974000724801290BD000290BD0DF206949800025
:109750000BF047FCF576607F022878D0F8BD0760F3
:10976000F8E74760F6E7FFF751FF0446604D002039
:109770003C3D6877624842682A63006868632978DC
:10978000002909D1A978002906D0554B5B681B78C0
:109790000B406978994309D000213173E10707D064
:1097A000104602F01CFD0121686B08E03773F5E7F5
:1097B000A10601D5022102E0A10702D5002102F095
:1097C0001DFD474F796806220931E81C0BF03FFA6E
:1097D000002807D1687A79680978C909884201D1D7
:1097E000012000E000207073204600F0C0F83F48E0
:1097F000C6260078002815D0012829D002283CD0A0
:10980000032859D03B4945480BF0EBFB287F002843
:1098100004D02878002861D0FFF7C5FE28780028FA
:109820005DD08CE0A00701D501F0D4FB200703D563
:109830000120AE6101F0F6FB600703D50020AE61A8
:1098400001F0F0FBA006E1D501F074FBDEE77AE061
:10985000A00701D503F00CFF200703D50120AE615E
:1098600003F085FE600703D50020AE6103F07FFEA4
:10987000A006CBD503F006FEC8E7A007BF27002847
:1098800002DA3C400AF096F8200704D53C4001205B
:10989000AE610AF08EF8600704D53C400020AE614E
:1098A0000AF087F8A00602D53C400AF081F860066D
:1098B000ACD50AF080F8A9E7A00701D50AF07EF838
:1098C000200703D50120AE610AF077F8600703D5C1
:1098D0000020AE610AF071F8A00621E025E027E043
:1098E0000015004080E100E080E200E06000002020
:1098F0008414002084940000B902000040810040DC
:109900004085004000F5014000120040001000407A
:10991000001100400014004040160040AE0400005A
:1099200000D473E70AF048F870E7FFF745FE75E7E3
:10993000A869002803D0696B091829484160687F2D
:10994000012800D00AE7F9F763FBF8BD2549032099
:10995000086088152449886090E5234823494030F1
:10996000C1612349816120494015486086E570B591
:109970000546FFF7EBFF1F4C217D080701D568075F
:109980001CD41D4AC80605D5507E002802D0907E02
:10999000002813D0880602D5107B00280ED1480677
:1099A00002D5507B002809D000208A070026002A13
:1099B00007DA4A0704D50122227002E00120F4E709
:1099C0002670CA0709D0AA0705D4890705D500283B
:1099D00003D0A80601D4FFF71AFD267570BD00005C
:1099E000408500400012004000F50140101000408A
:1099F0004481004048140020681400202E480021B3
:109A000001704170704770B5064614460D4601203E
:109A1000F7F762FE28490120284B08709E60DC6041
:109A20001D6170BDF8B504460120F7F755FE2249C7
:109A30000120087021494C60214900264E60032115
:109A4000204D8902A960204F002C0AD0012C03D0A0
:109A50001EA140200BF0C5FA3E6003208002686022
:109A6000F8BD386001208002F9E710B5124801788E
:109A700000290ED00321134A8902916010494A68D7
:109A80000021002A03D0154A1268427000E041709C
:109A900001700020F7F720FE10BD0748017800296B
:109AA00007D007484068002802D00C480068C0B2C0
:109AB00070474078704700006100002000F50040CA
:109AC00000F1004000F5014000F200407372635C59
:109AD00068616C5F63636D2E6300000000F40040FA
:109AE000364800210170417010218170704770B5B7
:109AF000064614460D460220F7F7EEFD01202F49D9
:109B00002F4A0870E41E14619660556070BD10B550
:109B10000220F7F7E1FD29490120087029480021BA
:109B20000160416081602849C014486010BD10B5D3
:109B3000224C2078002811D001202349C0028860DF
:109B400000F02EF80021002804D0012060701F488A
:109B5000006801E061701020A07021700020F7F70C
:109B6000BBFD10BD10B515480178002905D000F0E7
:109B700017F8002800D0012010BD407810BD10B5A6
:109B80000E480178002909D000F00AF8002803D017
:109B90000E480068C0B210BD102010BD807810BD06
:109BA00008480168002905D04168002902D0806872
:109BB000002801D00020704701207047630000207A
:109BC00000F5004000F1004000F5014000F40040C5
:109BD00010B528210BF0C5F810BD40788006800E26
:109BE000704740788006800EC01C70472820704760
:109BF00070B5054600780A0700090001120F1043EE
:109C000028700B000BF0DEFA0705070507050905AC
:109C10000B00062408E00C2406E0222404E00024C3
:109C2000FEA158200BF0DDF96878800980012043FF
:109C3000687070BD00780007000F704710B50622ED
:109C4000C01C0BF031F810BD0B4610B5C11C06222C
:109C500018460BF029F810BD10B5062209300BF09C
:109C600023F810BD0B46014610B5062209311846EF
:109C70000BF01AF810BD0278BF23C9071A40490E2D
:109C80000A430270704700784006C00F70470278A0
:109C90005206520EC9010A43027070470078C0098B
:109CA000704770B50C460546C11C20460622093097
:109CB0000AF0FAFF20784006400E20702978490605
:109CC000C90FC9010843207070BD70B515460E4616
:109CD00004461F2A03D9D1A1A9200BF082F92046FE
:109CE0002A46314609300AF0DFFF6078AD1D800951
:109CF0008001A906890E0843607070BD70B50546E5
:109D000040780E468406A40E062C03D2C3A1B920C7
:109D10000BF067F9A41FE4B21F2C00D91F242946B9
:109D20002246093130460AF0BFFF204670BD70B5AB
:109D300015460E4604461F2A03D9B8A1CD200BF0C4
:109D400050F920462A46314609300AF0ADFF6078C6
:109D5000AD1D80098001A906890E0843607070BDA1
:109D600070B5044640780E468506AD0E062D03D22A
:109D7000AAA1DE200BF035F9AD1FEDB21F2D03D9DE
:109D8000A6A1E2200BF02DF921462A4609313046E2
:109D90000AF08AFF284670BD10B504220F300AF081
:109DA00083FF10BD0B46014610B504220F31184643
:109DB0000AF07AFF10BD10B5032213300AF074FFC9
:109DC00010BD0B46014610B50322133118460AF0A8
:109DD0006BFF10BD4176090A81767047817E427E15
:109DE000080210437047C176090A01777047017F66
:109DF000C27E0802104370474177090A8177704795
:109E0000817F427F080210437047C175090A0176BD
:109E10007047017EC27D080210437047817570470C
:109E2000807D704720300279C90652095201C90E5F
:109E30000A430271704720300079C006C00E704797
:109E400020300279D206D20E49010A4302717047CE
:109E5000203000794009704710B505221F300AF004
:109E600023FF10BD0B46014610B505221F311846D1
:109E70000AF01AFF10BD30B5411C837E0A46190254
:109E8000D37D447E927D1B0221431343674D827D27
:109E90008C1FAC4210D8002A0ED0082A0CD88A4257
:109EA0000AD28B4208D8817F427F08021043A91D45
:109EB000884201D8012030BD002030BD00210A4673
:109EC0004254491C2229FBDB70474078C006C00E73
:109ED00070474078C006C00EC01C704722207047F3
:109EE00010B502788B07920892009B0F1A430270FC
:109EF0004278520952014270012908D0022906D045
:109F0000032905D0FF2045A1A3300BF06AF810BD4E
:109F100001210A43427010BD10B502788B079208E8
:109F200092009B0F1A43027042785209520142700C
:109F3000012908D0022906D0032905D0FF2037A126
:109F4000BD300BF04EF810BD01210A43427010BD28
:109F500000788007800F70470278FB23C9071A40FA
:109F6000490F0A430270704700784007C00F7047DE
:109F70000278F723C9071A40090F0A430270704795
:109F800000780007C00F70470278EF23C9071A4016
:109F9000C90E0A43027070470078C006C00F7047B0
:109FA00070B50546C1700B000BF00CF90E080A0CD9
:109FB0000E1012120C14141212160C180C2413E0AA
:109FC000082411E002240FE017240DE00D240BE01B
:109FD000012409E0092407E0062405E045200024C7
:109FE0000EA1C0000AF0FDFF68784009400120433F
:109FF000687070BDC078704770B5044640780E46F2
:10A00000C506ED0E1B2D03D904A109480AF0E9FF8E
:10A010006019C01C042231460CE000007372635CBE
:10A02000756C5F7064752E63000000007A0C000090
:10A030003A0200000AF038FE70BD70B50446407860
:10A040000E46C506ED0E1B2D03D9A049A0480AF007
:10A05000C8FF6119C91C042230460AF025FE70BDF4
:10A06000C171090A01727047017AC279080210436E
:10A0700070474172090A81727047817A427A0802F8
:10A0800010437047C172090A01737047017BC27A9D
:10A090000802104370474171090A81717047817944
:10A0A0004279080210437047017170470079704788
:10A0B0004173090A81737047817B427B0802104318
:10A0C000704730B5411C037A0A46C479190221430E
:10A0D000537914791B0223437E4D00798C1FAC42C7
:10A0E00010D800280ED008280CD888420AD28B42FB
:10A0F00008D8D07A917A00020843A91D884201D875
:10A10000012030BD002030BD10B50522001D0AF031
:10A11000CBFD10BD0B4610B5011D052218460AF0F7
:10A12000C3FD10BD4172090A81727047817A427A7B
:10A13000080210437047017170470079704710B5ED
:10A140000822001D0AF0B0FD10BD0B4610B5011D20
:10A15000082218460AF0A8FD10BD0A780273497853
:10A1600041737047027B0A70407B4870704710B59E
:10A1700008220E300AF098FD10BD0B46014610B5BE
:10A1800008220E3118460AF08FFD10BD10B50422CA
:10A1900016300AF089FD10BD0B46014610B50422A9
:10A1A000163118460AF080FD10BD10B50822001DBA
:10A1B0000AF07AFD10BD0B4610B5011D08221846A5
:10A1C0000AF072FD10BD10B504220C300AF06CFDCF
:10A1D00010BD0B46014610B504220C3118460AF09A
:10A1E00063FD10BD017170474171090A81717047AB
:10A1F000C171090A0172704700797047817942790B
:10A20000080210437047017AC27908021043704770
:10A21000017170470079704701717047007970478C
:10A2200010B50822001D0AF03FFD10BD0B4610B509
:10A23000011D082218460AF037FD10BD10B508228E
:10A24000001D0AF031FD10BD0B4610B5011D08229E
:10A2500018460AF029FD10BD70B515460E46044695
:10A260001B2A04D93720194900010AF0BAFE2A46F0
:10A270003146E01C0AF018FD6078E906400940010B
:10A28000C90E0843607070BD70B5054640780E4633
:10A29000C406E40E1B2C04D9DF200C4980000AF010
:10A2A000A0FE2246E91C30460AF0FEFC204670BDA6
:10A2B0004078C006C00E1B2801D80120704700203E
:10A2C000704710B522220AF0EFFC10BD1CA0000060
:10A2D000430200007A0C0000FEB50F46044601461A
:10A2E000064620302546C031603640350190032FA8
:10A2F00004D0002F2DD0012F2BD04BE00020608008
:10A30000A080E08020816081A082E085E082687486
:10A31000A074E074A076E076A073E073207460749B
:10A32000019B987401232B74A88228830876E88304
:10A33000B0706883A873E87320776077019988729A
:10A340000199087430727072B0723274B074A8835C
:10A35000FEBD0020A8822883012F52D0E08B009000
:10A36000608C0290C00000990AF018FD401C80B279
:10A37000E8820099192241439202914201DD401E78
:10A38000E8827D20000200990AF008FD401C308020
:10A39000002F01D0022FDBD10198007AC10601986D
:10A3A000C90E017200206873221824218B5C403290
:10A3B000D9075B08DE07C90FF60F71185B08DE07C7
:10A3C000F60F71185B08DE07F60F71185B08DE07E1
:10A3D000F60F71185B08DE07F60F71185B08DE07D1
:10A3E000F60F76185908891911726A7B401C5118AA
:10A3F000C0B269730528D7D3002FA9D10020A87453
:10A40000FEBD4A7F2046E030022A12D0097F022991
:10A4100013D050A173200AF0E4FD012000900290B7
:10A42000E08BA98B484300990AF0C6FCA8830298E8
:10A4300098E7818800910089F1E7018A0091808A7C
:10A44000EDE770B504464034667B0546002E68D0C3
:10A45000252E66D8002964D03E20405DA27B48436B
:10A46000101825210AF09AFC0846A1734207C90872
:10A47000520F3C4B691820319A5C09798A4367D0A6
:10A4800031460AF08BFC491CCAB2002006E00028C5
:10A4900004D029184031C979511ACAB22918482361
:10A4A0005B5C93423AD320310979C943CB07DB1770
:10A4B000D21A521E1206120E34D08B07DB17D21A94
:10A4C000521E1206120E2FD04B07DB17D21A521E45
:10A4D0001206120E2BD00B07DB17D21A521E1206D1
:10A4E000120E27D0CB06DB17D21A521E1206120EFE
:10A4F00023D08B06DB17D21A521E1206120E1FD063
:10A500004B06DB17D21A521E1206120E1BD009067A
:10A51000C917511A491E0A06120E17D0401C0528E9
:10A52000B5DB70BDC00013E0C000401C10E0C000EF
:10A53000801C0DE0C000C01C0AE0C000001D07E048
:10A54000C000401D04E0C000801D01E0C000C01D2F
:10A55000E07370BD7372635C6C6C5F7574696C2EB4
:10A5600063000000FC51010010B5FF48002101709C
:10A5700041708170C17041718171C171083009F001
:10A580005DFB002804D0FF20F8A184300AF029FDEB
:10A5900010BD10B5F44900204872081D09F04EFBAB
:10A5A000002804D0FF20F1A1C3300AF01AFDFFF704
:10A5B000DBFFF148FFF782FC0021EF48FFF7E4FCE6
:10A5C0000121ED48FFF78CFC10BDE2E71B2070472E
:10A5D000E5494A7A002A01D00020704748810120CD
:10A5E0004872704710B5E0494A7A002A02D049897A
:10A5F000814201D0002010BDDB48001D09F026FB80
:10A60000002804D0FF20D9A1B4300AF0EAFCD648D3
:10A61000001D09F033FBFFF7A7FF012010BD70B547
:10A62000D14C0025627A002A02D06289824201D090
:10A630000D700DE0227863789A4203D32278637814
:10A64000D21A04E062782378D21A10239A1A0A7078
:10A65000FFF7C8FF002801D06572012070BDC24914
:10A660004A7A002A04D04989814201D101207047E9
:10A6700000207047BC490A784B78521C1207120F11
:10A680009A4207D0097822225143BC4A89180160B6
:10A690000120704700207047B34801784278491C78
:10A6A0000907090F914206D00178491C0907090FD3
:10A6B00001700120704700207047AB494A7A002A98
:10A6C00004D04989814201D10120704700207047A0
:10A6D000A5490A784B789A4207D0497822225143FB
:10A6E000A64A89180160012070470020704710B504
:10A6F0009D4C20786178884216D06078401C000715
:10A70000000F6070201D09F0A1FA002804D0E07845
:10A71000401CE070012010BDA078401CA070924841
:10A72000001D09F0ABFAF5E7002010BD8E48017856
:10A730004078814201D101207047002070478A484B
:10A7400001784278914202D30178407803E0417861
:10A750000078081A1021081AC0B270470F207047FD
:10A7600070B5814C0D46617A002916D0618981420D
:10A7700013D100262E70201D09F068FA002805D19B
:10A78000A0782870A670201D09F078FA2878E17862
:10A7900040182870E670012070BD002070BD764919
:10A7A0000160704770494A7A002A04D04989814281
:10A7B00001D101207047002070476B494979002979
:10A7C00001D0002070476E49016001207047664843
:10A7D0004179002901D000207047012141710846CC
:10A7E000704761494A7A002A04D04989814201D1DF
:10A7F00001207047002070475B494979012901D049
:10A80000002070475E490160012070475648417939
:10A81000012901D0002070470021417101207047BB
:10A8200051484079012801D001207047002070472D
:10A830004D494A7A002A04D04989814201D1012038
:10A8400070470020704770B5474C0546A079072136
:10A85000401C0AF0A3FAE079814208D0A0792221B5
:10A8600048434749223140182860012070BD00202C
:10A8700070BD10B53C4C0721A079401C0AF08EFA3F
:10A88000E079814207D0A0790721401C0AF086FABE
:10A89000A171012010BD002010BD33488179C0791D
:10A8A000814201D101207047002070472E494A7A29
:10A8B000002A04D04989814201D10120704700203B
:10A8C000704710B504462848083009F0BFF9002841
:10A8D00015D125498879CA7990420CD0C8792221AE
:10A8E000484327492231401820601F48083009F0AA
:10A8F000C5F9012010BD1C48083009F0BFF900203F
:10A9000010BD10B504461848083009F09FF900281A
:10A9100015D115498879CA7990420CD0C87922217D
:10A92000484317492231401820600F48083009F089
:10A93000A5F9012010BD0C48083009F09FF900204E
:10A9400010BD094810B5083009F080F9002822D15F
:10A95000054CA079E17988421AD0E0790721401CA2
:10A960000AF01CFAE1710DE0660000207372635C6E
:10A97000646D5F712E630000B817002088140020FA
:10A98000A81600202046083009F078F9012010BDF3
:10A990000C4809F073F9002010BD0A480838817985
:10A9A000C079814201D101207047002070470548DD
:10A9B00008388179C079814201D101207047002097
:10A9C000704700006E00002070477047FF207047FE
:10A9D0007047704700207047002070470020704784
:10A9E000002070470020704700207047002070470B
:10A9F00000207047002070470120704700207047FA
:10AA0000002070470020704700207047F8B5FE4DC9
:10AA10000446287F002600280AD0002921D166702C
:10AA200010202070687FA070A87FE0702E7718E05B
:10AA3000A879012801D00020F8BD002911D1667045
:10AA4000F149E87901270831002801D0132000E0FE
:10AA5000052020701422A01C0AF026F9A771EE71BF
:10AA6000AE710120F8BD70B5E8480078002802D02A
:10AA70000C26304670BD0026E34D3446203DAE74B2
:10AA8000EE746E75AE752E7528466E73203846735B
:10AA9000E87D002804D0FEF782FDFFF748F8EC754A
:10AAA000D9488471C47104772030FFF791F8D648F3
:10AAB0004830FFF78DF8DCE710B5D44C0023237045
:10AAC000D14C203CE375D04B01241C71603B5833C2
:10AAD00007C3FFF7C8FF002803D0CDA1FF200AF06D
:10AAE00080FA10BDC8482038807C7047F8B5C64D44
:10AAF0000646407B203DE873C34837791346AF7361
:10AB0000B27B42710446603C217006221946601CEB
:10AB10000AF0CAF8B07960730622F11DE01D0AF050
:10AB2000C3F8687B0126002800D0EE74B648403890
:10AB3000407B002800D02E753B000AF043FB050443
:10AB400006234706490000211DE0AF4801212030BF
:10AB5000FFF74EF8AC48E11D2030FFF77DF8607B31
:10AB6000002807D0012807D0FF20A9A142300AF011
:10AB700038FA0CE0002100E00121A3482030FFF763
:10AB800086F804E00621A0482030FFF731F80020C5
:10AB90006875A8759C48611C2030FFF74FF89A48EB
:10ABA00021782030FFF767F8974804214830FFF7F5
:10ABB0001FF89548611C4830FFF740F8924821780B
:10ABC0004830FFF758F8AE740020F8BD0221DAE7EC
:10ABD000FF208FA14C30CAE770B58B4C0125203C7B
:10ABE0000246A57588488079002801D03A2070BDBA
:10ABF000854860380378934206D1002262750622A8
:10AC0000401C0AF051F86575002070BD70B504460F
:10AC10007D4D0020203D28752846224632380AF016
:10AC200043F82846203844730120287570BD7649C2
:10AC30000871704710B5744C0022203CE2746073B8
:10AC40000246204612380AF02FF80120E07410BDA9
:10AC5000F8B500F044FB6C4C0025203CE07D00285A
:10AC600004D0FEF79CFCFEF762FFE575674E357079
:10AC7000FEF759FCA07B012804D00021084601F012
:10AC800077FAF8BD0021022001F072FA5E4CA0793B
:10AC90000127002807D0207F0028F2D10520607707
:10ACA000A5772777F8BD70780028FBD05649062293
:10ACB0006039487B6073C91D0846673009F0F4FFAE
:10ACC0003C202072A7717570F8BD10B54E4C203C29
:10ACD000E17B207CCA0701D0C2070BD08A070FD5C1
:10ACE00082070DD42620FEF7E8FA207C02210843D3
:10ACF000207410BD2520FEF7E0FA207C0121F6E744
:10AD00004907F6D54007F4D42720FEF7D6FA207C71
:10AD10000421ECE770B53D4D2878002873D13A4CFA
:10AD2000203CA07C00287DD0FEF7F2FB0026267494
:10AD300066746E703046FEF7E8FB0020FEF7D5F92A
:10AD40003748FEF7B1FA2546403D296E8857FEF791
:10AD500077FA3348C01EFEF7C1FBFEF709FCFFF788
:10AD6000B4FFFEF727FAFEF7CBFB0120FEF70BFB43
:10AD70000F210520FEF742FA2978681CFEF730FA09
:10AD8000A07B01280CD004280AD0E07C002807D042
:10AD9000214612390846627B5230FEF796FFE67470
:10ADA000207D002808D0184840380146427B1239DF
:10ADB0008830FEF7BCFF2675607D00280BD0124856
:10ADC000691C2030FEF73AFF0F48691C4830FEF737
:10ADD00035FF6675A675E86D0178002903D0017806
:10ADE000001DFEF70FFAA86D0178002907D0017841
:10ADF000054A401C7332FEF77AFE0120E075FEF72B
:10AE000092FB002070BD0DE03C1800207400002073
:10AE10007372635C6C6C5F6164762E63000000008B
:10AE2000075201000C20EDE7FE494860704770B5FD
:10AE30000546FEF79DFB002D06D00020FEF759FACF
:10AE4000FEF7B8F9FFF741FFF74C607C002809D006
:10AE5000A07B012803D1F549F5480AF0C2F8FFF7B5
:10AE6000F7FECFE7002D15D0A07B01280CD0FF20E6
:10AE70002D30FEF73BFA0220FEF785FAEA48203033
:10AE80000079012803D005E099208000F1E7022035
:10AE9000FEF736FCE4484030FEF74AFB012008F09C
:10AEA00082FDFEF78FF9A07B03000AF08BF9050401
:10AEB000040406040A00032000E00120FEF719FA4A
:10AEC00004E0DB48D9492A300AF08BF8E17B207C8A
:10AED00081430120002903D1A17B012903D06074A3
:10AEE000D04908708EE700212174F9E710B5FEF70C
:10AEF0000FFBCC48007800280ED1CB48807C00287E
:10AF00000AD00020FFF793FFF6F75BFAC64820301F
:10AF10000079012806D007E000F0E1F9FEF703FB15
:10AF20000C2010BDF8F774F8002010BDBD490120B9
:10AF30004870704770B500F0BEFF00281BD0B94EB6
:10AF40003078B94C2034012818D0022801D00328C9
:10AF500034D0B649B7480AF044F83078002809D010
:10AF6000F6F72FFA3078022804D12079012801D190
:10AF7000FEF7C6FB46E7FFF76BFE43E7AA4DA87B4B
:10AF800003281BD0FEF7E5FAE87D002803D0FEF782
:10AF9000BEFDFEF7FDFAA4489030FEF7C9FA012085
:10AFA00008F002FDA87B01280CD004280AD06179A2
:10AFB0006F20012908D0032906D006E00120FFF701
:10AFC00036FFCAE7012000E07F20FEF792F9022059
:10AFD0003070C2E710B59448C07D002803D0FEF75A
:10AFE000DEFAFEF7A4FD00F066FF002817D08D4CB6
:10AFF0002078022804D08F488C492B3009F0F1FFCB
:10B000000120FFF714FF2078002807D020780128BE
:10B0100004D088488549333009F0E3FF10BDFFF7BD
:10B0200017FE10BDF1B582B0FEF73AF90746FEF7FC
:10B0300099FD012829D000267A480078022804D0FA
:10B040007C487A49563009F0CCFF774DE87D0028DE
:10B0500003D0FEF7A4FAFEF76AFDFEF789FA7248FC
:10B060009030FEF7E7FD0446029800286DD0FEF709
:10B07000C1F8002869D020466B4C030020340AF048
:10B08000A1F806646464066425640126D4E7A87BFD
:10B0900001285AD0042858D0374304D160790028B9
:10B0A00001D0022851D160486830FEF741FA0120F2
:10B0B00008F079FC0120FEF71CF95A4803210170C1
:10B0C0002079012844D1FEF71BFB41E0564890301F
:10B0D000C178D038C27991421DD10146D0310A7968
:10B0E000037A9A4217D14A79437A9A4213D18A79DC
:10B0F000837A9A420FD1CA79C37A9A420BD10A7ADB
:10B10000037B9A4207D10978407B4906C90F8142E7
:10B1100001D1012100E00021A87B012801D00428F1
:10B1200001D1002908D100280FD1374304D160791B
:10B13000002801D0012808D13B489030FEF79BFE43
:10B14000002802D0A87D002812D00120FFF76FFE52
:10B150003448017800290AD00178012907D0007805
:10B16000032804D0324831492A3809F03AFFFEBD9D
:10B170002C4F2D49786804229F31343009F094FD1A
:10B1800029484021903000784006C20F78680A5460
:10B19000254906229331413009F086FD224978681D
:10B1A0000322A331383009F07FFD1F483B21903046
:10B1B000827D78680A541C4990310A7ECB7D120248
:10B1C0001A4382878A7E4B7E12021A43C2830A7F09
:10B1D000CB7E110219430184134990318A7F4B7F42
:10B1E00011021943418410490522AF31243009F07E
:10B1F0005BFD0D497F68B0310879C20638462030C2
:10B20000D20E0090827709794909C177A079002888
:10B2100019D0207F002856D1E07900280CD01320C7
:10B220000BE00000740000201C18002010AE00008D
:10B23000E703000093020000052060770020A0775C
:10B24000012020773FE0E97D2B48002924D0002110
:10B250002172B98961814021C95D61733946062235
:10B26000413109F021FDF88BA082388CE082788C86
:10B2700020830098C07FA076E07E400840003043E5
:10B28000E076FEF77CFCE17E4000C907C90F014370
:10B29000E1760120E07115E000212172B989618118
:10B2A0004021C95D617339460622413109F0FCFC39
:10B2B000F88BA082388CE082788C20830098C07F45
:10B2C000A0760120A0710D4C0020207000F007F83E
:10B2D000FEF729F90120616800F04AFF38E710B550
:10B2E000FEF751F9FEF744F9FEF791F80020FEF75A
:10B2F00000F8FEF7FFF810BD4A1800207400002087
:10B300008107C90E002808DA0007000F08388008F6
:10B31000FA4A80008018C06904E08008F84A80007A
:10B3200080180068C8400006800F704710B500F014
:10B3300079FF10BD70B5F34C0546A26800290DD009
:10B34000002A04D0FF20F0A1363009F04AFEA560A3
:10B35000F6F738F80220F6F72FF870BD002A04D16E
:10B36000FF20E9A13E3009F03CFE0020A060F6F786
:10B370002AF80120F6F728F870BDE2480C30C07EAC
:10B38000002801D00020704701207047DD480C30B4
:10B39000C07E7047DB483430C07E70470021C176E4
:10B3A000817601604162D7480C30C07E002807D109
:10B3B000D4483430C07E002802D1D2490120087020
:10B3C000704710B50B46C17E847EA14204D0114661
:10B3D000184607F0A4FB10BDFFF7E0FF10BD38B51D
:10B3E000C84C606801684978012924D00121684669
:10B3F00006F04EF968460078C749000209F0CEFC15
:10B4000060680268C0685268511807F0A5F9616861
:10B41000C860BC49606834310022884215D0018B75
:10B42000002912D04272032101720271021D017FB4
:10B43000FFF7C7FF38BD7D21C068C90007F08CF950
:10B440006168C860B5480861E3E7018B491C018366
:10B4500002214172E7E7FFB5AA4E01460C36706A39
:10B460003468056885B060680190306A03906A8826
:10B470000798801A80B202900898002804D02746C6
:10B4800038372046483002E0371D284664300090A7
:10B4900003203871002915D001297DD0022951D00F
:10B4A00003297AD0AF2098A1C00009F09AFD08982E
:10B4B0000028387972D0032803D093A1984809F066
:10B4C00090FD3BE1306A002804D195488EA1723886
:10B4D00009F087FD9249A88F9F3948434018069983
:10B4E00000F0A6FEA0618E49E88B9F39484306997B
:10B4F00000F09EFEE0618A4AA88F9F3A316A50436D
:10B500000918A069874A091A89183B22A162844B4D
:10B51000525D9F3B5A4382181018FF30163020624C
:10B520006062306A081AFF38ED213538C900884258
:10B53000BDD27D49884204D2794873A1653809F0AB
:10B5400050FDB7E0764AA88F9F3AE168504308184B
:10B55000069900F06DFEA0617149E88B9F39484360
:10B56000069900F065FEE061306A002804D16C485D
:10B5700065A15D3809F035FD5820405B6B4A002815
:10B58000A88FE16820D050430818A169401AA06232
:10B590002169A068484302E01FE04EE0C9E0A169CC
:10B5A000624A40183B21495D514341180818FF3059
:10B5B00014302062E88BE1695043411A0F2080016A
:10B5C000081A6062A06A35E050430818A169401A61
:10B5D0003168D33849684018D9E72846403001908F
:10B5E000008B002802D0306A002804D14C4846A1C4
:10B5F000453809F0F6FCE88B4C49E3694843C01A2A
:10B60000A06201999C460A8B2169A368521A4B4398
:10B61000A169591863465343C9183B22525D434BF5
:10B620005A438A185118FF31143121620F218901C0
:10B63000411A6162316A401A35E00898002803D047
:10B640003420005D002873D1E88B38494843E16914
:10B65000401A02994843A062284640300490008B6B
:10B660000028019829D0002804D02D4826A11F3891
:10B6700009F0B7FC04982D4A018B02980818E1697B
:10B6800048434000FF3014302062E88B5043411A99
:10B690000F208001081A606200F0C4FD00281CD051
:10B6A000A16A0398081AFF38ED212338C90088429F
:10B6B00000D3FCE602203871F9E6002802D0039896
:10B6C000002804D1164810A1263809F08AFC0198F8
:10B6D000A16AD3380818A062CCE706F0A6FD01469F
:10B6E000706907F0CBFFA16A081AFF38ED211E38F8
:10B6F000C9008842DDD2012009B0F0BD00ED00E0B4
:10B7000000E400E0D41800207372635C6C6C5F6C22
:10B710006D2E73302E63000010270000B7891300D0
:10B720008105000036040000A3020000E2040000CE
:10B730002AE0032802D1FD4907200870A16A706938
:10B7400007F00AF8B860616A206A884202D9009856
:10B75000016001E0009908600098F5490068081848
:10B76000F860A9880798081A00B2002801DD0220B5
:10B7700000E000207871089838700898002805D0FB
:10B780003420005D002801D00220B5E7089801218F
:10B79000484020346075317F3A463046FFF711FE4D
:10B7A0000020A9E710B5E14900284A68516A0968F4
:10B7B00007D01268C98BDF4BD2695943891A09F047
:10B7C000EDFA10BDF8B5D94F35227868416A0C689A
:10B7D0000168525C002A0AD0498E6288914206D1E3
:10B7E000407A002803D1D449D44809F0FAFB06F086
:10B7F0001CFD01467868406907F040FFFFF7D2FF63
:10B80000796865880B682E185A8EB24202DB521C8A
:10B810005A8602E0401C2818588608683622125CB6
:10B82000002A05D1428E23899A4201D1521C4286B8
:10B83000088B032802D2401C088302E00868408E6F
:10B84000A08020464030C18A808A081A6188401E44
:10B85000401885B2203416E0496AE67F09797600FF
:10B860004B00B749007DCB5A895BC91889B20023C8
:10B87000FFF7F1FD002811D0012810D0AF48AE49E4
:10B880003A3009F0AEFB79680868428EAB1A1BB2F9
:10B89000002BE1DA0820E07400F00DFEF8BD7868B6
:10B8A0000068418E491C4186EDE770B59F4D1F2011
:10B8B0002870A86800210162C27E130009F082FC92
:10B8C000045454034654426A1468026811700268B2
:10B8D000516000682030407D002808D106F0A5FCAA
:10B8E000A9680968096C07F0C9FE002815DCA8687A
:10B8F00001684A8E61888A4204D12289511A618185
:10B90000628004E0511A61810168498E6180026899
:10B91000C1681164C16841610FE0A8680168098EBF
:10B920006288891A61810168098E618001680A6CE8
:10B93000C2600A6C4261886C6066204601F06FFC50
:10B9400000280ED07B487C49D33808E0C1684161AB
:10B95000FFF7E0F9002804D076487749CD3809F0A0
:10B9600040FBF5F72EFD70BD72487349C638F6E707
:10B9700010B56E4A0B00526809F024FC0906090F45
:10B980001F0C2D2D082A2D00FFF78FFF10BD00F092
:10B990005DFC10BDFDF7B8FE10BDD07E022806D0BC
:10B9A000D07E032806D00120634940020DE0FFF756
:10B9B00009FF10BDFFF713FD10BDD07E0228F6D0A1
:10B9C000D07E0328F6D05C495E4809F00AFBF1E717
:10B9D00006F011FC10BD5B4857490F3009F001FB20
:10B9E00010BDF3B581B0514C0298254600260127C1
:10B9F0000C35030009F0E6FB0906313C3C314343BA
:10BA00003C3C4300494801210C30FFF793FC02996C
:10BA10000198FFF7ADFFE87E022828D1A0680468EE
:10BA2000406A066806F0E0FBF18B424A5143E26946
:10BA3000891AD339FF223232E162904202D242485F
:10BA4000081802E0081A41494018E0624048E16ADB
:10BA5000814200D80846E06206E001460198FFF7FF
:10BA600087FFE87E022802D1286820300775FEBDD6
:10BA7000014665600198FFF77BFF6660FEBDFF2011
:10BA80002D49AB3009F0ADFAFEBDF8B506462748A2
:10BA90000D4600243430254F0B0009F093FB0906B6
:10BAA0000C10100C1616101016002048012134300E
:10BAB000FFF740FC29463046FFF75AFFF8BD786093
:10BAC0003046FFF755FF7C60F8BDFF201A49DF3094
:10BAD00009F087FAF8BDF0B5144C0020616885B014
:10BAE00003268E76CA7E0746032A03D0C97E002924
:10BAF0003FD03FE0087F002804D112480E49CE30E5
:10BB000009F06FFA6068057F68460671022141718D
:10BB100006F08BFB0290FF20F53003900121684670
:10BB200001706946284606F0FAFF14E0D418002098
:10BB300019170000E204000008B7000062060000C8
:10BB40000C5201000B0200007CF8FFFFADF9FFFF73
:10BB50003812000020BF6068007F07F01BFE00283D
:10BB6000F8D06068007F06F046FB60680777FFF753
:10BB700015FC012061688F7605B0BEE5FE494A6874
:10BB8000907600E020BF4A68D07E002803D0D07EA7
:10BB9000937E9842F6D0D07E002803D0002000216A
:10BBA000917670470120FAE770B5F34900240C3113
:10BBB000CA7EF14D032A03D02831CA7E032A17D149
:10BBC0006960002810D001280AD0EC49EC4809F03F
:10BBD00008FA00206968002C0860686008D070BD11
:10BBE0000320FFF7CBFF01E0FFF775FF0446F0E706
:10BBF0000C2070BDF8B5E04F04461F25E67E3300EB
:10BC000009F0E0FA042A20031B20DB480C308442B0
:10BC100003D0DA49DB4809F0E4F902207C60FFF741
:10BC2000ADFF002805D07968002008604862786080
:10BC300012E00C25002078600BE00120FFF7B4FF34
:10BC4000054604E0CF48CD490C3009F0CAF9002D73
:10BC500002D0E07EB042D1D1E07E002804D0C948B5
:10BC6000C649123009F0BDF9F8BDC34810B50C3013
:10BC7000FFF7C0FFC0483430FFF7BCFFBE490020CB
:10BC80005C310875C0494870BB490C3148610A46AF
:10BC9000283250618876907601220C390A708860CB
:10BCA000486010BD70B504460120FFF729FBC5B2FE
:10BCB0000B20FFF725FBC0B2854204D0B148AF4945
:10BCC000343809F08EF90120FFF71AFBC5B21820AD
:10BCD000FFF716FBC0B2854204D08920A749800037
:10BCE00009F07FF90420C043FFF70AFBC5B2192011
:10BCF000FFF706FBC0B2854204D0A2489F49323804
:10BD000009F06FF9A0489C490C38047000200C31F0
:10BD1000C87688760A462832D07690769A4B0124E7
:10BD2000083B1C7118604862506208601060FFF7A1
:10BD30009CFF70BD9048007870479349083908719E
:10BD40007047F3B50D468C4983B00C31CA7E084666
:10BD50002830894C002A02D1C27E002A03D0C97E35
:10BD6000022903D005E08948616006E0C17E002910
:10BD700001D00C2000E76060854806F0E8F96168B2
:10BD80000877606880490160007F002804D17C4802
:10BD90007A49623809F025F906F026FA7D49884289
:10BDA00000D20846FF30C83086B260680321C176F1
:10BDB0000027012D2FD0734A03991A32514302688C
:10BDC0005160006801210170684605F061FC684619
:10BDD00000787149000208F0E1FF019106F025FAB0
:10BDE0000199711806F0B8FC6168032DC86021D074
:10BDF0006A4808616068032101720221417207717B
:10BE0000021D017FFFF7DDFA6068078307202070BD
:10BE100000206760B0E606F008FA314606F09CFCA8
:10BE20006168C8605E480861086807700968012099
:10BE30004870DFE75B48DCE77047F8B54E4E0C36DC
:10BE4000F17E002904D131462831C97E002901D074
:10BE50000C20F8BD0221F176474C4B4F5C34083F73
:10BE600077623460002538602575397920304A00C2
:10BE70004D49C07F8A5A4000085A2B46101881B29B
:10BE80002A462846FFF7E7FA002804D03C483B49F9
:10BE9000323009F0A6F825610120A560207565867D
:10BEA000258635487C30857539684888401E48802D
:10BEB00035830020F8BD10B52F4801248068817EAD
:10BEC00003290CD001684978002906D0006A374957
:10BED000884202D90024FFF729F8204610BD00242B
:10BEE000FBE72548806802681178491C1170016AD7
:10BEF0000068C26A914204D8007D012801D0012067
:10BF000070470020704700207047F8B51A481A4C57
:10BF10000C306060416A00260D68006834212F46AD
:10BF20000E544037B97C002966D1007D032863D1C7
:10BF300006F07BF901466068406907F09FFB002826
:10BF40005ADDFFF72FFC6988401C411860680268C1
:10BF500011860068018E2A89511A09B200294BDD29
:10BF6000012120308175F88AB98A401A6988401EFB
:10BF7000401887B239E00000D418002008B700004C
:10BF8000770300005702000088000020E3B900009A
:10BF90008BBA0000F605000010270000F713000020
:10BFA000B7891300E20900000C5201002C84130031
:10BFB000496A09794A00CE498B5A028E007D94461F
:10BFC0003F22525D5200895AC91889B20123624644
:10BFD000FFF741FA00280FD001280FD002280BD01C
:10BFE000C920C449C00008F0FCFF61680868028EDF
:10BFF000BA1A12B2002ADBDA6660F8BD606800681F
:10C00000018E491C0186F0E7F8B5BB4D0026AA68F1
:10C010000128516A0C6810D00720287006F050F8EB
:10C02000B6480078F6F7BCFDA86806830268618808
:10C030005186006820308675F8BD08791368410084
:10C04000AB481F7D415A032F17D01A7D022A21D0F9
:10C050001A7D012AE2D13F231B5D22895B00C05A71
:10C060000023401881B20120FFF7F5F90028D5D050
:10C07000A049A34808F0B5FFD0E71E6112683F232E
:10C0800096601B5D22895B00C05A0023401881B274
:10C090000320E9E75822125B1A613F231B5D2289C6
:10C0A0005B00C05A0023401881B20220FFF7D3F989
:10C0B000AA68012112681175D8E738B58E4C0021A5
:10C0C000A0680D4600684278002A01D045701FE044
:10C0D0000078002809D00121684605F0D9FA6846A1
:10C0E00000788849000208F059FEA0680268C0681C
:10C0F0005268511806F030FB0146A068C160057116
:10C1000002214172021D017FFFF75BF9A0680583E0
:10C1100005F0D6FF79480078F6F742FD38BD10B536
:10C120000146754A0B00906809F04CF8060D15049D
:10C1300008190C1C012100F0A8F807E00021506844
:10C1400000F0A3F810BD0120FFF75EFF00210846B4
:10C15000FFF7F0F810BD00680321017510BD00F075
:10C16000A7F810BD3D206349400108F03AFF10BD1B
:10C1700070B5614C002809D0012816D0022821D0C2
:10C180005F485C49C73008F02CFF70BDFFF795FF92
:10C1900000210846FFF7CEF8A068807E002801D075
:10C1A0001F2000E00720207070BDA06800250168F6
:10C1B0004D70FFF7F3F80320F6F737FC05F080FF2A
:10C1C000A56070BDFFF779FFA068FFF7E7F80021D1
:10C1D0000846FFF7AFF80420F6F727FC70BD464984
:10C1E0008968CA7E022A08D10A681378002B04D114
:10C1F00050600968CA6A1018C862704710B53E4A94
:10C20000002992680CD0012907D0022907D03C48A8
:10C210003849E73008F0E5FE10BD401E00E0401F41
:10C22000106210BD34488068002800D0012070479B
:10C2300010B504460020002907D0334808F0AEFDB1
:10C240000146204608F0AAFD401C10BD10B52A4842
:10C250008068C07E030008F0B5FF041414030A14BC
:10C2600001F0E5F800280BD02249284806E0FEF747
:10C270003DFE002804D025481E49001D08F0B1FEEF
:10C2800010BD22481B490B30F8E710B504460029C1
:10C2900003D00020FFF7B8FE03E018480078F6F757
:10C2A0007FFC2046FFF77AF80020F6F7BEFB10BDB2
:10C2B00010B511488268506A11680068CB698B60BC
:10C2C000124BC18BB13359431368D9600146E03139
:10C2D0004B8883870C783B231C548B88C383CB8883
:10C2E00003840989418411680220087510BD00008B
:10C2F0000C52010008B70000D41800207C00002078
:10C30000FD0600001027000040420F00310400002D
:10C31000F8B5FEF714FA0646FEF782FAF94D07461D
:10C320006879F94C002809D0012823D0022826D0AA
:10C3300003282ED0FF20F5A1C63033E0F248183094
:10C34000FEF75AFA002801D003200FE0EE4818301B
:10C35000FEF7BEF9002804D060696030007A00283A
:10C3600006D0E9481830FEF71AFA012068711BE080
:10C370000220FBE7E4481830FEF711FA14E0E24827
:10C380001830FEF7A5F900280ED1FF20DFA1B83044
:10C3900008E0DD481830FEF72FFA002804D1FF200E
:10C3A000DAA1C03008F01DFEA169F722087810401C
:10C3B0000870AA79D207120F1043FB2210400870B0
:10C3C000EA79D207520F104308706B79EF22022BE3
:10C3D00004D0012B07D0032B07D00CE0012E06D888
:10C3E000002F04D007E07F1E3E43002E03D01040F4
:10C3F0001022104300E010400870287C002811D063
:10C40000687901280ED0BF485438FDF791F8BD492E
:10C41000606954397830A269FDF7F5FA0020FDF71C
:10C4200001FB04E00846FDF783F8FDF71EFBA06959
:10C430000078C00606D4E0690078C00602D4E0792E
:10C44000002802D0A079002801D0012000E00320BC
:10C45000FCF74FFF0320207001202071F8BDAA488F
:10C4600010B51C30FEF7EFF9A74C002802D00020D1
:10C47000607004E001206070A2485438E061A14877
:10C48000407C002802D06078002805D0E069FDF7E4
:10C490004FF8FDF7EAFA10BD9A485438FDF748F80E
:10C4A000984A6069543AA030E169FDF7ACFA01207E
:10C4B000FDF7B8FA10BD10B5934900224869322340
:10C4C0008276C27601221A544030807C002803D044
:10C4D0000A700021022001E000210320FFF71FFE67
:10C4E00010BD70B5884C6079C20620464169084687
:10C4F0004030002A01DA002202E0028B4B89D21878
:10C500000B460283C0331A7E002A03D0828B4D89EA
:10C5100052198283627A002A03D03D2001F0BEF8CE
:10C5200052E08A7E032A4FD0227A002A13D0500785
:10C5300001D4D00601D51E2036E0100701D53D20DC
:10C5400032E0D00705D1900703D470A1734808F0FA
:10C5500048FD2A2028E060318A78002A05D0C28B65
:10C56000551CC5830D88AA420FD25A7F062A02D0D5
:10C570001A7F062A05D1428B531C438309888A42BD
:10C5800003D2828BC18A8A4201D322200CE0027C32
:10C59000808A002A0FD006280FD35A48C07B012872
:10C5A00001D03E2000E0082001F078F86069807E2C
:10C5B000032809D001E08842F5D201202070002133
:10C5C0000846FFF7ACFD70BDFFF775FF70BD10B5F5
:10C5D0004C494D48CA7B002A2BD0012A29D0022A77
:10C5E00027D0032A04D049A14D4808F0FAFC10BD19
:10C5F000897B02290FD007291BD0406901464031B1
:10C60000CA8A898A511A891E89B2032900D3032153
:10C61000028951180BE04069014640318A8A032A99
:10C6200001D2018903E04288C98A5118491C8180DE
:10C6300010BD4069F5E700B5030008F0C3FD06042E
:10C64000070B0F12121700290ED00FE0491E022906
:10C650000AD90BE0491F012906D907E0072903D0B1
:10C6600004E00A390C2901D8012000BD002000BDDA
:10C67000FEB5054624481830FEF79FF8002804D17F
:10C68000274822A1CF3808F0ACFC1F4CA069FDF769
:10C6900015FC0321A069FDF73FFCA069EF2201789A
:10C6A000114001702946FDF77BFC002601272B0075
:10C6B00008F088FD0E5D5D085D1D6161155D4D5DD5
:10C6C000613D385D60697121095C002901D0062156
:10C6D00001E0C030417EA069FDF72DFD4BE0E0692F
:10C6E000FDF788FC0146A069FDF796FD43E061690E
:10C6F000A069D031FDF759FD6169A0699531FDF759
:10C7000062FD38E0D0190020900000207372635C55
:10C710006C6C5F736C6176652E6300006B020000C9
:10C72000780800000621A069FDF772FD23E020696A
:10C730000178A069FDF756FD20698188A069FDF7A1
:10C7400053FD20694188A069FDF752FD13E0009672
:10C75000019660696030007C002803D06946087843
:10C76000384308706946A069FDF768FD03E0FE499B
:10C77000FE4808F036FCFEF72AF8002804D1FB48F2
:10C78000F949801D08F02DFC0C2D07D0072D04D091
:10C7900060695E210E5260308770FEBD6069403076
:10C7A0004683FEBDF0B5F24CDC2061698DB0405C83
:10C7B000042809D0052834D16031487A002829D0CE
:10C7C00001204874022026E01022EA31684600F079
:10C7D0009DFF61691022C83104A800F097FF6846E8
:10C7E00005F0AFF8616908AA6CCA0F46CB677837C5
:10C7F0008A670846FE608030BD60074620376CC7F8
:10C800000023036343630120A0310876D9494874AB
:10C81000052000E00D20FFF72BFF61690020C031EB
:10C8200008770DB0F0BDF8B5D1481830FDF7C5FF59
:10C83000002842D0CE4C207A00283ED160690025E5
:10C84000C030007ECB4E00280BD0B17B0120FFF71B
:10C85000F2FE002805D1B17B0420FFF7ECFE002892
:10C8600006D060690127C030407F062807D00CE061
:10C8700060695C210D526030457402202FE0B17B6D
:10C880000420FFF7D8FE002810D0B07B030008F08A
:10C8900099FC173F3F3F3F1E3F3F3F3D3F203F3FFB
:10C8A0003F292C3F3F3F3F3F3F2F3F0060696A21B8
:10C8B000095CC90702D0C0304577F8BD0C20FFF7EE
:10C8C000D7FE60696030817A39438172F8BD0720F4
:10C8D00005E0FDF7E2FF0028F8D075740B20FFF7A4
:10C8E000C7FEF8BD00F021FFF8BDFFF75BFFF8BD04
:10C8F0006069002180308160C16005743774062052
:10C90000FFF7B6FE606960308570F8BD0920E6E784
:10C9100000F0CDFEF8BD70B5964DA87B072834D148
:10C92000934CDE2260694188125A491C91422CD1F5
:10C93000217A002929D10146E0318B88C28B9342AC
:10C9400007D1CA88068CB24203D10A89468CB2420A
:10C950000DD0884A8689303A56819381CB88D3811D
:10C960000989118201462E31516001211170012285
:10C970001146FDF7B1FC00210420FFF7D0FB6169EF
:10C980000020C0314877A873E87370BD70B5794C4A
:10C99000A07B162803D07449774808F022FB74481E
:10C9A0000021426973486032117291703038067EFE
:10C9B0000B250123002E06D0027D002A12D14575D9
:10C9C000817503750EE0567A002E06D051722288CA
:10C9D000828381760C22027604E02288828381762B
:10C9E00083770576A17370BDF8B5614DA87980078E
:10C9F00023D5287A002820D15E4C0120A17BFFF7A7
:10CA00001AFE002819D1A8690127C0780026030062
:10CA100008F0D8FB0E626208622E3B4F0A62146275
:10CA200020524562022021E0A07B042804D0524815
:10CA30004D49333808F0D5FAA673F8BDA07B082815
:10CA400004D04D4848492D3808F0CBFA6869603069
:10CA50008670F1E7A07B0A2804D04748424926386F
:10CA600008F0BFFA6869603007720B20A073F8BD48
:10CA7000A07B0E2804D0AB203B49C00008F0B1FADF
:10CA80006869603007720F20F0E7A07B0F2804D0A0
:10CA900039483549183808F0A4FA1120E6E7A07B98
:10CAA0000F2804D034483049123808F09AFA13207D
:10CAB000DCE7FFF76BFFF8BD69690846C0310A7F04
:10CAC000062A04D16030807A800700D50E77487F2F
:10CAD0000628F0D14E77F8BD274823496E3008F07C
:10CAE00080FAF8BD10B5234C0020A17BFFF7A3FD11
:10CAF000002804D11E480122017A1143017204204A
:10CB0000A07310BD10B51A4C60690146C0314A7F50
:10CB1000002A06D0097F062903D0217A0122114379
:10CB200021726030807A800715D4E069FDF764FBDC
:10CB300061696031C872E069FDF760FB616960316D
:10CB40008881E069FDF75FFB616902226031C8817D
:10CB5000887A10438872606900220146C0310B7FD9
:10CB6000062B00D10A7709E00CC70000ED07000092
:10CB700090000020D0190020770500006A231B5C7C
:10CB8000DB0703D106234B774030428310BDF8B555
:10CB9000FE48817B0020FFF74EFDFD4C012600285A
:10CBA00007D160696030407A002802D1207A304392
:10CBB0002072616900255E20455262204654C831CA
:10CBC000E069FDF7DAFA6169E0699131FDF7E4FAAD
:10CBD0006169042208469131B93008F065F8EB48E4
:10CBE0003038017E0827002906D0017D002912D1A6
:10CBF0004775857506750EE061690546898941832B
:10CC0000E249E0691439FDF7A0FAE049E0690C391E
:10CC1000FDF7A8FA2F76DD480E218173F8BD70B5B7
:10CC2000DA4D0020A97BFFF706FDD94C002803D17F
:10CC3000207A012108432072E069FDF742FA0028BA
:10CC40000ED0E069FDF738FA6169DE22505249885A
:10CC500000F0B6FD002806D0282000F01FFD70BDB2
:10CC6000FFF740FF70BDE069FDF720FA6169E03130
:10CC70000870E069FDF713FA6169E0314880E06906
:10CC8000FDF7F2F96169E0318880E069FDF7F5F9B7
:10CC90006169E031C880E069FDF7F8F96169E03168
:10CCA00008810720A87370BDF8B5B94CA079C007FA
:10CCB0006FD0207A00286CD1B44D0120A97BFFF7FA
:10CCC000BAFC002853D1E0690027C178022201266E
:10CCD0000B0008F077FA0D161308354A4A384C470E
:10CCE0004A1929444A00FDF728FA6169DA225054AA
:10CCF000AE735E20475260318E7038E000F06BFDFD
:10CD000035E0FFF78CFF32E0A97B0020FFF793FCB2
:10CD1000002802D1207A3043207260695E210F52D0
:10CD2000603086700A2018E0A87B0B2802D0207A99
:10CD3000104320722F746069603046720C200CE042
:10CD4000FFF725FF13E0A87B112802D0207A1043BB
:10CD500020726069603087701620A87307E0FFF7C3
:10CD6000D1FE04E000F004FD01E0FFF7BBFEFDF79B
:10CD700080FD002804D14F208649000108F031F9D8
:10CD8000606900238030016B426B491C5A41426349
:10CD90000163F8BDF8B57D4F012814D1787C0028D7
:10CDA00002D1387C002801D0FCF75FFEFCF7EBFBDA
:10CDB000FCF7DEFB0020FCF79CFAFCF728FBFCF7F5
:10CDC00099FBFCF7B0FBF87B01260025704C00288E
:10CDD0000FD16079C10705D00220F8736069403037
:10CDE000057402E0800717D5FE7300210120FFF7CC
:10CDF00096F9F87B012802D0022808D00CE060796F
:10CE0000C00709D00220F87360694030057460796A
:10CE1000000701D50320F87300F00EFDFFF703FDB6
:10CE20002079002801D03D8102E03889401C3881FA
:10CE30006079C007606904D072210D54403085824A
:10CE400003E04030818A491C8182E079002806D0C5
:10CE500061696031887C022806D8401C887460694A
:10CE60006030807C022804D93D817D81606960301A
:10CE70008574B97B0020FFF7DEFB002802D1B87B68
:10CE800006284BD160690146C0310A7F062A45D089
:10CE9000497F062942D03D49C97B03293ED16030F4
:10CEA000807C00283AD1FDF741FC002836D0FDF700
:10CEB000B7FC002832D06169C88801282ED90A46FB
:10CEC00040325674D08A978A831E9F4201DB01202C
:10CED00002E0C01B401E80B22C4B1F89A3899F42D9
:10CEE00001D3012302E0DB1B5B1C9BB2984200D9FB
:10CEF0001846012800D155742A22525C002A11D00C
:10CF0000224A898D52898A4201D3012102E0891A7D
:10CF1000491C89B2884205D9084603E061690120AD
:10CF200040314D7461694A8810180881FFF74FFB42
:10CF30006069122215490C3007F0B6FEFFF7D1FAEE
:10CF4000FEF7E1FF00280AD0104810388179002947
:10CF500005D1616902468989203A118586710C489C
:10CF60001C30FDF7CEFC00280FD0E0690078800768
:10CF7000800F012809D0022807D0FDF7E2FC002825
:10CF800003D10449044808F02CF807E0D019002028
:10CF9000900000200CC700007F0300006069403053
:10CFA0008574F8BD70B5FE4C607900283CD0FD4D0D
:10CFB000022810D1FDF79BFB002803D1FA49FB485A
:10CFC00008F00FF86A69002380329068D168401C2D
:10CFD0005941D1609060002666712079012804D102
:10CFE0002671A87910210843A871E078012816D18C
:10CFF000E670A87908210843A871FDF707FC00280E
:10D0000004D1EA48E849183007F0EBFF69690023CA
:10D0100080318A68C868521C58418A60C860A0790B
:10D02000012802D00120A07170BDA67170BDF8B5B5
:10D03000DC4CDB4DE26900271078042183079B0F4D
:10D04000E8790126012B11D0022B0FD0032B01D040
:10D05000207A30E06178002905D1AE70A1793143A2
:10D06000A17123E0EF71F8BDEE71F8BD5278D306DF
:10D070001CD060780028F8D1D006C00E1B2818D824
:10D08000607908436071FDF7F4FB002804D1C748BC
:10D09000C5494B3007F0A5FF606900238030026B63
:10D0A000416B521C594102634163E8790128DBD18D
:10D0B000D8E7207A102108432072F8BDF8B5B84DA2
:10D0C0000446303D287D002700280AD0002978D169
:10D0D000677010202070687DA070A87DE0702F75AB
:10D0E0006FE02878002814D000296AD107206770E3
:10D0F0002E462070083607E0686807802F700A22E5
:10D100003146A01C07F0D0FD28780028F4D1A77084
:10D1100057E0287EA24E143E002837D0002950D177
:10D12000297EA0480B0008F04DF80D2C2C2C2C2C3F
:10D130002C2C2C112C2C20082C0067700C21217019
:10D14000A97EA17040698089A08018E008216770DD
:10D15000217040690A468089914960801439201DF8
:10D1600007F0A2FD3089A08109E067700B212170D2
:10D17000A97EA17040698089A080A87FA0712F76C8
:10D180001FE089498A4807F02CFF1AE084481038CC
:10D190008279002A08D0002913D1677011212170EB
:10D1A000B189618087710CE0827A002A0BD0002956
:10D1B00007D1677012212170318A6180718AA18044
:10D1C00087720120F8BD0020F8BD7648007801285C
:10D1D00001D00C2070477249002030390870087562
:10D1E000087620318871704770B56E4C06462078FD
:10D1F0000D46002804D093206B49000107F0F1FE92
:10D2000001202661E07225622070FFF7DEFF002812
:10D2100004D067486449493007F0E3FE70BDF8B5B3
:10D22000604C2178012902D12178012901D00C20FC
:10D23000F8BD01460546606112220C31584807F0DE
:10D2400033FD01274035AF74554D2888FDF735FA79
:10D25000002827D02888FDF7EBFA002822D028885C
:10D26000FDF7A0FA00281DD02888FDF7BAFA00289B
:10D2700018D0FCF74DF960690026C088002825D039
:10D2800048481830FDF799FA00281FD06069C0306F
:10D29000007E00281AD0A97B0120FFF7CCF90028D6
:10D2A00002D013E01220F8BDA97B0420FFF7C3F9D8
:10D2B00000280BD1606901464030868360314E748E
:10D2C0000220FFF7D5F960694030467434483038A1
:10D2D0000078002804D16169C88D098C884201D882
:10D2E0006069008CA08160694189491E8AB22989E0
:10D2F00089182981297B002902D06E812E7302E0D2
:10D30000698989186981014640318B8A9B188B8213
:10D31000C388012B01D85B1CC380002A01D0603078
:10D320008674A87B032816D0487C002815D028894D
:10D33000A189884211D2FDF7F9F900280DD0606962
:10D340002A21095C002908D06989808D814204D393
:10D35000A670E77003E0A77001E0A670E670606950
:10D3600051210E54A97B052901D0062915D1DE21B2
:10D370004288095A511A09B200290EDB01460522DA
:10D38000E0312430F3F720FF012202216069FCF72D
:10D39000A3FF6069C0304677AE736069418909E0D8
:10D3A000D0190020900000200CC7000039070000B1
:10D3B000F1080000FDF745F8A07800282AD160693F
:10D3C0002030807A002800D06E810120FBF78DFE8E
:10D3D00060693830FCF782F860693430FBF764FF2D
:10D3E000216A00200856FBF72BFF0120FCF78DF87F
:10D3F000FBF7E4FEFCF784F80120FBF7C4FF60694B
:10D40000406EFCF798F8FFF72AF860694030C07B5F
:10D41000FBF753FF6671E671A6712672A6726672FB
:10D42000267102202070FCF77EF80020F8BD10B5B0
:10D43000F74C2078022801D00C2010BDA0780028DD
:10D4400003D00020FFF7A6FC17E0FCF761F800F01E
:10D450001DF960692030007C012809D0FCF7B5F87F
:10D46000FBF7B1FEF3F7ADFFE07A012803D004E04B
:10D47000FCF7B3F8F4E7F5F7CBFD002010BDE44965
:10D48000C872704710B5E24C2078032803D0E149F8
:10D49000E14807F0A6FDE14801218278002A06D084
:10D4A000002282700171A27904231A43A271A26939
:10D4B0001378DB439B0707D1C378002B04D1C170DD
:10D4C000A07902210843A0711078C00606D4E06953
:10D4D0000078C00602D4E07900280CD060780028DB
:10D4E00009D1A079002806D1FEF7FBFC002802D064
:10D4F000207A002803D00120FFF74CFC03E0FEF760
:10D50000AEFF00F0C3F82078012806D0F3F759FFEA
:10D51000E07A012801D1FCF7F3F810BD38B5BC4C16
:10D5200060692030007C012820D1A07A00281DD11C
:10D530006846FCF75AF8002818D061693120405C31
:10D54000012810D1B54A0D236D460020D356285628
:10D55000834208D050738989303A91851146203131
:10D56000887301208872A07A401CA07238BD70B503
:10D57000A74C06462078042804D0A748A549553072
:10D5800007F02FFD607910210843A44D6071002E33
:10D5900047D0FCF782FA61780126084300280ED1B3
:10D5A000687C00280BD0E0694178C90607D0007874
:10D5B000E9790007C00F884201D1667247E0E07840
:10D5C000002809D0E0694178C90605D10078C00675
:10D5D00002D4FFF7A3FF3AE0FFF7A0FFE069A979C3
:10D5E00000784007C00F884205D0FFF7DBFC607968
:10D5F000082108436071E069E97900780007C00FED
:10D60000884201D1FFF713FD60793043607100203B
:10D61000E071A079000702D5A87B022817D0207AF4
:10D6200013E0022108436071E079401CC0B2E07150
:10D6300001280CD8687C00280DD0784854384078F0
:10D64000C106C90E052906D2C006002803D0012054
:10D65000FFF7A0FB01E0FEF75BFE2078012806D073
:10D66000F3F7AFFEE07A012801D1FCF749F870BD6D
:10D6700010B567480078042804D067486549B7307A
:10D6800007F0AFFC0120FFF785FB10BD10B50720A8
:10D69000FBF72FFE5E490420087010BD5C49332261
:10D6A000496950545D4A032090738876704710B5DD
:10D6B000574C6069C030007F00281CD0062806D077
:10D6C0005648817B0020FEF7B6FF002813D0606922
:10D6D0000146C0310A7F130007F074FD070D0D0DE0
:10D6E0000D0D0D050D006030807AC20704D0C043D7
:10D6F000800700D1087710BD0C20FEF7B9FF6069E4
:10D7000001226030817A1143817210BD10B5002A68
:10D710000AD0002306E0D41A6418203CE47FC454E5
:10D720005B1CDBB29342F6D310BD10B503F0AFFF24
:10D730000C281CD3364C08216069D03003F0A8FFB8
:10D74000002806D060690421953003F0A1FF00286D
:10D7500003D13049324807F044FC6169042208468D
:10D760009531BD3007F0A0FA0420FEF781FF10BD0F
:10D770007CB52A4E0020B17BFEF75DFF0125244CCD
:10D78000002802D1207A284320726946E069FCF71C
:10D790005BFD684600780021C207D20F6846027020
:10D7A0006069002A02D06030057401E060300174C5
:10D7B00060695E221152603085700820B0737CBDB4
:10D7C000401A184900B2884201DC002801DC01201F
:10D7D00070470020704770B5104D0020A97BFEF700
:10D7E0002AFF0B4C002803D1207A01210843207224
:10D7F000E069FCF79BFC6169DE2250524988FFF723
:10D80000DFFF002810D02820FFF748FF70BD000080
:10D81000900000200CC70000320A0000D019002040
:10D8200062060000FE7F00006169E069E031FCF7FC
:10D8300071FC0520A873E9E770B500F047F8384C93
:10D84000384D6079400709D5A97B0520FEF7F3FE26
:10D85000002803D0207A082108432072FFF724FA19
:10D8600000F012F8FFF7C0F8A079C00609D5A87B30
:10D87000030007F0A7FC06060606060604060620B7
:10D88000A873FFF748F8C1E710B525488179490723
:10D8900014D5017A002911D12249897B0B0007F0A8
:10D8A00091FC080D050D0D0D0E0D100D40690022A7
:10D8B00062210A54C030807EFFF7F0FE10BD0121C6
:10D8C00000E002214069C030417710BD10B5144816
:10D8D000817909071DD5017A00291AD1114A947B53
:10D8E000230007F06FFC1416160B161616161616E4
:10D8F00016161616161616161616171640696030E6
:10D900008170407C002801D0062000E01620FFF73F
:10D91000C5FE10BD4069603001728170917310BD09
:10D9200090000020D019002010B5031D03600020D6
:10D93000521E04E05C181C60401C2346C0B290429A
:10D94000F8DB0020186010BD01460A680020002A9C
:10D9500002D0104612680A60704702680A600160CF
:10D960007047000000B51A2822D00ADC030007F037
:10D9700029FC0D111F131F1F191915171F1F1F1B1E
:10D980001F002A2814DD3A38030007F01BFC030FA0
:10D9900011091100002000BD1E4800BD042000BD7B
:10D9A0000D2000BD0F2000BD082000BD112000BDCE
:10D9B000032000BD10B50C46F4F79FFF00281AD0D5
:10D9C0002046F4F782F9002812D020780E280BD0D8
:10D9D0000F2809D0022807D0032805D00EA17720F0
:10D9E00007F0FFFA002010BDA078FFF7BBFF10BDC5
:10D9F00009A17D20F4E708A18320F1E710B5F4F731
:10DA0000EBF810BD10B5F4F760F910BD10B5F4F7E0
:10DA100042F910BD023000007372635C686F73746A
:10DA20005F6863692E630000F0B597B000210320A2
:10DA300004F080F90025FE4E022775807574347C51
:10DA400012E0F068E1004018818800290CD0858040
:10DA500069460F704D700168029180886946888020
:10DA600000216846F8F71AFD2046641EE4B200283B
:10DA7000E7D117B0F0BDEE4BD86019741A80D3E728
:10DA8000EB49EC4B4A8800201A4200D00120497C27
:10DA9000002901D0082108437047F7B504460E4617
:10DAA00000780121E34A8140521C114098B0E04ABD
:10DAB00000915188E04B994205D0009B002B05D086
:10DAC000DC4B194202D001201BB0F0BD009BD84AAC
:10DAD000194351801A9D002D11D000202870227802
:10DAE0001A980027401C130007F06CFB10EF0D156F
:10DAF0002137555D6A39AFAB85B3EEEDECEF0B28FE
:10DB0000EDD00420E0E702212970A1880170090A04
:10DB10004170032093E004212970A1880170090A53
:10DB20004170E1888170090AC170052087E00621F3
:10DB30002970A1880170090A4170E1888170090A81
:10DB4000C17021890171090A4171A289E81D216909
:10DB500007F0AAF8A089C01D71E00821297021787A
:10DB6000082901D110212970A1880170090A41708A
:10DB7000E1888170090AC1700520308020466A1D45
:10DB800001A9083003F0CDFB00287DD1694630881B
:10DB90000979401853E00A212970A1880170090A07
:10DBA000417003200AE00C212970A1880170090A44
:10DBB0004170E1888170090AC170052030809DE0C4
:10DBC000A08884464000401C81B2308888425BD3E4
:10DBD000052959D30E202870002008E0A3684200D0
:10DBE0009B5A521953701B0A401C937080B26045B7
:10DBF000F4D33180B6E08E49487C002873D0401EB3
:10DC00004874C86821790822C9004518A98828687D
:10DC100040180838A16807F047F8022168460171EA
:10DC20000021417128680390A9886846018100217C
:10DC300001A8F8F733FC0020A880002E00D0308027
:10DC400090E02978802211432970297840221143DD
:10DC5000297029788909890112312970A1880170F8
:10DC6000090A4170E288E81CA16807F01DF8E08805
:10DC7000C01C30802878410640D5C00972D00121EF
:10DC800068460171002100E02BE041713188ED1CF4
:10DC9000091D01811A980390E08840190490001D25
:10DCA000634D0590297C68460176002101A8F8F7AC
:10DCB000F5FB074630880C303080022F06D0002F4D
:10DCC00050D060E03CE032E01CE059E06946097E5B
:10DCD000E868CA0080182A7C914202D28188002913
:10DCE00002D004274FE02EE0697C491C69741A9920
:10DCF0000160318881800020308044E04C48A18858
:10DD0000C1802FE029788909890116312970A188FD
:10DD10000170090A4170E1888170090AC170228985
:10DD2000681DE16806F0C0FF2089401D46E728789D
:10DD300080098001183028702079687002207EE701
:10DD40003B480A0401D405271DE00289A3889A42B2
:10DD500001D0062717E01E222A70012249043280D2
:10DD6000490C4180009800280DD0314D00222888B0
:10DD700011468300032003F038FF2078287107E064
:10DD80000020308003272A48009942888A43428035
:10DD9000384699E6F7B59AB002000C4606D0172A25
:10DDA00004D82348244B4088984202D107201DB054
:10DDB000F0BD23785D0601D4DB0901D00820F6E729
:10DDC00000236D462B706B701D462378611C9F06E7
:10DDD000931E1893531E19939BB2169302AB17937D
:10DDE000134BBF0EDE883B0007F0ECF9208511F1E4
:10DDF0005EF16BF1A3F1C6F1F2F1FBF1EEF1EDF1A1
:10DE0000ECF1F1F1EBF1EAF1E9F1E8F185F1052A44
:10DE100071D1042269460A7005490A7969460A7176
:10DE2000E178A3780A021A436946CA80227905E09C
:10DE3000E4190020FE710000FFFF00004A706178C5
:10DE40008906890E0C2923D009DC891E0B0007F0F6
:10DE5000B9F9091352155219521B521D52001229B9
:10DE60001CD004DC0E2915D01029D1D114E01629BC
:10DE700016D01829CCD115E0800700E04007002813
:10DE800039DA2AE10007FAE7C006F8E78006F6E784
:10DE90004006F4E70006F2E7C005F0E7C004EEE74D
:10DEA0008004ECE74004EAE7800724D5032AAFD1D9
:10DEB00005206A461070487809780002084390806F
:10DEC0000BE14007F1D5062A15D31898617880B286
:10DED000012902D002299BD101E0022700E010278E
:10DEE000062269460A7000228A8001AEA11C023611
:10DEF000BA1C179218E0B6E04A780B7812021A435F
:10DF00003280801E891C1890B21C1691384603F08E
:10DF1000E2F9169918986B469A88C919C01BB61D64
:10DF2000521C9A80179A80B28242E5D900289CD16F
:10DF3000D3E00007B9D51998694682B20720087066
:10DF400000208880601C891D11E0437806781B0240
:10DF500033430B80C37886781B0233434B806E4675
:10DF6000121FB388001D091D5B1C92B2B380042AE6
:10DF7000EBD2002A77D1B0E0C00674D5022A72D362
:10DF80001898082182B2684601700021C180637828
:10DF90000371A01C17990EE04678077836023E43BD
:10DFA0000E80861C4E606F46D21AFE88C01808315B
:10DFB000761C92B2FE809342EED9DAE76FE076E00B
:10DFC00065E051E046E01EE014E00AE000E0A0E079
:10DFD000800648D509206A46107096801698D08031
:10DFE0000FE040063FD50A22684602708680169AE6
:10DFF000C28006E0000636D50B206A4610701698DF
:10E000009080029169E0C0052DD5022A7FD318982F
:10E010000C2182B2684601700021C18063780371CF
:10E02000A01C179913E04678077836023E430E800D
:10E03000C678877836023E434E80061D4E606F4696
:10E04000D21AFE88C0180831761C92B2FE80934224
:10E05000E9D98EE7C0045AD5012A58D10D21684666
:10E060000170868039E052E0800450D5052A4ED3F5
:10E070000E23684603708680C8788B7801021943A6
:10E080006846C180521F0281601D039025E0400454
:10E090003DD5012A3BD10F20694608701DE00304DD
:10E0A00035D44B780E781B023343244E3381032A38
:10E0B0002DD31B2F27D011236E46337001261F4B03
:10E0C000F6033043588048780B78010219436846BC
:10E0D0008180D21EC280E01C029020788006800ED3
:10E0E0001B280AD01D2808D00021032003F022FE9F
:10E0F00012484188C90BC903418068461C99F8F74A
:10E10000CDF9284653E610206B461870DBE707254B
:10E11000F7E70825F5E700B50022D243074997B095
:10E120004A80032807D103226846027009790171E9
:10E130000021F8F7B3F917B000BD0000E419002082
:10E14000FFB589B00020019009981027FE4C1E46AB
:10E150001546082806D0E06901F05EF8002809D0CD
:10E160003770BEE0288809213843108013980227B1
:10E17000017016E0E169012088710521E269C90298
:10E180009180E1698872E169F0480881E1690020C5
:10E190008873288820210843288011211398042798
:10E1A000017013980225801C0290307806900A2096
:10E1B0003070E5481830049001F022FA00200590F4
:10E1C00020462C3003906DE00998102808D1022DCC
:10E1D00006D001990298A28D401A8270110AC1706E
:10E1E000E08D0A99884202D901F0CDF806E0884214
:10E1F00004D10698002801D030701CE00298E18D0F
:10E200000170090A417012980088401BC01B82B23D
:10E21000FF20C01B904200D2024607A8009002983F
:10E220000021C319E08D01F056FA3070002805D0A6
:10E23000C0B2832858D0E08D20833EE005980028A6
:10E2400004D0206C00790A282CD336E06846808BF5
:10E25000C119C9B20191022D0DD01399019A4978C3
:10E26000914202D1228F824208D00191206C017824
:10E27000032908D023E0084613994870206C0178E0
:10E28000042906D007E000790A2818D20120059059
:10E2900008E0E18D818002990198081802900198A8
:10E2A000281885B20399049801F0ADF9002804D12B
:10E2B00012980088401BB84286DA022D0DD00998CA
:10E2C000102806D102990198A28D081A8270110AAD
:10E2D000C1701298058000203070206C00780328EF
:10E2E00002D000200DB0F0BD0220FBE7F8B5964A41
:10E2F0000026126D002A2ED0401F934D84B2403567
:10E30000E88A23460833AF8AC318BB4222D88B78E9
:10E310004F781B0210183B4303701B0A43700B79A4
:10E32000CF781A023A438270120AC2700471220A2C
:10E3300042712246491D801D06F0B6FCE88AA41DE4
:10E34000001980B28049E882096D00220818027025
:10E35000427000E009263046F8BD30B57A4B02889D
:10E3600040339B8A934213D9774B1C6DA3185C787A
:10E370001D7824022C430BD05C791D7924022C4398
:10E380006404640CA41D1219028000200B6030BDCF
:10E39000822030BDF0B585B007460026684606816C
:10E3A00055E00198417802780D02154341790279D0
:10E3B0000802104300044AD43D8003A80023012230
:10E3C000009052021946284601F085F9040044D114
:10E3D0006846018901820198417902790902114355
:10E3E000437802781C021443AC421CD10A041AD4AC
:10E3F0004A040121520C89030A430096C1788078AF
:10E40000090201430023204600F0C1FF040010D19F
:10E41000019948790A79000210430122D20310437E
:10E420000871000A487101A904A8FFF796FF0400CB
:10E43000D1D00199009648780978000208436946CE
:10E4400000238A89194600F0A2FF822C05D101A978
:10E4500002A8FFF782FF0400A3D06846068109E006
:10E46000019948790A79000210434004400C087170
:10E47000000A487101A902A8FFF76FFF0028EFD03A
:10E48000822C02D0204605B0F0BD0020FBE7F7B596
:10E4900084B014460646002700F071FF2A48002584
:10E4A000006D00282FD0059801282CD12046FFF7B9
:10E4B00071FF070027D1002E29D06846058118E09A
:10E4C000019948780978000208432080019B009553
:10E4D000587919790202D8780A4301029F7858784E
:10E4E00039431F7800029B1D384300F050FF00287D
:10E4F00005D101A902A8FFF730FF0028E0D082284B
:10E5000000D100200746002E01D00F48056500F01D
:10E510003AFF384607B0F0BDF0B597B000210420AF
:10E5200003F008FC084F00243D467C8040356C73A6
:10E53000AC73287BB96CC00008380E18B08800286E
:10E540000DD00120694603E0F819002001280000E1
:10E5500008703068019000216846F9F7A0FAB4808D
:10E560003C65AC82EC8217B0F0BDFE4B9864184657
:10E57000403001731A803838D861CDE7F94900205E
:10E5800049880A0700D501200A06120F01D002228D
:10E590001043CA0501D5042210438A0501D5102273
:10E5A0001043490501D520210843EE494031497BFC
:10E5B000002901D0082108437047FFB5A7B0040027
:10E5C000289816461B9022D00178E6484D064288CE
:10E5D0002292024640320092002D14DB8A06920EEF
:10E5E0001E2A0ED0229A5205520E10D13288172AB6
:10E5F0000DD3009A927B002A09D1DB4D229AAA42C0
:10E6000005D0CA0906D08A06920E122A02D003202B
:10E610002BB0F0BDD348826C0098007B2590C000E1
:10E62000083810181F9048060CD40098407B00282A
:10E6300008D0009988731F99289808601F988480D3
:10E640000220E5E7002718A90F7069460F72C54937
:10E6500002AA0A64309A4A6410A90F850F861B9893
:10E660001D46007820908106BE4B601F24901A46FC
:10E670002C3221922898DA691833890E1E93401C97
:10E680000B0006F09FFD1FFDFD11FD1AFD90FDFC26
:10E69000FDFBFDFAFDF9FDFCFDF8FDFDFDF7FDF6C6
:10E6A000FDFDFDFDFDF5FD00032C7BD10320287051
:10E6B00017226A700022AA70E0E2052CF5D1417899
:10E6C000027809021143A74B10AA19831185C27859
:10E6D0008078120202435A8300297DD091427BD870
:10E6E0000021184681720181491E01841E9800F0A4
:10E6F00087FF05202870A81C1D90022000902199FA
:10E700001E9800F080FF002803D047E018A9087089
:10E71000F0E294482030807C012803D00220687009
:10E72000102002E001206870022022908D483030D5
:10E730002390002220A9239802F0F3FD00282AD17B
:10E7400020A800782299814225D132880099801C26
:10E75000511A81421FDB83481D99C08D0870000A41
:10E7600048701D9820A9801C1D9000981D9A801C3F
:10E770000090239802F0D5FD20A909781D98401833
:10E780001D900098401880B2009021991E9800F0CA
:10E790003AFF0028CDD0009802288DD10A2018A970
:10E7A00008706CE26DE0072C6BD3417803780902A6
:10E7B00019436C4B8446198310AB1985C378807854
:10E7C0001B021843674B0029588305D0814203D8A8
:10E7D00001211846817200E0A4E061464B79097975
:10E7E0001B020B43038100218173104600F014FDCE
:10E7F00000280FD15B480121C26991710522C369CC
:10E80000D2029A80C2699172C26958491181C06965
:10E81000002181735349E01F08841B98C01D486282
:10E820001E9800F0EDFE07202870681C0090012063
:10E830001D904C480021C18530E01D98012815D05D
:10E840004848C169897901292FD000981038C17BC7
:10E85000807B0902014300980170090A4170009809
:10E86000801C00901D98801C80B21D903D4809E0DE
:10E8700013E2BEE17AE1D8E00DE2A0E080E03BE007
:10E880001EE2B6E0C18D00980170090A417000983F
:10E89000801C00901D98801C80B21D9021991E98AC
:10E8A00000F0B1FE002802D006E0818DD3E7318868
:10E8B0001D98081A0428C0DA1D98012800D16DE7B8
:10E8C0002848C1698979012903D0828D26498A4265
:10E8D00005D1818D00980170090A417009E0009806
:10E8E0001038C17B827B0802009910430870000A2F
:10E8F00048701D98801CC1E1072C01D0152C78D1DF
:10E900004178037809021943164B198310AB198516
:10E91000C37880781B02034312480029438301D047
:10E92000994201D90120F1E60E48012181720021AE
:10E9300001818173052C07D024981B99C0B2491D11
:10E9400002F0C9FC0028BAD100200649C04308845F
:10E950001B9800960195007818AB8006800E1CAAC3
:10E96000002105E0F8190020FFFF00000128000049
:10E97000FFF7E6FB0746FE4810A9008B08857EE1FD
:10E98000032CBCD1402210A90A86417802780802E3
:10E99000F7491043088310A9088520A90091318800
:10E9A0006B1C491E8AB2002100F095FE18A9087060
:10E9B000002830D10B20287020A8008833E0052CD7
:10E9C0009DD1802110AB1986014640780B78020258
:10E9D000E7481A430283CB7889781B021943E44B3A
:10E9E0001046198410AB1A85E24A914202D30720DF
:10E9F0008CE697E03F23DE4A9B021943118421AA4B
:10EA0000009232886B1C521E92B200F064FE18A96C
:10EA10000870002803D08328B1D102272FE10D20F0
:10EA2000287020A88088401C28E120990C22C90960
:10EA30005143C91C1E91A14204D92098400671D5AA
:10EA400000201BE1417800780902014310A80185EC
:10EA50001B98007842062898C01C1D90002A62DA94
:10EA600005206A4610721B980078C00944D008221D
:10EA7000684602728181A01A87B268468782289808
:10EA800006901E98201A81B26846C1811D98049094
:10EA9000401806F06AF9079006982599C019089061
:10EAA000491E08A8017102A83099F8F7F8FF074637
:10EAB000002168460172002F1BD0022F18D1009848
:10EAC00008A9007B0979401E884210DDA848289AD1
:10EAD000836CC9005A50816C08A80079C000001DE1
:10EAE0000C5200980099407B401C4873C7E00527F2
:10EAF000EAE0062069460872002000901E98002176
:10EB0000201A209082B21B9B10A8DB1C008D00F005
:10EB10003EFC014618A80170002268460272832953
:10EB200003D003E093E00720E4E702271B98007876
:10EB300040060ED58E484188C90506D510AA018B1E
:10EB4000128D914201D100214162002018A9087064
:10EB500094E0FF21013110A80186018D84480183D2
:10EB6000209901841D994162132085E0052C6ED304
:10EB7000417803780A021A4310A90A8594460922AB
:10EB800069460A720021009101222499D20311439F
:10EB90008AB2C178807809021B9B01435B1D6046E5
:10EBA00000F0F5FB18A90870002269460A720122DC
:10EBB000520210A90A86832802D0002805D099E0C5
:10EBC0006B48098D018302277EE06948006D0028AB
:10EBD00007D020461B99FFF789FB18A90870002869
:10EBE0004DD12B46324620461B9900F024FB0746A8
:10EBF00045E01B98022C4078009064D1002801D099
:10EC0000012860D10A2168460172009901731AAA8D
:10EC100000200099FFF73BFC014668464173002144
:10EC2000817302A83099F8F73AFF07460021684639
:10EC300001720121890210A80186022F08D04C48D8
:10EC4000006C8079002807D018A9087020E04BE0FC
:10EC500047490098088337E0002F03D0812018A986
:10EC6000087031E01AAA01200099FFF710FC18A9DA
:10EC70000870002803D119202870012030806846D0
:10EC8000007A002804D002A83099F8F708FF074658
:10EC9000002F2BD018E0062038E5229934480907C8
:10ECA00011D5012C0FD10B2269460A72C0888881C8
:10ECB0000021042003F03EF8082010A90886BFE6D2
:10ECC0002098400610D50327294810AA4188128EA3
:10ECD000114341805005400E04D01F9928980860C8
:10ECE0001F988480384693E404200FE518A8007824
:10ECF00000280ED0012028701B980078687010A89A
:10ED0000008DA870000AE87018A800782871052006
:10ED10003080174810AA4188128E91434180E1E764
:10ED2000FFB506469FB000201B9031780120884037
:10ED30001149124A084010A908860D494988914294
:10ED400003D0002804D0080702D5012023B0F0BD6D
:10ED5000219D00272F7020983C46018810A801842F
:10ED600018A8077100F00BFB6846077202A907E0BC
:10ED7000F81900200102000009F80000FFFF000060
:10ED8000FA48016401464031826C1A91097BC9003E
:10ED90000839571822994164307801282AD002286E
:10EDA00009D0032879D12878800980011D30287086
:10EDB000EE48B188C1803078022804D128788009D3
:10EDC00080011B30287001A8009010A8008CEB1C5B
:10EDD000C01E82B2B088002100F07DFC0028E1D185
:10EDE000B1886970090AA9706946888810A9C01C91
:10EDF00008842DE1717918A801713079012802D0B9
:10EE00000228CFD1E6E0D9487F2340881B01024683
:10EE1000184010AB1886802840D006DC102810D08F
:10EE200020280ED040280AD120E0FF38013859D0E0
:10EE3000FF3801386AD0FF38FF3802387ED0052409
:10EE400091E0D00601D5082000E010201B9004209E
:10EE5000694608720020888118A8009001953189C0
:10EE600019AB1CAA1B98FFF76BF977E0BF4B3289EF
:10EE7000188B82424FD10A221B92002973D101A91B
:10EE8000009110A9098C6B1C491E8AB2002100F068
:10EE900022FC18A908710B2017E0F6E0B34B328969
:10EEA000188B824237D10C221B9200295BD101A919
:10EEB000009110A9098C491E8AB21946098C6B1C55
:10EEC00000F009FC18A908710D202870694688888F
:10EED00010A9401C0884042069460872A348008BCE
:10EEE000888140E0A14A3389108B834213D11223D9
:10EEF0001B93002937D1536A002B05D00091128C47
:10EF000000F045FA18A9087113205EE0974832898D
:10EF1000038B9A4201D00424E7E016221B92026D73
:10EF2000002A09D1F268002A06D002651A98328AAE
:10EF300082821A9A0020D082002900E02FE012D1AC
:10EF4000B8883968FFF7D2F918A9087100280AD1E2
:10EF5000B8882B4618AA396800F06DF904460228D3
:10EF600018D0042C16D0B88800280FD06846007A34
:10EF7000002804D002A82299F8F791FD0446012048
:10EF800069460872386803900020B880002C5FD072
:10EF9000052C7BD06846007A032873D0A5E01820A2
:10EFA0001B90002905D0714831890183002101653A
:10EFB000D9E76E480246017E18320120FFF767FA52
:10EFC00018A908710028CED119202870012010A995
:10EFD0000884C8E71A98407B002856D0307AC000D1
:10EFE0001358001D0193105A1D9000291AD100F0EA
:10EFF000CAF9062069460872002000901D980F3853
:10F0000082B201988178437808021843019B00215D
:10F01000DB1C00F0BCF918A90871002269460A72CD
:10F02000832830D0002118A8017110A80184012183
:10F0300068460172019803901A981A99407B401E05
:10F0400048731A98807B002802D01A99401E887352
:10F0500010A8008E7F21090102468A431DD0434833
:10F060000022008811468300042002F0BEFD3F48C4
:10F070003178017110A94088098E08433B494880C6
:10F080000FE003E02BE002242FE00524374810AA0C
:10F090004188128E9143418027E034494A88824357
:10F0A0004A806846007A002805D03048416C02A8A2
:10F0B000F8F7F5FC044618A80079002815D01B982D
:10F0C0006870012028702948008BA870000AE87039
:10F0D00018A800792871052110A8018405E02348AB
:10F0E000416C02A8F8F7DBFC044600F04CF91F481D
:10F0F00040884005400E20D11A98807B00281CD102
:10F10000B888002819D0209910AA0988118422995A
:10F110000091396818AA219BFFF74FFA044602288C
:10F120000BD00120694608723868039002A8229922
:10F13000F8F7B5FC04460020B88010A8018C209890
:10F140000180204602E600B50022D243074997B06D
:10F150004A80042807D102226846027009790171A9
:10F160000021F8F79CFC17B000BD0000F819002042
:10F1700010B5394C03780022216C012B02D0022BF0
:10F1800044D126E00B78002B01D0042B03D10A7167
:10F19000226C03211170216C83880A79D200921DA0
:10F1A0008B52216C0A79D20008328918C2880A80F1
:10F1B000216C03890A79D2000A328B524289206C71
:10F1C0000179C9000C314252216C0879401C087148
:10F1D00020E00A74226C81889180216CC288CA80E8
:10F1E000226C01891181226C41895181216CC06896
:10F1F000C860616C206CF8F752FC0146022807D009
:10F20000206C007C002802D1002903D0812010BD91
:10F21000832010BD002010BD8178012909D100880C
:10F220000521C902884202D0491C884201D1002030
:10F2300070470520704710B51488844201D205201C
:10F2400010BD17241C701080421E491C581C05F06C
:10F250002BFD002010BD0000F819002010B58B78A0
:10F26000002B11D082789A4207D10B88002B0BD04B
:10F2700003E0091D8B78002B08D08B789A42F8D1D7
:10F2800003880C88A342F4D1002010BD812010BD5A
:10F2900010B5002902D001290DD102E00088000537
:10F2A00001E000888004800F07D001281CD00228CC
:10F2B00009D0032810D0812010BD002901D00320DF
:10F2C00010BD022010BDF5F719FE03280CD004284C
:10F2D0000AD0002806D009E0F5F710FE042803D074
:10F2E000022803D0052010BD002010BD0F2010BD46
:10F2F000F3B5C81C80080E46800081B0B04201D032
:10F300008620FEBDFE4C354626600198A080002078
:10F310002081E08014E0B807A978800D0843F949FE
:10F3200005F03CFDE088401CE080B80607D4208949
:10F33000401880B220810199081A8019A8600C3504
:10F340002F887807E7D40020A072FEBDEC480C227D
:10F35000C18800895143081880B2704770B51346C0
:10F36000E74A45189488AC4201D2842070BD1268E7
:10F3700010180A46194605F097FC002070BDE049B8
:10F38000012088727047DE49002088727047FFB5FF
:10F3900089B097040E460546BF0C029200F034FA7D
:10F3A000040021D0002069460873D548807A0128DE
:10F3B00012D001212046FFF76BFF002815D12078DD
:10F3C000400609D5022168460173058221884182E1
:10F3D0008682C7820C9806900298000407D5002701
:10F3E0003E46012501970CE001200DB0F0BD2078CC
:10F3F000A1788007800D0843C249019005F0CEFC3A
:10F400000D46029840040AD50198A84207D12088E9
:10F41000E1788005800F00020843B04201D3AE427C
:10F4200001D90720E1E7B81980B20290A84201D9BA
:10F430000D20DAE76846007B002804D003A8F8F71F
:10F440002AFB0028D1D10198A8420BD120880321A2
:10F450000902884302998905890F0902084320801F
:10F460000298E0701298002800D007800C980028BD
:10F470000CD02078000609D4A0683A4680190C996F
:10F4800005F012FC20881021884320800020ACE782
:10F49000FFB59B4D81B00E46E8882F680C21009087
:10F4A00048433C189749039805F078FC0A46288998
:10F4B000E11B84460C314018318880B28B0601D59F
:10F4C000002300E013461818AB8880B2834202D8AC
:10F4D000842005B0F0BD0098894D401C80B2E880C2
:10F4E00021800D99002900D00C600399A170E27071
:10F4F0002188039D8908AD058900AD0F29430325A7
:10F500002D02A9439505AD0F2D022943042529435A
:10F5100021800C99002900D0088001998978A17177
:10F5200001990988A1803178890601D50B9905E0F8
:10F530007349624492B20A81991AC919A1600021E3
:10F5400021733278920601D50020C2E700910B9B0F
:10F550000A9A0499FFF71BFFBBE7FEB5044600F0CB
:10F5600053F9070008D0664D641EE8880190A6B2E2
:10F5700028683446009015E00120FEBD0C2000995B
:10F580006043095A8A060BD489078A0D0099801CAA
:10F59000085C5C49104305F001FC2889401A288169
:10F5A000641CA4B20198A042E8D8EE800020387014
:10F5B000FEBD002803D0401E0880002070470120B7
:10F5C000704710B54E490288CB889A4201D38220F9
:10F5D00010BD0B680C21514359180B88CC789B0542
:10F5E0009B0F1B02234341608C7904738C884481F8
:10F5F000C3818968521C016102800281002010BD14
:10F60000012101827047FEB505460020C0430880F5
:10F6100068680F4681786846817068680188684626
:10F62000018000218171288A2C88A04200D30446E1
:10F630002C8234E0288A401C2882301D6968FFF73C
:10F640000DFE002829D139882F48814201D1601E42
:10F6500038806888A04227D33088F1788005800FF1
:10F660000002084302906946301DFFF7F7FD0028AD
:10F6700013D12989244881421AD000213046FFF74E
:10F6800007FE002809D12A890298824205D1E9683B
:10F69000B06805F0DCFA00280AD0641CA4B2204649
:10F6A00000F0B2F80600C5D1641E2C828220FEBD97
:10F6B0007C80B079B871B088B88030883881307873
:10F6C0008007810DB078014379810298B881B068D4
:10F6D00038610020FEBDFFB585B014460F46059881
:10F6E00000F092F8050037D00548BE05807AB60DC7
:10F6F00001281CD000212846FFF7CAFD002805E09C
:10F70000501A002001020000FFFF000022D12878DB
:10F7100040060CD501216846017005998180298831
:10F72000C18006814481F8F7B6F9002812D12888F3
:10F73000AA788107890D11438005800FEA780002BD
:10F740001043BE420AD0374A914207D3611E81421C
:10F7500004DD0B2009B0F0BD0120FBE7864201D992
:10F760000720F7E7801B82B2A24200D922460E98FA
:10F77000002800D002800898002804D0A8688119C9
:10F78000089805F091FA0020E4E770B514460D469C
:10F7900000F03AF800280DD001882980002C0DD007
:10F7A000017880788907890D01431E48814203D280
:10F7B000012002E0012070BD00202070002070BDFB
:10F7C00070B516460D4600F01FF804000DD02D88C8
:10F7D0002580FF2E16D0A807A178800D0843114977
:10F7E00005F0DCFA002E06D101E0012070BDFF31EA
:10F7F000FF31033189B2A170A80880008905890F03
:10F8000008432080002070BD0749CA88824207D380
:10F81000002805D00C22096850430C38081870479E
:10F820000020704701020000501A0020F0B585B09A
:10F830000E4605460020694608707078FE49C000F3
:10F8400003900C58FD4F002D0ED0022D73D0002CCC
:10F8500072D02078801E030005F0B4FC09837F7FFE
:10F860007F83797F77727F00002C03D1F4A16B2016
:10F8700005F0B7FB2078801E030005F0A3FC090605
:10F880005E5E5E19365E50545E003078062803D006
:10F89000EBA1762005F0A5FBB8687168806C0322A7
:10F8A00005F002FA012069460870002835D1CEE73C
:10F8B00030780C2803D0E2A1812005F092FBE068AB
:10F8C0000078002806D0B8687168806B102205F0B7
:10F8D000EBF928E0B8681021006B05F042FAB8682F
:10F8E000816A006B0A787168F1E730780D2803D0DF
:10F8F000D3A1942005F075FB042069460870716857
:10F900004878097800020843B9684A6A5178127841
:10F9100009021143484069468880084608E0C8A1AA
:10F92000AF2005F05EFB6846007800288FD068465F
:10F93000F5F7E9FA8BE727E01CE0C1A1B420F0E776
:10F94000B8686169006CFEF708F8A16900E0E16839
:10F95000B868006CFEF701F803E0B9A1E32005F0F8
:10F9600040FBB8682146006CFDF7F7FFB24A0399E7
:10F9700000205050022D07D0002D05D0012D03D0BE
:10F98000AFA1EF2005F02DFB05B0F0BD10B501785B
:10F990000124012902D0022910D112E04268A748AF
:10F9A000002182600170A4486C38C166016741671C
:10F9B0008167D28902214C3001F0DFF90024204612
:10F9C00010BDFF209EA1163005F00BFBF7E7F0B548
:10F9D00005469EA103C997B014911390002008A971
:10F9E000087595492A781031944C04912178059135
:10F9F0000126914FA168130005F0E4FB0CEF0730DE
:10FA00009AF0EDECEBEAE9E9E8EF20700124FF263B
:10FA10004F36054610A80570457001F0BFF907463E
:10FA2000012803D086A1304605F0DBFA10A938463C
:10FA3000FFF7FCFE2046641EE4B20028EAD10A204B
:10FA4000694608706846029501F086FA002803D0DE
:10FA5000FF207BA1583068E0002646E3C86A0078A2
:10FA6000C0072FD0012069460870684601F074FA7B
:10FA7000002804D0FF2072A16B3005F0B2FAA06814
:10FA8000006CFDF761FF050004D1FF206CA16E3012
:10FA900005F0A7FA08984078C0003D50062028706D
:10FAA000A068016869600069A8606448C01CE860DB
:10FAB000284601F051FA022804D0FF2060A17830D6
:10FAC00005F08FFAA068C06A00784007C4D501200D
:10FAD00069460870684601F03FFA002804D0FF200C
:10FAE00057A1803005F07DFAA068006CFDF72CFF6F
:10FAF000050004D1FF2052A1833005F072FA089866
:10FB00004078C0003D5006202870A06801686960F8
:10FB10000069A8604948401DE860284601F01CFAC9
:10FB2000022899D0FF2046A18D3005F05AFA93E7BC
:10FB3000A968002933D0694608712979012932D092
:10FB4000022904D0FF203EA1A73005F04AFA3A4826
:10FB500010221030A96805F0A7F837481030364950
:10FB6000203148602078C1062CD5EF210840207054
:10FB7000032069460870304810300290684601F052
:10FB80000DF90446022808D0002C06D0012C04D020
:10FB9000FF202BA1B83005F024FA69466FE101215E
:10FBA0006A461171DBE7244A04996C3AD0674860D1
:10FBB0008860C8600621A86803F002FF1E49103162
:10FBC0000860CAE720210843207045E7A1E15AE117
:10FBD00019E1E6E086E056E000E081E2886C4079D9
:10FBE0008009012804D0FF2015A1CC3005F0F9F9D7
:10FBF000A068017A002906D1416B406801F01DFA26
:10FC0000A16801200872012069460870684601F069
:10FC1000A3F9002804D0FF2009A1D73005F0E1F9AD
:10FC2000A068006CFDF790FE050004D1FF2004A140
:10FC3000DA3005F0D6F90DE0C81A0020B400002033
:10FC40007372635C736D2E630000000004411A88B8
:10FC500000A4800008984078C0003D500220287021
:10FC6000A068416B6960806CC01CA860284601F0E8
:10FC700073F9040004D0FF20FD49E23005F0B1F92A
:10FC800029462831FBE017226846027201220270E1
:10FC900080788208287992008007800F02436846A6
:10FCA0008270FB20024028794007C00F8000024389
:10FCB00068468270EA8882804A6C02A901F08EF957
:10FCC000002804D0FF20EA49F73005F08AF9052121
:10FCD00008A801756846017A0187A0680026406C73
:10FCE0000F9006E2012069460870684601F034F979
:10FCF000002803D0DE49DF4805F073F9A068006CE6
:10FD0000FDF722FE060004D18320D949800005F0CA
:10FD100068F9A068006CFDF717FE1290002804D166
:10FD2000D448D349801D05F05CF9D3488068006C45
:10FD3000FDF70AFE040004D1CE48CD49093005F094
:10FD400050F908984078C0003E500A203070287A58
:10FD500030716868C84DB060A868406C3061172089
:10FD600030731298B4617061304601F0F5F80446C2
:10FD7000022808D0002C06D0012C04D01120BC4948
:10FD8000400105F02EF92046316AFFF74FFD287833
:10FD900005210140042900D05EE6FB2108402870BF
:10FDA0002AE0059840084000207082071CD5FD22FB
:10FDB000104020700F206A46107017201071486C98
:10FDC0000290684600F0EAFF0546022808D0002DA0
:10FDD00006D0012D04D0A748A5493A3005F001F915
:10FDE00069462846FFF722FD2078052101400429B5
:10FDF000D2D1FB2108402070072008A908759E4831
:10FE00008078087628E6012069460870684601F087
:10FE1000A3F8002804D097489549543005F0E1F83C
:10FE2000A068006CFDF790FD060004D113209049F6
:10FE3000400105F0D6F890488068006CFDF784FD1D
:10FE4000040004D18B488A495A3005F0CAF8089852
:10FE50004078C0003E500720307087488068406876
:10FE600070606868F460B060304601F075F80400B6
:10FE700004D080487E49653005F0B3F8316A2046E9
:10FE8000FFF7D4FCE8E5012069460870684601F0F8
:10FE900063F8002804D0774875497A3005F0A1F856
:10FEA000089840781190A068006CFDF74DFD0600A1
:10FEB00004D151206E49C00005F093F8A068006C91
:10FEC000FDF742FD040004D16A486949823005F01B
:10FED00088F81198C0003E50C01929694160092076
:10FEE000307068687060A868B060A889B0816348A5
:10FEF00030611030B4617061304601F02DF8022895
:10FF000004D05C485A49903005F06BF81198287578
:10FF1000A2E55A4A00208C32107002206B461870FD
:10FF200001922879002801D0107098E052480323EC
:10FF30000C304068FB2703708378504A9B089B0075
:10FF40003B4083704B7A00271B07DB0F43708C32DA
:10FF500057600B7BC370CB7A1372537A0C7D5B08AE
:10FF6000E4075B00E40F23430C461534D460FD2402
:10FF70002340CC7EE407A40F234353720B461C336B
:10FF80001361477107718B7A3B4A9C070C32A40FAF
:10FF90001268012C04D19478A407A40F012C1DD061
:10FFA0009B089B008B7293785B0702D48B7A5B076C
:10FFB00028D54B7A13AF5B075B0FDC005B00E318BF
:10FFC000147864001B19DBB2DC083C5D5F077F0F0F
:10FFD0000623DB1BDC40A3079B0F14E04C7A53790C
:10FFE0006406640F23404371147906273C40047172
:10FFF000E4001C43204B5C7083789B089B005B1CD7
:020000040001F9
:100000008370D0E700238478FB273C408F7A7F07FA
:10001000FF0FBF003C4384704C7A6407640F047088
:100020005078012807D1487A000704D5032008A991
:10003000087502202DE0022B27D0012B2BD00F4B6F
:100040000020049AD86750609060D06018467C30D9
:10005000024610325060887AFB221040887268464F
:1000600000F09CFE040035D0012C34D0004907E09C
:1000700040FC000009020000B40000205C1A0020CF
:100080006520C00004F0ADFF25E0032008A9087535
:1000900001200876E3E77D4C0D21E01C04F061FEB1
:1000A000204610304460022008A908750E94A86804
:1000B000002807D000682060059975482022114368
:1000C0000170CCE705980007C9D57249724804F061
:1000D00088FFC4E7002669462046FFF7A7FB04E037
:1000E0006D486C49203004F07CFF08A8007D002892
:1000F00002D00DA8F4F707FF304617B0F0BDF0B5F9
:1001000097B00C46054600206946087060482F7875
:100110005E4E0178583E82683B0005F053F80BA80C
:100120008207263B4C6977778D9AA8002B20694679
:1001300008730CA903A8FDF73DFC002804D056481D
:100140005449413004F04DFF54490D9804F026FE07
:100150004E4801604E4869680C300160AA684260F0
:1001600001910820694608708AE08A0610D5DF22CE
:100170001140017003202070444810304168A16094
:100180004068002802D00020207175E00120FBE7C4
:10019000102254E02B20694608733C4903A85C39BF
:1001A000FDF708FC002804D03B483A496A3004F0C7
:1001B00018FF042019E02A2069460873102204A8B9
:1001C000696804F071FD102208A8A96804F06CFDAC
:1001D0002E4903A85C39FDF7EDFB002804D0392037
:1001E0002C49000104F0FDFE05202070666043E00C
:1001F0002A79002A02D001221143017005206946A4
:10020000087028798880A868029039E0D06A402375
:10021000018819430180D06B6968102204F044FD05
:100220002AE0FB2211400170062069460870A96887
:1002300068680291019023E0CB0703D002221143AA
:1002400001705AE70F20207017202071506CA060B9
:1002500012E0937A9B0706D0D26A44781388FF3461
:1002600001342343138004221143017004E00A483F
:100270000849BD3004F0B5FE684600780028E0D09B
:100280006846F4F740FE38E701207047D81A00208E
:10029000B400002040FC00001503000040420F00A5
:1002A00070B504780D460646230004F08BFF0B1C46
:1002B000181C1C1C1C07181C1C181C0000210520E5
:1002C00001F038FDB068007805280CD0FA4800220B
:1002D000008811468300052001F087FC03E000211F
:1002E000052001F027FD002D0ED0002028702946A2
:1002F0003046FFF704FFF1482978005D884201D1BC
:10030000032070BD022070BD00213046FFF7F7FECC
:10031000002070BD30B5E8494B68497A0A011146A2
:100320000C315C5C032C0CD0044600252034257174
:1003300025725C5CA500AA18641C5C5498500320CC
:1003400030BD062030BDF0B50446264620360D46A9
:100350003279012008218FB0002A0CD0012A21D047
:10036000022A2BD0032A04D12A78052A01D1297028
:1003700000200FB0F0BD01203071606800280AD065
:10038000A069017061684160216981606169C16033
:10039000FFF7C0FFEDE707202870206968606069FB
:1003A000A86009E029780729E3D1022030710520EF
:1003B0002870C248203868600320DAE729780529C8
:1003C000D7D1A08910280AD9103880B2A081A1689D
:1003D0001023091803A86A6800F054FE2DE01028C5
:1003E00004D0C1B20BAA1020A76809E0102322692B
:1003F000A16817E0491EC9B2401EC0B27B5C13540D
:100400000029F7D100280AD0401EC0B28021115423
:10041000002102E0401EC0B211540028FAD16269E6
:1004200010230BA907A800F02DFE102307A903A88D
:100430006A6800F027FE032030716068019003A80D
:10044000029005206946087029466846FFF728FF94
:100450008FE7F0B5044626460D4620363179012057
:100460008DB000290BD0012938D0022905D1297877
:10047000052902D10920287000200DB0F0BD217D92
:100480006846CA07D20F02738807C10F6846017415
:10049000012203A905A800F0EDFD04A9012205AF82
:1004A000481D00F0E7FD0722B81CE16800F0E2FDFE
:1004B00007A807220130216900F0DCFD6068019087
:1004C00009A80290102305AAA16800F0DBFD012015
:1004D0003071052168460170294621E029780529F7
:1004E000CBD1062203A8E16900F0C4FD04A80622CE
:1004F0000230A16900F0BEFD042106A800F0B2FDA3
:100500006068019007A80290102303AA696800F0B0
:10051000B9FD0220307105206946087029466846F9
:10052000FFF7BEFEA9E7F0B5074685B00D460020EF
:10053000694608703E466248203632798179133820
:1005400001240078130004F03DFE180DFEFDFCFBB5
:10055000FAF9F8F7F6F5F4F3F2F1F0EFEEEDECEB73
:10056000EAE9E8E7B968039100291BD0012269464E
:100570000A7003220A710A224A7139690291397993
:1005800000297DD0039A1278002A7AD00C2A78D2DA
:10059000130004F017FE0BEF09EF354D8498B0F10E
:1005A000EDECEF000020C8E30021062001F0C2FBC3
:1005B0003879072866D1424C133C2078022802D0B3
:1005C00000287FD101E00020207003980079C11F2E
:1005D0000A2901D30A2598E1607039480722C01F13
:1005E000039900F047FD0120307120700220694618
:1005F00008703348801F01903869401C029037E230
:1006000011293DD12E4C133C0228DAD16068617863
:10061000007A884201D9062577E1039926481022FD
:10062000491C303800F026FD03202070022045E1EF
:100630001129E6D1224C133C0428C2D10520207098
:1006400003991D481022491C203800F013FD062094
:100650003071786903210170626851684160164900
:100660002039816021460C31C160C91D0161017DC5
:10067000537A49084900DB07DB0F1943017502E093
:1006800070E354E384E1D3688361FD231940537A16
:100690009B07DB0F5B0019430175116976E10229A5
:1006A000AFD1002867D005206946087103984078CB
:1006B00048713869029051E32C1B0020445201001C
:1006C000DB00002082E011299BD1F74C06287DD168
:1006D000A0680399806B1022491C00F0CBFC062116
:1006E0006846017038690290002168460171FFF781
:1006F000D7FD072057E00B299BD1EB4C07287ED173
:10070000A0680399006B0222491C00F0B3FCA068AA
:100710000822406B039917E00EE116E3FDE2DDE2EB
:10072000C7E2BCE29EE267E248E241E21FE2F5E195
:10073000DFE1C8E1BEE1B1E1A5E16AE147E128E11D
:10074000DAE0BEE0AFE075E0C91C00F093FC0621E2
:100750006846017038690290002168460171FFF710
:100760009FFD204613304179490849003EE041E0B1
:100770001BE001E05CE0EFE2112991D1CA4C0828AE
:100780003DD1A0680399C06B1022491C00F072FC97
:10079000062168460170386902900021684601719F
:1007A000FFF77EFD09202070C9E208298CD1BE49DF
:1007B000092824D1039842788868016C0A7003994B
:1007C000406C0622891C00F055FC00E017E0062171
:1007D0006846017038690290002168460171FFF790
:1007E0005FFDB14813304179FD221FE041715EE2A7
:1007F0003071F2E11129C0D1AB490A2801D0082596
:1008000083E088680399806C1022491C00F032FC58
:10081000062168460170386902900021684601711E
:10082000FFF73EFDA04813304179FB221140DDE780
:1008300007256AE0297802297ED19B490128FBD14E
:100840006A684A6015780846002D5CD106216A4620
:1008500011703969029107211171029902240C70FB
:10086000CA785207520FCA704B795B075B0F4B7106
:100870008B795B075B0F8B71D20701D18A714A714B
:1008800005460A794078824200D26A70864807227B
:10089000133000F0EFFB00202C70307101466846E9
:1008A000FFF7FEFC4BE229780429C5D103286FD15C
:1008B00008227E48696800F0DDFB032030710420C7
:1008C000F2E129780429B7D1774F0328B4D17748CA
:1008D00008220830696800F0CDFB04203071786888
:1008E0004168002906D00321297000212971406840
:1008F000A86072E10320D7E1287803289CD12879E9
:1009000000281AD00546002D16D006216846017031
:100910003869029002216846017102980521017030
:10092000457000216846FFF7BBFC01216846017055
:1009300004210171457115E293E15B49A86849689A
:100940000028486001D15A48486005203071786914
:10095000032202704A684260544A8260524A0C3252
:10096000C260D21D0261027D4B7A5208DB07520041
:10097000DB0F1A430275CB688361FD231A404B7A63
:100980009B07DB0F5B001A4302750969C16130E107
:100990000DE12978092988D14349032885D104200C
:1009A00008700620694608703869029011200871A5
:1009B000029803210170401C1022696800F05AFB64
:1009C00000216846FFF76CFC00203071B7E1297800
:1009D000092993D1052891D134496A68203910201A
:1009E000401EC0B20B5C145CA34203D0002004255F
:1009F00030718AE70028F3D107203071786904212B
:100A00000170294949684968416028498160103965
:100A1000EEE028780A28BED10620694608703869B9
:100A2000029011200871029804210170401C1022CC
:100A30001E4900F01FFB00216846FFF731FC1A48F1
:100A4000102140786A68091AC9B2101800F00AFB30
:100A50006868019014481330C178C9070BD08179B8
:100A6000002902D14079002805D0082030711BE10F
:100A700029466846EFE0072069460870002168466D
:100A8000FFF70EFC5FE128780E2884D106486968DC
:100A900081608969407808700920A9E6C80701D0FB
:100AA0000A20FFE00F20A3E6C80000201C1B002046
:100AB0002452010028780F2879D1A8683861287954
:100AC00038730B20FAE628780428F5D1FC4C6968C5
:100AD000A0680822006A00F0CDFA0C203071786915
:100AE0000722B9690270A268D3684360126A826003
:100AF0007EE028780D28DFD1F14C6968A0680223D8
:100B00000269C06900F0BEFA0D20307178690621D3
:100B10000170A1688A684260096966E028780C283B
:100B2000CAD1E74C6968A0686278406A00F0A2FA0E
:100B30006078A2681021091A526AC9B2101800F030
:100B400091FA0621684601703869029011226846C0
:100B50000271029810220170A168401C496A00F0DD
:100B600089FA00216846FFF79BFB0E206EE028788B
:100B70000F2876D1062168460170386902900B2152
:100B800068460171029C0720CD4D2070A8680222A2
:100B9000C169601C00F06EFAA8680822016AE01CB6
:100BA00000F068FA00216846FFF77AFB7AE7C8E0B0
:100BB000880701D5102075E0132019E628780F2842
:100BC0004FD1A86838612879387311203071BC483A
:100BD000816848690078002801D00324CAE0786958
:100BE00006220270C9684160B6498160B549091D95
:100BF000C160FFF78FFB30E0B14880684169097838
:100C000000290CD129780C292BD1AD4C6968806A58
:100C1000102200F02FFAA16801204969087006210E
:100C20006846017038690290112168460171029886
:100C300008210170A249401C89681022896A00F0CD
:100C400019FA00216846FFF72BFB122030710921A9
:100C5000684601702946FFF723FB044601287DD032
:100C600088E06FE028780F286CD10620694608706C
:100C70003869029008200871029809210170904992
:100C800089680A78D207D20F427049680622801C10
:100C900000F0F0F900216846FFF702FB8CE74807F7
:100CA00005D514203071092069460870E0E6162049
:100CB0009EE528780F2851D1A868386128793873C3
:100CC000152030717869062101707D4989688A682C
:100CD0004260096981607B49891D89E728780C2871
:100CE00045D1774C6968A0681022C06A00F0C2F94B
:100CF0000620694608703869029011200871029830
:100D00000A210170A168401CC96A102200F0B2F9E2
:100D100000216846FFF7C4FAC9E7694813304079F3
:100D2000002810D0C10703D065480621017006E0F5
:100D3000800701D5082000E00A20614908700024DE
:100D400018E00BE013E0172052E55D49002805D0BC
:100D50000020307108700A206946087068460078E3
:100D6000002804D000216846FFF79AFA002454486E
:100D700000210170204605B0F0BD10B5524BFF2494
:100D80005C72586019721A80002204E0491EC9B2D0
:100D90000B010C33C2540029F8D110BDF0B54A4EF6
:100DA0000546717A01208DB0FF2971D00127727A32
:100DB000736811015C180C31595C8900091F645873
:100DC0006A7021780B0004F0FDF90B960709272CB7
:100DD00059888D4A4F5492002F707CE02146203173
:100DE0000A9109790120002902D0012967D10EE07A
:100DF0006068019005A802900D21C01C00F032F936
:100E0000032205A8A16800F035F90A984EE0297878
:100E1000052974D106215DE029462046FFF719FB1C
:100E200069E021462031069109790120002902D08C
:100E3000012964D10EE06068019007A802900822A1
:100E4000E16800F017F9082209A8A16800F012F97A
:100E500006982BE02978052951D10A213AE0294644
:100E6000204600F01AF946E029462046FFF76BFAC3
:100E700041E029462046FFF756FB3CE02146203161
:100E8000059109790120002903D0012937D11DE0FE
:100E900056E06068019007A802900822A16800F05F
:100EA000E9F8082109A800F0DDF8059869460771FE
:100EB0000520087029466846FFF7F2F91BE00BE0B1
:100EC000C80000201C5201002C1B00202978052995
:100ED00015D10B212970002011E02946204600F091
:100EE00023F908E02946204600F04EF903E02946A0
:100EF0002046FFF7C9F9002801D001280CD125624E
:100F0000717A736809010C315A5C521E1206120E76
:100F10005A5401D003204AE70328FCD0737A726840
:100F200019011D010D312C46515C7172FF270D34E2
:100F300017550C35545D002C02D0FF2903D1737274
:100F40000DB0F0BD21460C010D34145DFF2CF9D11C
:100F500009010D315354F3E770B5AD4C0546607A85
:100F6000214603464A6811E0010108460C30105C36
:100F700008E0401EC0B286008E199659AE4201D1DB
:100F8000042070BD0028F4D10D31505CFF28EBD156
:100F90009F480021007A01E0491CC9B2884204D967
:100FA0000E010C36965D002EF6D1884201D8052040
:100FB00070BD08010D30135461722846FFF7AAF97D
:100FC000032806D0617A626809010D31515C6172B3
:100FD00070BD28462830FFF7E1FE70BD10B50478DB
:100FE0000123012C14D10C78022C11D30B23137084
:100FF00083785B075B0F537002220A708088002899
:1010000005D0830000221146062000F0EEFD0023EB
:10101000184610BD0EB50022012105280AD0062869
:1010200007D1684601700221017142710021FFF76A
:1010300066F80EBD68460170F6E710B58EB00C4636
:1010400006216A461170019072480290001D0390BB
:101050006846FFF781FF102220460B9900F00AF83E
:101060000EB010BD002202E0491EC9B24254002950
:10107000FAD1704703E0521ED2B28B5C8354002A2F
:10108000F9D1704730B505E05B1EDBB2CC5CD55CB6
:101090006C40C454002BF7D130BD3EB5044620301F
:1010A0000D4602790121002A02D0012A3AD10FE02F
:1010B00061680191574908310291012101710520B0
:1010C0006946087029466846FFF7EAF8014629E0B4
:1010D0002878052826D169681022A06800F087F8D2
:1010E0006868C07B000606D54A4AA06810231832FB
:1010F0000146FFF7C7FF1022A168E06800F077F80B
:10110000A068C07B000606D5424AE068102318326A
:101110000146FFF7B7FF07202870A0686860E06805
:101120000021A86008463EBDF0B5044626460F469D
:1011300020363179012089B0002909D0012905D153
:101140003978052902D10C203870002009B0F0BD93
:10115000606803AD01900295022203A8A168FFF721
:1011600089FF0222A81CE168FFF784FF0C21281DDB
:10117000FFF778FF01203071052069460870394675
:101180006846FFF78DF8E1E710B5034620331C7978
:101190000122002C04D0012C10D0022C25D11EE0FD
:1011A00001211971C16806220A7040684860194817
:1011B000801C8860801CC86008460CE00C780C2CF1
:1011C00013D102221A71C268052313704968516055
:1011D000806890601046FFF79DF8024605E00878A9
:1011E0000B2802D10D2008700022104610BD10B54A
:1011F000002409E00B78521E5B0023430370401C5F
:101200000B78491CD2B2DC09002AF3D110BD0000D2
:101210002C1B00201C52010070B50D46040012D09A
:10122000002D10D02101284603F09BFD10225449C7
:10123000284603F039FD52480121083801804480D6
:101240004560002070BD012070BD70B54C4E00247B
:101250000546083E11E0716820014018817BAA7B99
:10126000914209D1C17BEA7B914205D10C222946EA
:1012700003F0EDFC002806D0641C30888442EADBD1
:101280000020C04370BD204670BD70B50D460600FD
:101290000AD0002D08D03A4C083C20886188401CB8
:1012A000884203D9042070BD102070BD3046FFF77E
:1012B000CCFF002801DB401C0AE0208861680001A7
:1012C00040181022314603F0EFFC2088401C20809B
:1012D0002870002070BD70B514460D001FD0002C82
:1012E0001DD00021A170022802D0102817D108E0DB
:1012F000687829780002084311D00121A17010807C
:101300000BE02846FFF7A1FF002808DB401CA07077
:10131000687B297B000208432080002070BD0120EB
:1013200070BD70B5054614460E000AD0002030701E
:10133000A878012807D004D9114908390A889042B1
:101340000BD9012070BD002C04D02878207028888B
:10135000000A50700220087010E0002C0CD0496880
:101360000001411810391022204603F09DFC287816
:1013700020732888000A607310203070002070BD30
:10138000EC00002073490968016000207047714932
:1013900008600020704701216F4A704B002803D07D
:1013A000012805D06E48704791630020187001E055
:1013B000D1631970002070476A49012008606848AD
:1013C000801C70470422684B6649002805D05A608B
:1013D000086901221043086108E0086940084000DC
:1013E00008619A605C490020C03188600020704725
:1013F0005C490622002808D0012809D002280DD017
:1014000003280FD05648401C70470869904302E0FB
:1014100008699043801C0861002070470869904368
:10142000001DF8E708691043F5E74E494A6A024390
:101430004A62002070474B494A6A82434A62002050
:1014400070474849496A0160002070474549CA69A8
:101450000243CA61002070474249CA698243CA6197
:10146000002070473F49C96901600020704730B5CE
:101470000546002072B601463A4A384C4032002DEB
:1014800011D00123012D0CD0022D02D0072062B60D
:1014900030BDA3706478002C01D09363F7E79163AB
:1014A000F5E7A170F9E7A170F9E72F4904208860FA
:1014B00029490020C03188602849012008702B4943
:1014C0000A688023120A12021A430A602849086037
:1014D000704722480078704770B5EFF31080C50759
:1014E000ED0F72B61D4C6078401C0006000E607057
:1014F00003D120A1CC2003F074FD6078012806D12F
:10150000A078002803D01749012040318863002DBE
:1015100000D162B670BD70B5EFF31080C507ED0F56
:1015200072B60E4C6078002803D112A1DC2003F0C3
:1015300058FD6078401E0006000E607006D1A0784D
:10154000002803D00749002040318863002D00D1D6
:1015500062B670BD0004004040000040FC00002066
:1015600004200000000500400003004000E400E00B
:1015700000E100E07372635C736F635F706F7765A7
:10158000722E63008107C90E002808DA0007000FD9
:1015900008388008B94A80008018C06904E08008D3
:1015A000B74A800080180068C8400006800F704766
:1015B000B44948788978884201D3401A02E0212250
:1015C000511A0818C0B27047AE492331487889785B
:1015D000884201D3401A02E02122511A0818C0B2F1
:1015E0007047A849463148788978884201D3401A23
:1015F00002E02122511A0818C0B27047A04810B565
:101600000C300168FF22120291430122D2031143E0
:1016100001609C490020233148708870233948704C
:101620008870463148708870974802F007FB9648EA
:10163000401C02F003FBF2F79DF900F015F910BD14
:1016400020207047B4E770B50C4605460026FFF72A
:10165000AFFF8C49A04214D30A46203A002320460B
:10166000641EE4B200280BD08878105C287088785B
:101670006D1C401CC0B288702128F0D18B70EEE741
:10168000012600F0F1F8304670BD202070479BE73E
:1016900070B50C4605460026FFF796FF79492331C1
:1016A000A04214D30A46203A00232046641EE4B226
:1016B00000280BD08878105C287088786D1C401C3E
:1016C000C0B288702128F0D18B70EEE7012600F0BF
:1016D000CBF8304670BD202101700020704710B556
:1016E0000446FFF77EFF2070002010BD70B50C4649
:1016F0000546FFF776FF63494631A04215D30A46F7
:10170000203A00232046641EE4B200280BD08878DB
:10171000105C287088786D1C401CC0B2887021282D
:10172000F0D18B70EEE7002400E0584C00F09CF8FC
:10173000204670BD70B50C460546212904D9FF200E
:1017400053A1473003F04DFC4C484068103840B27C
:10175000FFF718FFC6B20D20FFF714FFC0B2864294
:1017600007D2FF204AA14D3003F03BFC01E0F2F725
:1017700041F921462846FFF766FF0028F7D070BDE3
:10178000F8B5404E07462336B1787078212200F034
:1017900060F8354623353B4C00280ED0A1786078A0
:1017A000212200F056F8002814D0A9786878212268
:1017B00000F04FF800281AD025E032497078C91C93
:1017C0000F547078401CC0B2707021281BD10020CB
:1017D000707018E02B49607820390F546078401CF5
:1017E000C0B2607021280ED1002060700BE0254946
:1017F000687826310F546878401CC0B26870212880
:1018000001D100206870B1787078212200F021F8B1
:1018100000281DD0A1786078212200F01AF8002855
:1018200016D0A9786878212200F013F800280FD08C
:10183000F2F7C2F8144802F009FA0121490388427C
:1018400003D013A1C12003F0CCFB0F4802F016FA1D
:10185000F8BD401C884205D0904201D1002901D03A
:10186000002070470120704710B5074802F0EEF9DC
:10187000002801D1F2F78FF810BD000000ED00E064
:1018800000E400E0581B0020FF00002007200000BB
:101890007372635C736F635F72616E642E630000CA
:1018A00010B5284802F0CAF9002803D026A11D204F
:1018B00003F097FB2348401C02F0C0F9002803D036
:1018C00021A1212003F08DFB10BDF1B5224D6F68E1
:1018D00001261C4802F0BAF91A4C002803D1002650
:1018E000601C02F0CBF91D4A1D490120506000BF69
:1018F00000BF00BF00BF00BF00230B604B60009B18
:101900006B60106000BF00BF00BF00BF00BF086871
:10191000002802D148680028F9D048680028E4D19E
:10192000002E04D06F60601C02F090F907E0601C8C
:1019300002F08CF90028D3D1024802F09FF9002070
:10194000F8BDC2E7010100207372635C736F635FCF
:101950006563622E6300000000E5004000E0004087
:1019600000E1004030B5EFF31081CC07E40F72B610
:101970001D4A116910230D461D431561002C00D12D
:1019800062B61A4DC406E40E0120A0402C68044241
:101990000DD0C8060AD4EFF31080C007C00F72B68E
:1019A000116999431161002800D162B630BD20BF92
:1019B00040BF20BFEAE70E4908784A78401CC0B211
:1019C000904200D008707047084A094820BF40BFC5
:1019D00020BF4178037843701368002B02D103784D
:1019E0008B42F3D00020704700ED00E000E200E001
:1019F00003010020FEB5F64C07466068FF213E015A
:101A000081552178FF2913D0090108314158324608
:101A1000491E083209020192090A805800F0CEF9E5
:101A2000002802D02478254615E061682078885582
:101A30002770FEBDE64842680198115828010090C1
:101A40000830105800F0BAF9002806D1E0482C46BA
:101A5000416800980D5CFF2DECD1DD482101406804
:101A600085554754FEBD70B5D94A04460020157A05
:101A700053680AE00201561C9E5DA64203D10C3257
:101A80009A588A4204D0401CC0B28542F2D8FF2046
:101A900070BDF8B5CE4F3E7801F01AFE0146FF2E1C
:101AA00071D03401254678680835405900F086F930
:101AB00002280CD97868405901F0FDFD01F008FEBC
:101AC00001467868405900F079F902285BD8C0498E
:101AD0004868025D0A70A11C425C002A0CD0521EAC
:101AE000425441590122D20589180902090A41517B
:101AF0003046FFF77FFF30E0631CC25C0092221D7E
:101B000094468258002A10D001239B029A420FD992
:101B10009205920D43595703DB191B021B0A4351CF
:101B20006346C3589A1A920A09E0FF21C1540AE099
:101B3000435952039A181202120A42510022425487
:101B40003046FFF757FFA2480C344168C26800983E
:101B5000095980001258009890479D4C2078FF2822
:101B600011D0000161680830085801F0A4FD01F0AF
:101B7000AFFD01462078626800010830105800F07F
:101B80001DF9022886D3F8BDF8B51C4615460E4649
:101B90000746FF2B03D38FA1D42003F022FA8C48F1
:101BA000FF21C76045600472067401700022427014
:101BB000104604E00201521C401CA954C0B2A042CD
:101BC000F8D3F8BD70B5824C06466578207C854216
:101BD00003D380A1E72003F004FAE068A90046508F
:101BE0006078401C6070284670BDFFB581B01D460E
:101BF000FF2401F06DFD764F064679780198814209
:101C000003D874A1F52003F0ECF971480021037AA0
:101C1000406810E00A019446521C825CFF2A25D0DD
:101C2000019FBA4205D162460C328758029A974208
:101C30001ED0491CC9B28B42ECD8FF2C18D0210110
:101C40004A1C019B83540B460C33029AC250039BDF
:101C50005F4F0022012B0ED00B1DC25001239B02AF
:101C60009D4216D9AA05920D08D008E00C46E0E77F
:101C7000FF2005B0F0BD0B1DC550EFE71A4653031A
:101C80009B190E461B0208361B0AAA1A8351920A98
:101C900009E0002D00D101256B039B191D022D0ABF
:101CA0000B460833C550891C42543D463E782046B9
:101CB000FFF7A0FE2878B04214D000016968083010
:101CC000085801F0F8FC01F003FD29786A68090161
:101CD000083152580146104600F070F8022801D22F
:101CE000FFF7D7FE0198C4E770B50C46054601F032
:101CF000EFFC064621462846FFF7B5FEFF2817D021
:101D0000334D04012046696808300858314600F018
:101D100055F80121090340186968A41C095D400BAE
:101D2000002901D089020818002800D1012070BDC7
:101D3000002070BDF3B581B00F460198FFF793FE08
:101D4000FF282AD0224E3578726829460C4604E0D6
:101D5000844205D025462301D45CFF2CF8D11CE039
:101D6000FF2C1AD0A5421CD10801105C3070FF284E
:101D700015D000010830105801F09DFC01F0A8FCBE
:101D800001463078726800010830105800F016F8EB
:101D9000022806D2FFF77DFE03E00020FEBD01F021
:101DA00092FC39460198FFF79FFF22017168FF23DB
:101DB000541C0B558A5C2B01CA54FEBD401A00020C
:101DC0000121000AC905884200D90020704700009F
:101DD000A41B00207372635C736F635F74696D652D
:101DE000722E6300F0B500241C4A01211C4B08032D
:101DF000546018601B4B1C601B4C20601B4804691E
:101E0000E443E406E6170469761C10252C430461BC
:101E1000174C6160174D296000E020BF1F68002F3C
:101E2000FBD0002E03D107691026B74307619068E5
:101E30008005906801D5104A10436960A1600021B7
:101E400019600121084A09031160F0BD10B504466C
:101E5000FFF7C8FF2060002010BD000000C5004053
:101E600080E100E000C1004080E200E000ED00E021
:101E700000C3004000C0004000FCFFFF70B51F49D8
:101E80000A68002A17D000231D4601244A68521C04
:101E90004A60092A00D34D600E792246B2400E688E
:101EA00016420AD072B60B6893430B6062B649685B
:101EB0000160002070BD052070BD5B1C092BE5D3BF
:101EC0000FA1362003F08DF8F5E7012010498005B9
:101ED00008607047EFF31081CA07D20F72B6012174
:101EE00081400648036819430160002A00D162B6A8
:101EF000EBE70248002101604160704708010020C3
:101F00007372635C736F635F6576742E63000000A9
:101F100000E200E00120810708607047012081078E
:101F2000486070471048C068C00700D00120704763
:101F30000D488068C00700D0012070470A484069FA
:101F4000C00700D0012070470748C06970470649A4
:101F50008A69D20306D589698907890F814201D12F
:101F6000012070470020704700040040F8B5FE4C87
:101F7000207BE17A88421AD00126FC4D0027E07AC6
:101F8000215C14200A4642435019037C052B0FD0D4
:101F9000062B1BD0072B28D0437C012B33D0F4A178
:101FA000F64803F01EF8207BE17A8842E7D1F8BDBD
:101FB0000674E07A0A2807D0E07A401CE072491CD7
:101FC000C8B2AA5802210CE00020F7E70674E07AB4
:101FD0000A2808D0E07A401CE072491CC8B2AA580E
:101FE00003219047DFE70020F6E70674E07A0A282D
:101FF00007D0E07A401CE072491CC8B2AA580821F8
:10200000EFE70020F7E74774E07A0A2807D0E07A84
:10201000401CE072491CC8B2AA580721E1E7002021
:10202000F7E770B5D64D06206872D648002444778D
:10203000047738300473C472D34801F0FFFDD348ED
:102040000475EC72D249601E88606C71AC70EC70E3
:102050002C716C70CF48022104704470CE4804701B
:10206000047528300470491EFAD10120F1F744FDAF
:102070000020F1F741FD0120A871F0F75BFDC74892
:10208000F0F76AFDC64C2070C648F0F765FD607039
:10209000F1F7D6FC70BD10B5F1F7FDFCC04C20780F
:1020A000F0F778FD6078F0F775FDB54C207A0028E0
:1020B00005D0FFF730FAF0F7FCFD0020207210BDCC
:1020C00070B5AF4CA079002804D0A9A1B64802F0A1
:1020D00088FF70BDE07A002804D11320A4A140013C
:1020E00002F07FFF0126A6710025E572607A0421C7
:1020F000142250439D4A80180174A5488168491CE8
:1021000004D0691E81600120F1F7F6FC0020F1F790
:10211000F3FCF1F7D7FC01F02BFEF1F7DCFDA3484F
:10212000056005600120A249C0030860F1F750FE78
:1021300098480078022804D0032804D1E0780028C9
:1021400001D0A67000E0A570F1F7B1FD70BD0346A7
:1021500086490520142242435218203A127F002A51
:1021600004D0401E0006000EF4D1704714224243F2
:1021700051180A46403AD362012220390A77704743
:10218000012805D0032805D1002903D1002070477C
:102190000029FBD010B47A4C002363707D4A0028DC
:1021A00090700CD002280AD007291AD20B007B4469
:1021B0001B79DB189F441505070D0F111300D37011
:1021C00003E01B2000E03A20D0700120607010BCBA
:1021D00070475820F8E77720F6E79620F4E7B52017
:1021E000F2E710BC0020704710B56A484078F1F75C
:1021F00079FD80B210BD411E1422504310B55B4AD8
:102200008418203C042902D8207F002803D158A13B
:10221000684802F0E6FE207F012803D054A16648FA
:1022200002F0DFFE0020207710BD70B5554C607FB6
:10223000217F884201D1012500E00025F1F7EBFC68
:10224000F1F750FD617F227F914201D1012100E031
:102250000021A942EBD170BDF7B50646481E844661
:102260008EB0C0B2142204905043404A85182846CC
:102270000595007C2D1D07282AD13B4C0027E07ACC
:10228000227B824221D0235C049A934201D1012710
:1022900001E0002F04D00A2811D0421CA25C225475
:1022A0000A280ED0401C227BC0B28242EBD1002F04
:1022B0000BD0207B002806D0207B401E04E00022AB
:1022C000ECE70020EFE70A202073059A0120107444
:1022D00060462B4C04280FD814204143234808188B
:1022E0002038007F002807D00598007C012807D0FF
:1022F0001098807A012807D01DA1304802F071FEA5
:102300001098807A012871D10598184B007C02281A
:102310001AD0154C207B0A2874D0207BE17A401C0F
:10232000884204D1C92012A1800002F05AFE05990A
:1023300001204874217B04986054207B0A2865D0D2
:10234000207B401C20731CE1607A049A0146904275
:1023500006D0014614277843C018807C9042F8D1FB
:10236000627A824235D12BE0B01C0020C01C0020D4
:102370007372635C72656D2E63000000D50500000A
:10238000441D0020781C0020501D0020981C0020B7
:10239000241D002012010020D01C0020931A0100EF
:1023A000100100206D1F01007F02000000F50040B9
:1023B00080E200E0CD020000CE0200001703000022
:1023C000617A14225143C918897C61720121A1727A
:1023D00007E014224243D21814277943927CC9188B
:1023E0008A74142206215043C01881741098007A10
:1023F000062819D203007B441B79DB189F4408127E
:10240000100E0C0AE07A00288CD090E7002099E7A3
:1024100000210FE0B4210DE073210BE0322109E02F
:102420000A2107E0062105E0FF20FE49E23002F024
:10243000D8FD0021109802910068401A2860109978
